:100000000C948C080C94BD080C94BD080C94BD088D
:100010000C94BD080C94BD080C94BD080C94BD084C
:100020000C94BD080C94BD080C94BD080C94BD083C
:100030000C94BD080C94BD080C94BD080C94F953A5
:100040000C94BD080C94BD080C94BD080C94BD081C
:100050000C94BD080C94BD080C94BD080C948A5FE8
:100060000C94BD080C9494590C946A590C94BD08D6
:100070000C94BD080C94BD080C94BD080C94BD08EC
:100080000C94BD080C94BD080C94BD080C94BD08DC
:100090000C945A5A0C94CA590C94115A0C94BD08D9
:1000A0000C94BD080C94BD080C94BD080C94BD08BC
:1000B0000C94BD080C94BD080C94BD080C94BD08AC
:1000C0000C94BD080C94BD080C94BD080C943459D4
:1000D0000C940A590C94BD080C94BD080C94BD08EE
:1000E0000C94BD08520A070A150A520A520A600AFD
:1000F0006E0A4C0A520A520A630D680D6D0D770D97
:10010000810DFA0D8B0D930D9B0DA50DAF0DB90D46
:10011000C80DD20DFA0DDC0DE60DF00DF20FE40F57
:10012000E40FF20FF20FF60F04100410F20FF20FAB
:10013000FD14D814181518151815181518151815B4
:100140001815181518156711361457145014411442
:100150001815181518151815181518151815EC1464
:10016000041BF81AF81A041B041BDF1AEC1AEC1A09
:10017000041B041B782165216521782178217821D1
:100180008321832178217821613364337C33933355
:10019000DC33EF330F345B415B415B415B415841E2
:1001A00058415F415F415F415F415F415F415F4156
:1001B0005F41584158415F415F415F415F415F414D
:1001C0005D415B416A5E665E665E6A5E6A5E6A5E4D
:1001D000735E345E6A5E6A5ECD5ED05EBF5EC35E95
:1001E000C95E075FD45ED85EDE5EE25EE65EEC5E10
:1001F000F05EF45E075FFA5EFE5E025F0763423602
:10020000B79BD8A71A39685618AEBAAB558C1D3CA7
:10021000B7CC5763BD6DEDFD753EF6177231BF006B
:100220000000803F08000000BE922449123EABAAA5
:10023000AA2ABECDCCCC4C3E00000080BEABAAAA00
:10024000AA3E00000000BF000000803F0000000048
:1002500000084178D3BB4387D1133D190E3CC3BD81
:100260004282AD2B3E68EC8276BED98FE1A93E4C2E
:1002700080EFFFBE01C4FF7F3F00000000000C9430
:1002800057140C945F410C94075F0C94F8510C9434
:1002900028310C94345E0C94025F0C9420320C9440
:1002A000F0570C9450470C949C420C94041B0C94F3
:1002B0009C2D0C94810D0C94A5420C941A520C9414
:1002C0007C330C940E520C94AE450C949B310C94E0
:1002D000F00D0C94A9520C94630D0C94150A0C9417
:1002E0009D470C9418520C9458410C94CE570C9482
:1002F000520A0C949B0D0C945D410C94D45E0C94AA
:1003000004100C94B5560C94AF0D0C9446520C94FA
:1003100073310C9469520C9436310C944E320C9417
:10032000AB570C947D460C94F7440C9467350C94B1
:10033000600A0C94E40F0C940C4C0C94F45E0C9436
:10034000B90D0C946D0D0C9497470C94F81A0C94FD
:10035000E60D0C94B45B0C945E480C9478420C94BB
:1003600052440C94A4420C94DF1A0C946D520C94D9
:1003700068560C94EC5E0C94B95B0C94E1460C94BA
:1003800005570C940F340C94F60F0C94DC330C943A
:1003900018150C945E320C94F20F0C94665E0C945B
:1003A000BC5B0C94D20D0C948F450C941A490C94A0
:1003B00070420C9478210C9441140C9493330C9457
:1003C00020270C94C35E0C94A50D0C9431320C9430
:1003D0004C0A0C9450460C949C480C94EC140C94CD
:1003E000BF080C94CD5E0C94F05E0C9434530C94C6
:1003F000C95E0C94DC0D0C94D05E0C94FD140C942E
:100400006A5E0C9452570C9464330C9461310C94D2
:1004100091420C9408490C942D680C94D8140C94B7
:1004200065210C94AB320C9492560C94C7230C9417
:100430005A420C94B85B0C948B0D0C94CF470C94DF
:10044000070A0C94D85E0C94DE5E0C94EC1A0C94A3
:10045000E9300C94680D0C94FD550C94EF330C941A
:100460005B410C9460430C94C80D0C94E65E0C94B4
:1004700088420C9474420C9406310C94735E0C9474
:1004800083210C94542A0C9461330C94502A0C94BC
:10049000582A0C94E25E0C9487520C94FA5E0C94E9
:1004A000770D0C9436140C9444440C94D0300C9476
:1004B00059420C94930D0C94FA0D0C94BF5E0C945D
:1004C000EB420C94BA470C946E0A0C94DA300C94FC
:1004D000D7450C94A9570C94FE5E0C94A2310C9451
:1004E000C3560C9450140C94A1560C946711636479
:1004F000696E6F70737578585B003D00564323003A
:1005000020636D643D003D0056435F686561742360
:10051000003D0050696E3A003D0050696E3A00207F
:1005200048616C7465640A003D00526573746F72B3
:1005300065643A20003A204E6F2073746F726564D0
:100540002076616C756573202D2064656661756C1D
:10055000740A00466F7263652057686974650A0003
:10056000416C7265616479204163746976650A0043
:100570005475726E696E6720584F4E0A00584F4688
:100580004620736B69707065642E2050726576200A
:10059000636D643A005475726E6564206F66662000
:1005A00066726F6D3A00526573746F72656420668F
:1005B000726F6D3A003E20003C00205061723D2079
:1005C0000020436D643D00205375623D0020497456
:1005D000656D3D00204D454D3D00476F74204950ED
:1005E00020616464726573733A00276970205B69E7
:1005F000705B2C646E735B2C67775B2C7375626E1B
:1006000065745D5D5D5D27202D20736574207374B6
:10061000617469632049500A004661696C65642011
:10062000746F20636F6E66696775726520457468C4
:1006300065726E6574207573696E67204448435017
:100640002E20596F752063616E2073657420697068
:10065000206D616E75616C6C7921005374617274E8
:10066000696E67206C616E00246E6F646573002490
:10067000666F726D61740024646174617479706571
:1006800000302D31303000696E7465676572006826
:10069000737600636F6C6F72004F4E2C4F46462C82
:1006A00048414C542C524553542C584F4E2C584FC3
:1006B00046462C544F47474C4500656E756D0066A5
:1006C0006C6F617400322E312E300024686F6D69BA
:1006D0006500757074696D652C6672656568656125
:1006E0007000366661363631365F323031392D3042
:1006F000332D3233004C69676874487562200024DA
:100700006E616D6500726561647900207472792094
:10071000616761696E20696E2035207365636F6E55
:100720006473006661696C65642C2072633D0041EE
:1007300077616974696E6720666F72207265746193
:10074000696E656420746F7069637300636F6E6EA9
:1007500065637465642061732000202E2E2E0020B6
:10076000757365723A003A000A417474656D70746D
:10077000696E67204D51545420636F6E6E656374CB
:10078000696F6E20746F2000247374617465006457
:100790006973636F6E6E6563746564005573696E2B
:1007A00067204D5154542070617373776F726420C9
:1007B00066726F6D20636F6E666967004465766967
:1007C0006365204E616D653A00526562696E642012
:1007D000737563636573732E20495020616464727E
:1007E0006573733A004572726F723A20726562697E
:1007F0006E64206661696C0052656E657765642081
:10080000737563636573732E20495020616464724D
:100810006573733A004572726F723A2072656E6545
:10082000776564206661696C004E6F206C696E6B41
:1008300000416363657074696E6720636F6D6D61FD
:100840006E64732E2E2E0A003E3E3E004E6F204DEB
:10085000414320636F6E666967757265643A207301
:100860006574206669726D776172652773204D41EA
:10087000430A004D6F6462757320706F6C6C696E13
:1008800067206572726F723D002D0020504920561E
:10089000616C203A004D6F6462757320706F6C6CF0
:1008A000696E67206572726F723D002D0020464DA3
:1008B0002056616C203A004D6F6462757320706F32
:1008C0006C6C696E67206572726F723D00205661B4
:1008D0006C3A20004D423A20004E6F7420737570C0
:1008E000706F727465642072656720747970650A30
:1008F00000496C6C6567616C20617267756D656E2F
:1009000074730A00757074696D6500667265656858
:100910006561700024737461747300200020000A04
:10092000667265653A00202D746172676574207A7D
:100930006F6E652D00204F464600204F4E00204F21
:1009400046460020636D643A00204375723A0020E9
:100950005365743A0020457870697265640A0052E4
:1009600065747279696E6720434D440A004E6F7456
:1009700020737570706F727465642072656720747F
:100980007970650A00293A0028543A003D3E004D2E
:100990006F64627573206F70206661696C65640AAC
:1009A000003D00494E3A007267620063737600684A
:1009B00065617400766F6C00706F776572007365A7
:1009C00074706F696E74006D6F64650074656D702E
:1009D0000073657400536574436D643A002056617A
:1009E0006C3D002053746F726520004445435245AE
:1009F00041534500494E4352454153450066616CA1
:100A00007365007472756500584F464600584F4E26
:100A10000048414C5400544F47474C450052455301
:100A200054004F4646004F4E00636F756C64206E55
:100A30006F742070617273653A2000557064617440
:100A400065640A002B002D00485454502F312E317C
:100A50002025690020485454502F312E310D0A486A
:100A60006F73743A2025730D0A4163636570743A9D
:100A7000202A2F2A0D0A436F6E6E656374696F6EAC
:100A80003A20636C6F73650D0A0025730020000D1A
:100A90000A00474554002074727920616761696ECD
:100AA00020696E2035207365636F6E64730A00667B
:100AB00061696C656420746F20636F6E6E6563742A
:100AC000004552524F523A20536572766572207239
:100AD000657475726E65642000446F6E652E0A0041
:100AE0004170706C79696E672E0A00436F6E66699B
:100AF000672070617273696E67206661696C6564F6
:100B00000A00676F7420436F6E6669670A00436F5F
:100B10006E666967205552493A20687474703A2F9E
:100B20002F006C617A79686F6D652E7275000A28E6
:100B30002D29524553544152545F4C414E5F4F4E04
:100B40005F4D5154545F4552524F5253000A282D65
:100B5000294841524452455345542C207573696EBF
:100B60006720736F6674000A282D29434F554E5431
:100B70004552000A282D29444854000A282D294F9F
:100B800057495245000A282B294D4F4442555300DE
:100B90000A282B29444D58000A282B294453323463
:100BA00038322D313030000A282B294672656552C3
:100BB000616D207072696E74696E670064653A6178
:100BC000643A62653A65663A66653A6564000A4663
:100BD00069726D77617265204D4143204164647292
:100BE00065737320006C617A79686F6D652E72751C
:100BF000000A436F6E666967207365727665723AA4
:100C0000000A282B295741544348444F47003230AB
:100C1000313130334C0020432B2B207665727369C1
:100C20006F6E3A00366661363631365F32303139B2
:100C30002D30332D3233000A4C617A79686F6D653F
:100C40002E7275204C6967687448756220636F6EF8
:100C500074726F6C6C657220000000200023002607
:100C60000029002C002F00320000010000030106C3
:100C70000109013D00494E3A002F00496E3A20001B
:100C800000002200250028002B002E003100340037
:100C900002010000050108010B0100000A0B020916
:100CA0000C0D0E0807030401000000000000000006
:100CB0000000000000000000000000000000000034
:100CC00000000000000012111000000000000000F1
:100CD0000000000000000000000000000000000014
:100CE00000002100240027002A002D0030003300DE
:100CF00001010000040107010A010102102020087F
:100D00000810204010204080020102010804020166
:100D100001020408102040808040201008040201D5
:100D2000800402018040201008040201080402012E
:100D300001020408102040800102040810204080B5
:100D400005050505070508080808020202020A0A47
:100D50000808040404040101010101010101030365
:100D6000030303030303040707070C0C0C0C0C0C10
:100D70000C0C0202020206060606060606060B0B0D
:100D80000B0B0B0B0B0B43757272656E74204C4191
:100D90004E20636F6E6669672869702C646E732CD1
:100DA00067772C7375626E6574293A000A5573650E
:100DB00020746865736520636F6D6D616E64733A4E
:100DC000202768656C7027202D2074686973207453
:100DD0006578740A276D61632064653A61643A62DC
:100DE000653A65663A66653A303027207365742047
:100DF000616E642073746F7265204D41432D616490
:100E0000647265737320696E20454550524F4D0AD8
:100E1000276970205B69705B2C646E735B2C67774D
:100E20005B2C7375626E65745D5D5D5D27202D20A2
:100E3000736574207374617469632049500A277361
:100E400061766527202D207361766520636F6E665D
:100E5000696720696E204E5652414D0A27676574B6
:100E600027205B636F6E66696720616464725D272B
:100E7000202D2067657420636F6E66696720667237
:100E80006F6D207072652D636F6E66696775726530
:100E9000642055524C20616E642073746F7265201B
:100EA000616464720A276C6F616427202D206C6F67
:100EB000616420636F6E6669672066726F6D204E95
:100EC0005652414D0A2770776427202D20646566AD
:100ED000696E65204D5154542070617373776F7241
:100EE000640A276B696C6C27202D2074657374204D
:100EF0007761746368646F670A27636C6561722742
:100F0000202D20636C65617220454550524F4D0A7B
:100F1000277265626F6F7427202D207265626F6F74
:100F20007420636F6E74726F6C6C657200536F66C1
:100F300074207265626F6F74696E672E2E2E004486
:100F40004D58696E2042756666657220616C6C6FE3
:100F5000632065727200496E697420696E2063684F
:100F60003A000A6D71747420000A6D6F64627573C3
:100F700020000A696E7075747320000A6974656DCB
:100F80007320000A436F6E666967757265643A0084
:100F90002C003D0050696E3A00444D58206F757426
:100FA00020737461727465642E204368616E6E658F
:100FB0006C733A2000444D5820696E20737461723E
:100FC0007465642E204368616E6E656C733A000A26
:100FD0004C6F616465640A000A6C6F61642066612D
:100FE000696C65640A000A4E6F2073746F726564E1
:100FF00020636F6E6669670A006C6F6164696E6773
:1010000020436F6E666967000A7265717565737457
:10101000204D51545420436F6E66696700536176CA
:10102000656420746F20454550524F4D00536176E2
:10103000696E6720636F6E66696720746F2045452F
:1010400050524F4D2E2E0053617665640A0045457F
:1010500050524F4D20636C65617265640A005061A7
:101060007373776F726420757064617465640A00CD
:101070002C20002E00696E00735F6F7574006D790F
:10108000686F6D6500436F6E6E65637465642E00F6
:10109000436F6E6E2E2061626F72746564003E3E17
:1010A0002000496E76616C696420636F6D6D616EBE
:1010B00064004163746976650A0047727020636852
:1010C00065636B3A0A002D3E005075623A20005568
:1010D0006E6B6E6F776E20636D64200A00537461CF
:1010E0007475732064656666657265640A00536B87
:1010F000697070696E672E2E004F4F4D21005D2084
:10110000000A5B003A00436F6E666967757265643A
:10111000204D41433A002D6811241FBECFEFD1E28C
:10112000DEBFCDBF00E00CBF15E0A0E0B2E0EAE713
:10113000F2EF00E00BBF02C007900D92A632B1079C
:10114000D9F72AE0A6E2B5E001C01D92A13CB207A2
:10115000E1F718E0CCE8D8E000E006C021970109EB
:10116000802FFE010E941A74CB38D10780E0080757
:10117000A9F70E94D45F0C943B790C9400002F9245
:101180003F924F925F926F927F928F929F92AF9217
:10119000BF92CF92DF92EF92FF920F931F93CF9364
:1011A000DF93CDB7DEB76B970FB6F894DEBF0FBEF7
:1011B000CDBF6C013B015B8B4A8B5901088BFF8AC9
:1011C000EE8ADC011296ED91FC911397E080F1809C
:1011D000FE0131961F010091B50A1091B60A011562
:1011E000110511F401EC1AE064ED75E087EA97E06F
:1011F0000E942E58A101401B510B052E000C660BBE
:10120000770B2AE087EA97E00E9467586DEC75E05B
:1012100087EA97E00E942E58B70187EA97E00E947C
:10122000FC5867EC75E087EA97E00E942E586E89BB
:101230007F8987EA97E00E948F3E61EC75E087EA3C
:1012400097E00E942E58B30187EA97E00E948F3EF4
:101250006AEB75E087EA97E00E942E58D601129655
:101260008D919C911397892B09F43BC61B861A8696
:101270001D861C861F861E86A114B10469F1850196
:101280004E01BAE08B0E911CE12CF12CEA89FB890E
:10129000EE16FF060CF5F3E0EF16F104E9F0D801C5
:1012A000AD90BD908D01F401A192B1924F0168EB18
:1012B00075E087EA97E00E942E58B50187EA97E02B
:1012C0000E948F3E65EB75E087EA97E00E942E58FA
:1012D000FFEFEF1AFF0ADACF87EA97E00E94F8588B
:1012E00060E070E0C6010E9417282C0124E062161D
:1012F000710451F037E06316710459F183E0681608
:10130000710409F053C007C0C6010E94F75D892B24
:1013100009F02AC1EBC5D60118968C91873009F4E3
:101320001FC360E0C6010E946A28853009F0DBC552
:1013300066EA75E087EA97E00E942E5865E070E063
:1013400087EA97E00E948F3E87EA97E00E94F8586C
:10135000CDC5F6018085873009F402C360E0C6017F
:101360000E946A28082F10E0863081F465E975E054
:1013700087EA97E00E942E58B80187EA97E00E941A
:101380008F3E87EA97E00E94F858EEC06DE775E05F
:1013900087EA97E00E942E58B80187EA97E00E94FA
:1013A0008F3E87EA97E00E94F8589DC5F2E06F16DD
:1013B000710409F4D9C04CF46114710489F031E06E
:1013C0006316710409F019C1ACC085E06816710498
:1013D00009F4EBC096E06916710409F48AC00DC1E6
:1013E000D60118968C91853021F06EE0C6010E94DE
:1013F0004528F601808590E08A30910508F06EC09E
:10140000FC018827EE58FF4F8F4F0C941A748C857F
:101410009D85892B51F42A893B892330310591F42C
:101420008FE7D60118968C9304C0EA89FB8933971D
:1014300049F44A855B850C851E85B801C6010E946A
:10144000BB2717C0C6010E94F3277B01082F1A850E
:10145000AB01B801C6010E94BB27EA86FB86802F3C
:10146000000F990B9D878C87812F110F990B9F87F8
:101470008E87F889FF2371F101E09E01265F3F4FBF
:1014800043E050E060E070E0C6010E94FB5C23E0B6
:1014900030E03B8B2A8B22C04A855B850C851E85FC
:1014A000B80114C03889332359F001E09E01265F4A
:1014B0003F4F41E050E060E070E0C6010E94FB5CFD
:1014C0004A855B85052E000C660B770BC6010E94D2
:1014D000BB2704C083E090E09B8B8A8B0E947E5FD9
:1014E000609326057093270580932805909329051E
:1014F00084C0C6010E94F75D892B39F460E775E06E
:1015000087EA97E00E942E580CC060E675E087EAF3
:1015100097E00E942E58D60118968C91873009F0DA
:10152000E2C4F6018085813009F00AC560E0C60199
:101530000E946A28813009F003C50E947E5F0091F5
:101540002605109127052091280530912905DC01F9
:10155000CB01801B910BA20BB30B853F9140A105E2
:10156000B10508F0C7C4ECC460E0C6010E946A2857
:101570008530B9F01B861A861D861C861F861E863E
:1015800062E0C6010E944528F889FF2351F000E07F
:1015900020E030E040E050E062E070E0C6010E94F0
:1015A000FB5CA2E06A2E712C28C0C6010E94F75D88
:1015B0001816190614F51B861A861D861C861F86AA
:1015C0001E8660E0C6010E946A28863011F462E03F
:1015D00001C065E0C6010E94452800E020E030E03F
:1015E00040E050E062E070E0C6010E94FB5C6FE109
:1015F00075E087EA97E00E942E58EC84FD84C701CD
:101600000F2C000CAA0BBB0B888F998FAA8FBB8F56
:10161000AE85BF85BD8BAC8B2FEF30E00E9431745F
:10162000F4E68F2E912CA12CB12CA50194010E94DF
:10163000D9738901F6018085843009F47FC150F4A3
:10164000813009F44CC0F0F1823089F1833009F423
:10165000D6C146C4883009F47EC338F4863009F414
:10166000A6C1873009F03CC47BC1893009F4E6C2C9
:101670008F3709F035C460E0C2010E94E55460E094
:10168000C20101960E94E55460E0C20102960E94E8
:10169000E554AE85BF852FEF30E00E943174A5017F
:1016A00094010E94D973622FC201039644C12FEFA7
:1016B00030E0D7010E943174A50194010E94D973D2
:1016C000D22E78C0AA85BB852FEF30E00E943174FE
:1016D000A50194010E94D973622FC2012CC192010D
:1016E0002D5F3F4F390132E3E316F1040CF049C09E
:1016F00082E390E08E199F09EC89FD898E9FD001CD
:101700008F9FB00D9E9FB00D11242FEF30E00E94EF
:10171000317428E833E140E050E00E94D973622F31
:10172000C3010E94E5540C851D852EEF31E0D801E0
:101730000E943174E2E3CE2ED12CE12CF12CA701D2
:1017400096010E94D973AE85BF850E942974A501B8
:1017500094010E94D97349015A019801A5E6BFEF8F
:101760000E942974A70196010E94D973DD24DA949E
:10177000D20E84010F3F1105E9F0E4F00FEF10E005
:1017800019C0288D398D4A8D5B8D2253310941094D
:101790005109ABE9B0E00E94F87322E330E040E089
:1017A00050E00E94D97364E6D62ED20E60E0C301E9
:1017B0000E94E554AA85BB852FEF30E00E9431746A
:1017C0002DE631E040E050E00E94D973322F122F15
:1017D0001F71110F110F812F880F15E5682F619F61
:1017E000060E60E0611D1124922F9074207237FD67
:1017F00024C091110CC0211104C0862F8095F62EB3
:1018000014C055E5F52EF60E10E06BEA36C0211136
:101810000FC0182F3AEA139F010E10E0111D11247A
:101820008BEA811B4AEAF42EF60E682F10E025C0E1
:1018300080E0F62EF094162F0FC0911112C02111E6
:101840000DC0182F2AEA129F010E10E0111D11245D
:101850003BEAF32EF11A1B5A60E00FC0162F1095C9
:101860000BC0211104C085E5860F1BEA03C08AEA7C
:10187000860F90E0161B682FF12CFFEFDF1609F49E
:101880002AC0DD2009F423C0662329F02D2D629F94
:10189000060E60E0611DFF2039F03F2D2D2D329F97
:1018A000030E30E0311DF32E112329F03D2D139F3F
:1018B000010E10E0111D11242D2D2095229F020EE6
:1018C00020E0211D1124620FF20E120F04C01FEF41
:1018D000FF24FA946FEF0F3F09F422C020E00023A9
:1018E00021F0009F212D09F02F5F2223B1F0662304
:1018F00021F0629F060E60E0611DFF2031F03F2D58
:10190000329F030E30E0311DF32E112321F0129F80
:10191000010E10E0111D112403C010E0F12C60E055
:10192000C2010E94E5546F2DC20101960E94E55448
:10193000612FC20102960E94E554D2C2E480F58074
:10194000F7018085853009F0CBC2C7010E944B4268
:10195000A82EB12CF2E0AF16B1040CF00FC4C0C237
:10196000D6011496ED91FC9115978085853009F08C
:10197000B7C2C680D780C114D10409F4B1C2F60140
:1019800061857285C1010E94241EEE88FF88088946
:101990009E01265F3F4F4A895B89B301C1010E94C6
:1019A000BF08D6011296CD90DC901397E4CFF42CAB
:1019B00061E0842D0E94085F11E000E0B1E06B1649
:1019C000710429F0E6E06E16710409F010E0612F51
:1019D0008F2D0E94B03C6AE175E087EA97E00E9493
:1019E0002E58B20187EA97E00E948F3E68E175E0C9
:1019F00087EA97E00E942E58612F702F16C157FE7C
:101A000006C051944194510801E010E002C000E08A
:101A100010E0F42C61E0842D0E94085F8091A10009
:101A2000887F8093A10080919100887F80939100AE
:101A30008091A10082608093A100809191008260DA
:101A400080939100AA85BB85012B99F0CD01BB0F36
:101A5000AA0BBB0B9C01AD01245631094109510968
:101A6000AFEFB0E00E94F8732CE93FEF4FEF5FEF6C
:101A700008C02FEF30E00E94317424E630E040E0EF
:101A800050E00E94D973890161E08F2D0E94085FA8
:101A90000115110509F4B1C00F3F110509F4AFC0DC
:101AA000F201FF27E656F34FE4918E2F90E0FC0100
:101AB0003197E231F10508F09DC08827E458FF4FC7
:101AC0008F4F0C941A7484B5806884BD07BD9BC089
:101AD00084B5806284BD08BD96C080918000806816
:101AE0008093800010938900009388008CC08091BF
:101AF000800080628093800010938B0000938A00A6
:101B000082C08091800088608093800010938D0057
:101B100000938C0078C08091B00080688093B00002
:101B20000093B30070C08091B00080628093B000D9
:101B30000093B40068C0809190008068809390000A
:101B400010939900009398005EC08091900080628D
:101B50008093900010939B0000939A0054C0809152
:101B6000900088608093900010939D0000939C00EB
:101B70004AC08091A00080688093A0008091A0005E
:101B80008F7B8093A0001093A9000093A8003BC016
:101B90008091A00080628093A0001093AB0000931E
:101BA000AA0031C08091A00088608093A0001093AB
:101BB000AD000093AC0027C0809120018068809325
:101BC000200110932901009328011DC0809120015C
:101BD00080628093200110932B0100932A0113C08F
:101BE0008091200188608093200110932D01009343
:101BF0002C0109C00038110514F460E001C061E057
:101C00008F2D0E94B03C63E175E087EA97E00E9467
:101C10002E58B20187EA97E00E948F3E61E175E09D
:101C200087EA97E00E942E58B80187EA97E00E9461
:101C30008F3E87EA97E00E94F85852C11A8560E00B
:101C400070E0C6010E941728082FF92E6CEF74E08F
:101C500087EA97E00E942E58602F7F2D87EA97E051
:101C60000E948F3E6AEF74E087EA97E00E942E5848
:101C7000612F012E000C770B87EA97E00E948F3EC0
:101C800087EA97E00E94F8588091EC059091ED0565
:101C9000892B89F06FE879E087EA97E00E942E5857
:101CA000662D6064C6010E944528412F110F550B17
:101CB000660B770BADC081E090E09093ED058093CB
:101CC000EC0526E040E855E260E070E08AE097E04D
:101CD0000E942F3F0093F5088AE097E09093F40864
:101CE0008093F3081092000A1092020A1092010ADF
:101CF00080ED97E090937B0980937A0910927D099B
:101D000010927C09112339F085E090E090937F09CF
:101D100080937E0904C010927F0910927E0986E0AC
:101D20000E94943F62E370E080E090E00E94445F94
:101D300082ED97E090937B0980937A0910927D0958
:101D400010927C09F4E61F02A001112450937F0930
:101D500040937E09BEC00480F581E02D61857285C7
:101D6000C1010E94241EC1010E94AE27882309F4EC
:101D7000B7C08985893009F0B3C0162DEA8460E0C8
:101D800070E0C1010E941728082FF92E68E075E065
:101D900087EA97E00E942E58602F7F2D87EA97E010
:101DA0000E948F3E66E075E087EA97E00E942E5819
:101DB0006E2D0E2C000C770B87EA97E00E948F3E69
:101DC00060E075E087EA97E00E942E58662D062CA9
:101DD000000C770B87EA97E00E948F3E87EA97E036
:101DE0000E94F8588091EC059091ED05892BA1F0A7
:101DF0006FE879E087EA97E00E942E58662D6064CC
:101E0000C6010E9445284E2DEE0C550B660B770B34
:101E1000C6010E94BB2764C081E090E09093ED056D
:101E20008093EC0526E040E855E260E070E08AE04F
:101E300097E00E942F3F0093F5088AE097E0909387
:101E4000F4088093F3081092000A1092020A10928C
:101E5000010A123009F4F7C1153009F4F4C16E2DEE
:101E6000EE0C770B880B990B0E94547522E538EB2A
:101E700042E152E40E94397420E030E040E251E453
:101E80000E9409762DEE3EE94CE35EE30E94AA74BF
:101E90006B017C0120E030E0A9010E94047620E083
:101EA00030E040E05FE387FDC9C1C701B6010E9491
:101EB00039740E941C7583ED97E090937B098093A1
:101EC0007A0910927D0910927C0970937F096093C2
:101ED0007E0986E00E94943F1092ED051092EC0579
:101EE000B5C18FEF01C08DEF9FEFB0C16624639441
:101EF000712C17CB63E575E087EA97E00E942E58B6
:101F00008FE7F60180871D861C8684E690E09F8718
:101F10008E874A855B8560E074E6C6010E94BB2718
:101F2000F889FF2309F469CB00E09E01265F3F4F4B
:101F300043E050E060E070E0C6010E94FB5C5DCBD6
:101F4000662DC6010E944528C6010E94F327F62E81
:101F5000E72E8C01D60118962C91233008F0FCC096
:101F6000213070F46A307105810591052CF4B2E3DB
:101F7000FB2EE12C00E010E04F2D5E2D602F0AC0FB
:101F8000611571058105910519F01A300CF412E301
:101F9000AB01682F712FC6010E94BB274F2D5E2D0C
:101FA000B8011416150616061706E4F5D60118969C
:101FB0008C9190E08A30910538F5FC018827E25732
:101FC000FF4F8F4F0C941A74C7019A878B87802F0D
:101FD000000F990B9D878C87812F110F990B9F877D
:101FE0008E8753C05B874A8701E07FC05B874A8743
:101FF000B889BB2309F401CB00E020E030E040E0E9
:1020000050E061E070E00AC0E889EE2309F4A8C05E
:1020100000E020E030E040E050E0B301C6010E9463
:10202000FB5C9EC02AE030E087EA97E00E94B0584F
:1020300065E375E087EA97E00E942E58D60118966E
:102040008C918530C9F0A0F48150823008F041C0F5
:1020500084E690E09B878A871D861C869F878E87F3
:1020600044E650E060E074E6C6010E94BB270DC064
:102070008630C9F0883069F584E190E09B878A87D3
:1020800044E150E060E070E02CC001E09E01265F7A
:102090003F4F43E050E060E070E0C6010E94FB5C0F
:1020A00003E010E02EC084E690E09B878A8744E638
:1020B00050E060E070E0C6010E94BB27B889BB23F6
:1020C000F1F000E020E030E040E050E061E070E05E
:1020D00013C084E690E09B878A8744E650E060E086
:1020E00070E0C6010E94BB2700E09E01265F3F4FC3
:1020F00041E050E060E070E0C6010E94FB5C01E05E
:1021000010E05E01EAE0AE0EB11CE12CF12CD5012D
:102110008D909D905D016AE275E087EA97E00E94EC
:102120002E58B70187EA97E00E948F3E68E275E07B
:1021300087EA97E00E942E58B40187EA97E00E9450
:102140008F3E87EA97E00E94F858BFEFEB1AFB0A30
:102150000E151F05E1F604C0243009F403CF1ECF8D
:10216000F6018085813009F048CA8C859D85892BD0
:1021700009F043CA8FE7F60180873FCA60E0C701D4
:102180000E94A93EDC0119968D919C911A97998B1A
:10219000888B61E0C7010E94A93EFC014184528402
:1021A000638474842A843B84F2E0AF16B104E9F1BD
:1021B00062E0C7010E94A93EDC0119960D911C91B5
:1021C0001A97B3E0AB16B10491F163E0C7010E9426
:1021D000A93EFC0181849284F4E0AF16B10451F071
:1021E00064E0C7010E94A93EDC011996AD90BC9045
:1021F0001A9703C032E0A32EB12C8114910461F030
:102200009401D1010E94297424E630E040E050E0BE
:102210000E94D973790101C071019501A2016889F9
:102220007989C6010E94401E5BCE0FEF1FEF8FE33E
:10223000882E912C92E0A92EB12CE2CFC701B601D5
:102240000E94387436CE60E070E035CE6B960FB6E3
:10225000F894DEBF0FBECDBFDF91CF911F910F91DC
:10226000FF90EF90DF90CF90BF90AF909F908F90B6
:102270007F906F905F904F903F902F9008954F9276
:102280005F926F927F928F929F92AF92BF92CF9206
:10229000DF92EF92FF920F931F93CF93DF93CDB70F
:1022A000DEB7C15AD1400FB6F894DEBF0FBECDBF26
:1022B000E0919505F09196053B96E831F10508F01F
:1022C000B7C38827E856FF4F8F4F0C941A740E94AB
:1022D0007E5F0091F6051091F7052091F805309189
:1022E000F905061717072807390708F0A1C30FE0FB
:1022F00013E0CF56DE4F19830883C159D140CD5624
:10230000DE4F188219821A821B82C359D140CF57DF
:10231000DE4F19830883C158D140CD57DE4F188254
:1023200019821A821B82C358D140CF59DE4F1983BC
:102330000883C156D140CD59DE4F188219821A82C6
:102340001B82C356D140CF5BDE4F19830883C15433
:10235000D140CD5BDE4F188219821A821B82C35492
:10236000D1406BE576E087EA97E00E942E58BE01E7
:102370006F567E4F86E090E00E94A339892B09F4C6
:1023800067C16CE673E087EA97E00E94FC581A8305
:102390000983CD56DE4F88819981AA81BB81C359BB
:1023A000D1408B839C83AD83BE83CE0101960E9476
:1023B000914EBE016F577E4F8AE090E00E94A33994
:1023C000892B09F42EC162E873E087EA97E00E9446
:1023D000FC581A830983CD57DE4F88819981AA81E1
:1023E000BB81C358D1408B839C83AD83BE83CE0118
:1023F00001960E94914EBE016F597E4F8EE090E093
:102400000E94A339892B09F4DFC068E873E087EAEA
:1024100097E00E94FC581A830983CD59DE4F8881CA
:102420009981AA81BB81C356D1408B839C83AD83A4
:10243000BE83CE0101960E94914EBE016F5B7E4F1E
:1024400082E190E00E94A339892B09F477C06DE8FE
:1024500073E087EA97E00E94FC581A830983CD5BFA
:10246000DE4F88819981AA81BB81C354D1408B837F
:102470009C83AD83BE83CE0101960E94914E1A8348
:102480000983CD5BDE4F88819981AA81BB81C354CA
:10249000D1408B839C83AD83BE83CF57DF4F19839D
:1024A0000883C158D040CD59DE4F88819981AA81D7
:1024B000BB81C356D140CD57DF4F88839983AA8310
:1024C000BB83C358D040CF53DF4F19830883C15C0F
:1024D000D040CD57DE4F88819981AA81BB81C358F6
:1024E000D140CD53DF4F88839983AA83BB83C35CDC
:1024F000D040CF5FDE4F19830883C150D140CD5605
:10250000DE4F88819981AA81BB81C359D140CD5FBB
:10251000DE4F88839983AA83BB83C350D1409E0139
:102520002F5F3F4FAE014F575F4FBE016F537F4F3D
:10253000CE018F5F9E4F0E946F3D85C01A83098335
:10254000CD59DE4F88819981AA81BB81C356D14084
:102550008B839C83AD83BE83CF57DF4F1983088362
:10256000C158D040CD57DE4F88819981AA81BB8167
:10257000C358D140CD57DF4F88839983AA83BB834B
:10258000C358D040CF53DF4F19830883C15CD0407C
:10259000CD56DE4F88819981AA81BB81C359D14034
:1025A000CD53DF4F88839983AA83BB83C35CD0401C
:1025B000AE014F5F5F4FBE016F577F4FCE018F530C
:1025C0009F4F0E94BB3D3FC01A830983CD57DE4F0A
:1025D00088819981AA81BB81C358D1408B839C8318
:1025E000AD83BE83CF57DF4F19830883C158D040D6
:1025F000CD56DE4F88819981AA81BB81C359D140D4
:10260000CD57DF4F88839983AA83BB83C358D040BB
:10261000BE016F5F7F4FCE018F579F4F0E940D3ECF
:1026200012C01A830983CD56DE4F88819981AA8111
:10263000BB81C359D1408B839C83AD83BE83CE01C4
:1026400001960E94583E87EA97E00E94F8580BC115
:1026500064E973E087EA97E00E94FC580FB6F894AB
:10266000A89580916000886180936000109260005E
:102670000FBE80918805811107C08DE695E00E940C
:10268000464381E0809388058AE295E09093510863
:10269000809350080E94DF3CCE0101960E944322A5
:1026A00089819A810E94A65246E050E062E077E07C
:1026B00089E090E00E9454368FE093E09A8389830A
:1026C0001B821C821D821E82CE0103960E949052A4
:1026D0000E94A5528091500890915108DC01929679
:1026E0001D921D921D921C929597FC0116A217A295
:1026F00010A611A69A961D921D921D921C929D974E
:1027000040EE5EE260E070E046AB57AB60AF71AFA9
:1027100040EA5FE060E070E0DA964D935D936D9380
:102720007C93DD973E9624E1DF011D922A95E9F71F
:1027300026E0E2E0F7E0DC01189601900D922A9580
:10274000E1F7FC01EE5BFF4F10820E94D6378C014F
:10275000019709F04AC0CE0101960E944322898167
:102760009A810E94A6526091500870915108625F50
:102770007F4FCE0101960E94FE58CE0103960E9423
:10278000905260915008709151086A5E7F4FCE015F
:1027900001960E94FE58CE0103960E949E526091BF
:1027A0005008709151086E5E7F4FCE0101960E94D5
:1027B000FE58CE0103960E9497520E94A552609146
:1027C000500870915108625E7F4FCE0101960E94C1
:1027D000FE588B819C81AD81BE8180934C08909383
:1027E0004D08A0934E08B0934F0899E288E10FB6C8
:1027F000F894A895809360000FBE90936000A89510
:10280000012B19F569E176E087EA97E00E942E58DE
:102810006AEE75E087EA97E00E942E5886EF9FEFF8
:1028200090939605809395050E947E5FDC01CB0115
:10283000805A9541AF4FBF4F8093F6059093F705AF
:10284000A093F805B093F905F3C06AED75E087EA47
:1028500097E00E942E58CE0101960E94E74ECE01CD
:1028600001960E94914E81E090E0DEC0809190053B
:1028700081111AC060E070E080E090E00E94942E28
:10288000D3C00E947E5F0091F6051091F70520915C
:10289000F8053091F9050617170728073907C8F119
:1028A0000E94AE1F8111C4C082E090E0BDC0A89517
:1028B000CF55DE4F1882C15AD140FE01EF56FE4F70
:1028C000119211928EE0DF011D928A95E9F7009135
:1028D000830A1091840A0115110529F0C8010E948C
:1028E0004B42811137C20E94AE1F8111A1C0E090FE
:1028F000830AF090840AE114F10409F499C0C70135
:102900000E944B42082F10E0023011050CF03FC22C
:102910008FC020E030E043E050E060E48E010F5FC4
:102920001F4FC8010E946C5568ED74E0C8010E94F9
:102930005178F80101900020E9F7CF01801B910B3D
:1029400008968138910538F50E94AE1F882319F149
:102950008091D8089091D908019611F481E090E017
:102960009093D9088093D8088091D8089091D9087D
:1029700090935D0880935E0847E050E068E578E05A
:10298000C8010E94251FAC014550510968E578E057
:1029900082EA0E94451F83E090E090939605809321
:1029A000950561E378E087EA97E00E942E5840C0E1
:1029B0000E947E5F0091F6051091F7052091F805C1
:1029C0003091F905061717072807390788F510927F
:1029D0009605109295052CC00E947E5F0091F60529
:1029E0001091F7052091F8053091F90506171707A2
:1029F0002807390708F458CF1BC00E94B14B892B18
:102A000009F052CF0E947E5FDC01CB0188579C4EBB
:102A1000AF4FBF4F8093F6059093F705A093F8054D
:102A2000B093F90586EF9FEF9093960580939505F7
:102A30000FB6F894A895809160008861809360003B
:102A4000109260000FBE8091950590919605181622
:102A500019060CF059C10091500810915108011548
:102A6000110509F451C10E947E5F4B015C017801A0
:102A7000FEE3EF0EF11CF70180819181A281B38109
:102A8000A5019401281B390B4A0B5B0BCA01B90144
:102A9000683E33E073078105910508F446C028EECF
:102AA00033E040E050E00E94B773861A970AA80A04
:102AB000B90AD7018D929D92AD92BC921397F801FD
:102AC00086A597A5A0A9B1A969017A01CC0CDD1C46
:102AD000EE1CFF1C8C159D05AE05BF0528F416A63F
:102AE00017A610AA11AA09C0821B930BA40BB50B41
:102AF000F80186A797A7A0ABB1ABF80182A993A96B
:102B0000A4A9B5A98C159D05AE05BF0528F412AA88
:102B100013AA14AA15AA09C0821B930BA40BB50B08
:102B2000F80182AB93ABA4ABB5ABF80186A597A532
:102B3000A0A9B1A9892B8A2B8B2B69F4EE5BFF4FDF
:102B40008081833041F484E08083C8010E94D637BD
:102B500001967C0102C0E12CF12CF80182A993A915
:102B6000A4A9B5A9892B8A2B8B2BA1F4EE5BFF4F6F
:102B70008081833011F081110DC01082F8013E96E2
:102B800084E1DF011D928A95E9F7C8010E94D637DA
:102B900003967C01B2E0EB16F10429F0E4E0EE16B6
:102BA000F10409F04AC0CE0101960E9443228981B6
:102BB0009A810E94A6526091500870915108625FFC
:102BC0007F4FCE0101960E94FE58CE0103960E94CF
:102BD000905260915008709151086A5E7F4FCE010B
:102BE00001960E94FE58CE0103960E949E5260916B
:102BF0005008709151086E5E7F4FCE0101960E9481
:102C0000FE58CE0103960E9497520E94A5526091F1
:102C1000500870915108625E7F4FCE0101960E946C
:102C2000FE588B819C81AD81BE8180934C0890932E
:102C30004D08A0934E08B0934F08F3E0EF16F1044F
:102C400009F451C064F431E0E316F10451F142E0BB
:102C5000E416F10409F058C068EF77E049C054E089
:102C6000E516F10409F442C085E0E816F10409F024
:102C70004BC069E278E087EA97E00E942E5887EA25
:102C800097E00E94F8580E94AE1F81110E94144FD5
:102C90000E947E5FDC01CB01805D9A48AF4FBF4F41
:102CA00013C065E178E087EA97E00E942E580E9401
:102CB000AE1F81110E94144F0E947E5FDC01CB0188
:102CC00088519C4FAF4FBF4F8093F6059093F70507
:102CD000A093F805B093F90586EF9FEF90939605C2
:102CE0008093950511C065EE77E0DDCF69EC77E064
:102CF00087EA97E00E942E58CE0101960E94E74E87
:102D0000CE0101960E94914E99E288E10FB6F894A7
:102D1000A895809360000FBE909360008091950508
:102D200090919605CF55DE4F0FB6F894DEBF0FBEDB
:102D3000CDBFDF91CF911F910F91FF90EF90DF906A
:102D4000CF90BF90AF909F908F907F906F905F904B
:102D50004F90089560E0C8010E94A93EDC011996D9
:102D60000D911C911A9710938C0A00938B0A6CEBAF
:102D700077E087EA97E00E942E58B80187EA97E04B
:102D80000E94FC5887EA97E00E94F858ACCD61E0B9
:102D9000C7010E94A93EFC016184728402301105C2
:102DA00009F450C362E0C7010E94A93EFC0181847E
:102DB00092840330110551F063E0C7010E94A93EDF
:102DC000DC011996ED90FC901A9704C0FE01EF55B6
:102DD000FE4F7F0140E150E0BE016F567E4F86E31B
:102DE00090E00E941B2E892B21F4053011050CF078
:102DF00032C38E010F561E4F7092EC086092EB08A2
:102E00009092EE088092ED088CEB9BE59093E4089D
:102E10008093E3085E01FFE7AF1AFEEFBF0A40E1CF
:102E200050E06FE877E0C5010E94586C6E012FE911
:102E3000C21A2EEFD20A20E030E041E050E060E21A
:102E4000C6010E946C5540E250E068E877E0C60198
:102E50000E94486C68E677E087EA97E00E942E5867
:102E6000B30187EA97E00E94FC5866E677E087EABC
:102E700097E00E942E58B40187EA97E00E948F3EA7
:102E80006FE577E087EA97E00E942E58B70187EA5E
:102E900097E00E94FC586AE577E087EA97E00E9495
:102EA0002E580FB6F894A8958091600088618093A1
:102EB0006000109260000FBE80908B0A90908C0A88
:102EC0000E94AE1F81113BC16091EB087091EC082C
:102ED00080915608909157084091ED085091EE0866
:102EE000DC01ED91FC916115710521F00088F189FB
:102EF000E02D16C00684F785E02D2FE033E03A83FD
:102F000029834090E7085090E8086090E9087090A5
:102F1000EA084B825C826D827E82BE016F5F7F4FCA
:102F200019958130910509F003C19093D9088093D8
:102F3000D80887E0E2E1F2E0DE01119601900D92FF
:102F40008A95E1F7FE013196ADE5B8E0CE0108962D
:102F500021912D93E817F907D9F7E114F10429F02D
:102F60000115110521F086EF03C086E301C086EB51
:102F700080936408109265088FE080936608F401DE
:102F800001900020E9F7CF0188199909409681380E
:102F9000910508F0C1C04FE050E068E578E0C40159
:102FA0000E94251FF60101900020E9F73197EC19E6
:102FB000FD09E80FF91F3296E138F10508F0ACC0C1
:102FC000AC0168E578E0C6010E94251FF50101907B
:102FD0000020E9F73197EA19FB09E80FF91F32964B
:102FE000E138F10508F098C0AC0168E578E0C5016A
:102FF0000E94251FE114F10479F1F70101900020EE
:10300000E9F73197EE19FF099C012E5F3F4FE20F60
:10301000F31FE138F10508F07FC0AC0168E578E006
:10302000C7010E94251F01151105B1F0F80101909B
:103030000020E9F73197E01BF10B9C012E5F3F4F19
:10304000E20FF31FE138F10508F066C0AC0168E556
:1030500078E0C8010E94251FAC014550510968E580
:1030600078E080E10E94451F0E947E5F6093DA084D
:103070007093DB088093DC089093DD086093DE0892
:103080007093DF088093E0089093E10880915608E0
:1030900090915708DC01ED91FC910084F185E02DC1
:1030A0001995892BC1F40E947E5F0091DE08109172
:1030B000DF082091E0083091E108DC01CB01801BA2
:1030C000910BA20BB30B88399A43A105B105F0F21D
:1030D0008CEF9FEF1DC0CE018F579F4F0E94494C30
:1030E0000497D1F480915B08811111C00E947E5F2A
:1030F0006093DE087093DF088093E0089093E10806
:103100001092E2081092F2081092F10818C090E0B4
:103110009093F2088093F108809156089091570897
:10312000DC01ED91FC910488F589E02D1995A6C18B
:103130008EEF9FEF9093F2088093F1089FC100916A
:103140008B0A10918C0A6CE477E087EA97E00E9482
:103150002E58B80187EA97E00E94FC5887EA97E06A
:103160000E94F85899E288E10FB6F894A8958093E8
:1031700060000FBE9093600081E08093900520E096
:1031800030E043E050E060E4CE018F5F9E4F0E944C
:103190006C5568ED74E0CE018F5F9E4F0E945178B0
:1031A000CE018F5F9E4F0E94633920E030E042E005
:1031B00050E060E4CE018F5F9E4F0E946C5568ED39
:1031C00074E0CE018F5F9E4F0E945178BE016F5F09
:1031D0007E4F87EA97E00E94525887EA97E00E9464
:1031E000F858CE018F5F9E4F0E94633920E030E097
:1031F00041E050E060E4CE018F5F9E4F0E946C552D
:1032000068ED74E0CE018F5F9E4F0E945178BE0141
:103210006F5F7E4F87EA97E00E94525887EA97E0F7
:103220000E94F858CE018F5F9E4F0E946339FE01C5
:10323000EF53FF4F119211921EE3DF01212F1D92D8
:103240002A95E9F71A821982FE0133968EE7DF018B
:103250001D928A95E9F720E030E041E050E060E41B
:10326000CE018F539F4F0E946C5540E450E068E8B8
:1032700077E0CE018F539F4F0E94486C40E850E0AA
:1032800065E077E0CE0101960E94586CBE016F5F49
:103290007F4FCE018F539F4F0E94372020E030E0B8
:1032A00041E050E060E4CE018F539F4F0E946C5587
:1032B00040E450E06FEF76E0CE018F539F4F0E94C5
:1032C000486C40E850E065EF76E0CE0101960E9440
:1032D000586C40E850E062EE76E0CE0101960E9424
:1032E000486CBE016F5F7F4FCE018F539F4F0E948E
:1032F000372020E030E041E050E060E4CE018F5321
:103300009F4F0E946C5540E450E064E179E0CE01AB
:103310008F539F4F0E94486C40E850E062ED76E08A
:10332000CE0101960E94586CBE016F5F7F4FCE01A7
:103330008F539F4F0E94372020E030E041E050E063
:1033400060E4CE018F539F4F0E946C5540E450E0E3
:103350006BEC76E0CE018F539F4F0E94486C40E8A3
:1033600050E065EC76E0CE0101960E94586CBE01FB
:103370006F5F7F4FCE018F539F4F0E943720A091E8
:10338000EE05B091EF05109709F443C08091190242
:1033900090911A02AE014F5B5E4FFA0181939193B7
:1033A0002EE111922A95E9F79E012F573F4FF9011F
:1033B0008193919311921A95E9F716960D911C91AC
:1033C0001797E090EE05F090EF05E114F10471F02D
:1033D0000115110559F0D80118968C918530A9F77F
:1033E000C8010E944B42882381F370C020E030E086
:1033F00041E050E060E4CE018F539F4F0E946C5536
:1034000040E450E068E676E0CE018F539F4F0E9483
:10341000486C84E090E090939605809395050E9417
:103420007E5FDC01CB0188579C4EAF4FBF4F80932E
:10343000F6059093F705A093F805B093F9056FE2B0
:1034400077E0B1CA8BE5882E87E0982E9E012F5534
:103450003E4F7901BFCC64E08091830A9091840A49
:103460000E94A93EDC0119960D911C911A976CE9F6
:1034700077E087EA97E00E942E58BECC0091F108D1
:103480001091F20863E277E087EA97E00E942E58F5
:10349000B80187EA97E00E948F3E6BE077E087EA09
:1034A00097E00E942E580E947E5FDC01CB01885776
:1034B0009C4EAF4FBF4F8093F6059093F705A093B6
:1034C000F805B093F9058CE090E0AECA60E0C80161
:1034D0000E94A93EFC0181859285A385B4858A302E
:1034E000910508F463C020E030E041E050E060E482
:1034F000CE018F539F4F0E946C55F80160817181FE
:1035000040E450E0CE018F539F4F0E94777860EBEC
:1035100073E0CE018F539F4F0E94517840E450E0FA
:1035200067E776E0CE018F539F4F0E94486CBE0143
:103530006F5B7E4FCE018F539F4F0E943720CF5736
:10354000DF4F8881C158D040882361F120E030E00E
:1035500041E050E060E4CE018F539F4F0E946C55D4
:10356000D8016D917C9140E450E0CE018F539F4F84
:103570000E94777860EB73E0CE018F539F4F0E94DB
:10358000517840E450E06FE676E0CE018F539F4FD4
:103590000E94486CBE016F577F4FCE018F539F4FE3
:1035A0000E943720F801028113810BCFFC0140E219
:1035B00050E08827E055FF4F8F4F0C941A746FEB43
:1035C00076E0CE018F5B9E4F0E94586CCF57DF4F45
:1035D0001882C158D04087CF6AEB76E0CE018F5B6E
:1035E0009E4F0E94586C40E450E069E976E017C0B5
:1035F00063E976E0CE018F5B9E4F0E94586C40E4F9
:1036000050E06FE876E00BC067E876E0CE018F5BB4
:103610009E4F0E94586C40E450E061E876E0CE0195
:103620008F579F4F0E94586C5ECF2F923F924F92C0
:103630005F926F927F928F929F92AF92BF92CF9242
:10364000DF92EF92FF920F931F93CF93DF93CDB74B
:10365000DEB728970FB6F894DEBF0FBECDBF8C0142
:103660006B010E945B34019609F4D3C2D801ED913D
:10367000FC910284F385E02DC80119957C018F3FF0
:10368000BFEF9B0709F4C5C2D801ED91FC910684F8
:10369000F785E02D682FC8011995B2E2EB16F10409
:1036A00029F4B601C8010E947C34B5C2EDE2EE16E1
:1036B000F10429F0C701C0970A9708F044C1D80166
:1036C000ED91FC910284F385E02DC80119957C01F0
:1036D0008F3FBFEF9B0709F49CC28D9789F4D801F7
:1036E000ED91FC910284F385E02DC80119957C01D0
:1036F000019609F48EC2EFEFFFEFF887EF8304C065
:1037000021E030E038872F83C701C097A12CB12C6E
:103710000A97C8F49AE0992E9A9CC0019B9C900D40
:103720001124B701605371095B01A80EB91ED801BD
:10373000ED91FC910284F385E02DC80119957C017F
:10374000C0970A9748F3BEE2EB16F104D1F0C70127
:103750008F7D85349105A9F0EF81F885AE9EC0017B
:10376000AF9E900DBE9E900D1124092E000CAA0B49
:10377000BB0BF60181879287A387B48782E080879D
:10378000D8C0B501BB0C880B990B0E9454752B0156
:103790003C01FEE2EF16F104A1F5D801ED91FC9198
:1037A0000284F385E02DC80119957C01212C312C70
:1037B00020E030E040E251E4C301B2010E9409760A
:1037C0004B015C01B70160537109072E000C880B97
:1037D000990B0E945475A50194010E9439742B0124
:1037E0003C01B1E02B1A3108D801ED91FC91028423
:1037F000F385E02DC80119957C01C0970A97C0F2A6
:1038000002C0212C312CC7018F7D8534910509F030
:1038100042C0D801ED91FC910284F385E02DC801EE
:1038200019957C018B32910559F4D801ED91FC91E9
:103830000284F385E02DC80119957C01B1E00CC02C
:103840008D9761F4D801ED91FC910284F385E02D10
:10385000C80119957C01BFEFBE8302C0E1E0EE8391
:10386000A12CB12C8AE0982EC701C0978A3091050F
:10387000B0F49A9C90019B9C300D11245C01A20E27
:10388000B31ED801ED91FC910284F385E02DC801AF
:1038900019957C01E9CFB1E0BE83A12CB12CEF8159
:1038A000F885BF01FF0F880B990B0E945475A30187
:1038B00092010E9409762B013C01B501BB0C880BDB
:1038C000990B0E9454754B015C01FE816F2FFF0F15
:1038D000770B880B990B0E9454759B01AC01C501B5
:1038E000B4010E9409764B015C01B101330C880BD5
:1038F000990B0E9454759B01AC01C501B4010E9453
:1039000039749B01AC0160E070E080E291E40E94B8
:1039100076769B01AC01C301B2010E940976D60103
:1039200019966D937D938D939C931C9783E01896C5
:103930008C93D801ED91FC910684F785E02D6E2DD6
:10394000C801199522C0BBE5EB16F10409F060C06F
:10395000D801ED91FC910284F385E02DC801199501
:103960008B35910509F055C185E0F6018087C801C6
:103970000E945B34D801ED91FC910284F385E02D27
:10398000C80119958D35910519F480E090E043C187
:10399000D801ED91FC910684F785E02D682FC801D0
:1039A0001995BB24BA940E9434357C01009709F420
:1039B00030C1BB2021F0F6019783868308C0D40173
:1039C00013969C938E931297FC0195828482C80172
:1039D0000E945B34B701C8010E94151B892B09F0B6
:1039E00018C1C8010E945B34D801ED91FC9102849A
:1039F000F385E02DC8011995B12C47018C32910552
:103A000091F221E030E08D35910509F089C086C042
:103A1000BBE7EB16F10409F088C0D801ED91FC91E9
:103A20000284F385E02DC80119958B37910509F0C3
:103A3000F0C086E0F6018087C8010E945B34D8019F
:103A4000ED91FC910284F385E02DC80119958D3725
:103A5000910509F49ACFD801ED91FC910684F78580
:103A6000E02D682FC801199599249A940E94343545
:103A70007C01009709F4CDC0992021F0F6019783CD
:103A8000868308C0D50113969C938E931297FC01F0
:103A9000B582A482C8010E945B34B701C8010E94AC
:103AA0007C34019609F4B5C0C8010E945B34D7018B
:103AB00019968D919C911A9711969C938E931A96B4
:103AC0001C921E921997D801ED91FC910284F38506
:103AD000E02DC8011995CA9709F09BC0C8010E9442
:103AE0005B34B701C8010E94151B019609F491C00F
:103AF000C8010E945B34D801ED91FC910284F385EA
:103B0000E02DC8011995912C57018C32910509F4CB
:103B1000ADCF21E030E08D37910511F420E030E0A9
:103B200088279927821B930B76C0BEE6EB16F1041B
:103B300011F519821A821B821C82D801ED91FC9129
:103B40000484F585E02D44E050E0BE016F5F7F4FB7
:103B5000C8011995049709F05CC044E050E063E3A4
:103B600074E0CE0101960E948778009709F051C059
:103B7000F601108650C0F6E6EF16F10421F59E011D
:103B80002F5F3F4F790185E0D9011D928A95E9F7B2
:103B9000D801ED91FC910484F585E02D45E050E0DD
:103BA000B901C80119950597A1F545E050E068E312
:103BB00074E0C7010E948778009759F521E0F6016B
:103BC0002087118628C0F4E7EF16F10411F5198259
:103BD0001A821B821C82D801ED91FC910484F58528
:103BE000E02D44E050E0BE016F5F7F4FC8011995A2
:103BF000049779F444E050E06EE374E0CE0101965E
:103C00000E948778009729F421E0F6012087218718
:103C100002C08FEF9FEF28960FB6F894DEBF0FBE5D
:103C2000CDBFDF91CF911F910F91FF90EF90DF906B
:103C3000CF90BF90AF909F908F907F906F905F904C
:103C40004F903F902F900895CF93DF93EC0189E63A
:103C500092E0998388836115710559F08091EE0592
:103C60009091EF05009729F00E94B63E9B838A83CE
:103C700002C01B821A82CE01DF91CF910C947D2865
:103C80006F927F928F929F92AF92BF92CF92DF926C
:103C9000EF92FF920F931F93CF93DF93CDB7DEB7D1
:103CA0002C970FB6F894DEBF0FBECDBF4C01762E19
:103CB000672E6A0159018091EC059091ED05892BE1
:103CC000A1F06FE879E087EA97E00E942E5860E45F
:103CD000C4010E944528A701FF0C660B770BC401A5
:103CE0000E94BB278FEF9FEF9BC081E090E09093F5
:103CF000ED058093EC0526E240E855E260E070E0D7
:103D00008AE097E00E942F3F7092F5088AE097E0E2
:103D10009093F4088093F3081092000A1092020A1C
:103D20001092010A0115110541F00130110539F415
:103D3000FE2CEE24EE24EA9402C0FF24FA94C7017C
:103D4000A0E0B0E08F839887A987BA8780E190E0F0
:103D50009C878B87A60160E070E049835A836B8360
:103D60007C839E838D83672D762D87EA97E00E9462
:103D70008F3E6CE879E087EA97E00E942E58BE01FA
:103D80006F5F7F4F87EA97E00E94D7288C0168E831
:103D900079E00E942E58B501C8010E948F3E65E867
:103DA00079E0C8010E942E58BE01695F7F4FC801AB
:103DB0000E94D7280E94F858A114B10491F082E023
:103DC000A816B10409F5D0927B09C0927A09109225
:103DD0007D0910927C09F0927F09E0927E0986E0CD
:103DE00010C0D0927B09C0927A09E11003C080E034
:103DF00090E002C080E09FEF90937D0980937C0962
:103E000085E00E94943F06C06DE679E087EA97E07E
:103E10000E942E581092ED051092EC0580E090E083
:103E20002C960FB6F894DEBF0FBECDBFDF91CF91B9
:103E30001F910F91FF90EF90DF90CF90BF90AF90C8
:103E40009F908F907F906F900895CF93DF93EC01B8
:103E5000FA013296E60FF71FDC01AD014C1B5D0B3A
:103E6000CF01861B970B2D91222311F02193F5CFC3
:103E70009C01241B350B620F731FFB01329750838B
:103E800031964083DF91CF910895EF92FF920F9387
:103E90001F93CF93DF9300D01F92CDB7DEB77B0186
:103EA000BA0130E0962F9F77660F672F661F770B5A
:103EB00071956115710509F0906821E0230FE1E02B
:103EC000F0E0EC0FFD1FE30FF11D9083611571050C
:103ED00011F0322FE7CF30E0B701621B730B6C5F3C
:103EE0007F4FDB018C93DE011196F701E21BF30B90
:103EF000359685E0E80EF11CEE16FF0619F08D915F
:103F00008193FACF80915608909157082F5F3F4FC9
:103F10008901040F151FDC01ED91FC910280F381F2
:103F2000E02DA80119957C010E947E5F6093DA085C
:103F30007093DB088093DC089093DD0881E00E1518
:103F40001F0509F080E00F900F900F900F90DF9108
:103F5000CF911F910F91FF90EF900895CF93809193
:103F6000560890915708009771F1DC01ED91FC9192
:103F70000688F789E02D1995C1E0811125C0C0E0C0
:103F80008091F1089091F208892BF1F48DEF9FEF69
:103F90009093F2088093F108809156089091570809
:103FA000DC01ED91FC910680F781E02D199580915F
:103FB000560890915708DC01ED91FC910488F58931
:103FC000E02D199501C0C0E08C2FCF910895DF92AC
:103FD000EF92FF920F931F93CF93DF938C01D62E16
:103FE000E72EEA01F22E0E94AE1F8823B9F1F801F4
:103FF00001900020E9F73197E01BF10BCE01079605
:10400000E80FF91FE138F10548F545E050E068E5B3
:1040100078E0C8010E94251FAC01ED2DFE2DDC01CA
:10402000A85AB74F9F012C0F3D1FE217F30719F055
:1040300081918D93FACF2597FF2011F081E301C084
:1040400080E34C0F5D1F68E578E0DF91CF911F9111
:104050000F91FF90EF90DF900C94451F80E0DF916F
:10406000CF911F910F91FF90EF90DF900895FB018A
:1040700001900020E9F73197AF01461B570B21E073
:104080000C94E71FCF92DF92EF92FF920F931F9352
:10409000CF93DF931F921F92CDB7DEB76C0161E023
:1040A0000E946A28182F86FF1BC0C6010E94F327B2
:1040B0007A8369836FE579E087EA97E00E942E585A
:1040C000612F70E06F7BE12CF12C01E09E012F5FEE
:1040D0003F4F41E050E0C6010E94BF0881E001C0AF
:1040E00080E00F900F90DF91CF911F910F91FF9083
:1040F000EF90DF90CF9008958F929F92AF92BF92F2
:10410000CF92DF92EF92FF920F931F93CF93DF93A3
:104110001F921F92CDB7DEB76C017B0162E070E0A9
:104120000E9417288C0197FF03C080E090E099C09F
:1041300063E070E0C6010E941728AC01181619064A
:1041400014F04FE350E0E982FA820130110531F4B6
:104150008F2D880F880BF9828A8303C002301105E6
:104160002CF489819A8199279A838983A981BA81BC
:1041700024E630E00E9431749A01550F440B550B30
:104180000E94D97349015A0189013A83298360E069
:10419000C6010E946A28E82EF12CC6010E94F3276E
:1041A000092C000CAA08BB08681579058A059B052F
:1041B00059F4012BE9F182E0E816F10459F085E0A9
:1041C000E816F104A9F506C0012B71F182E0E816AA
:1041D000F10479F500E020E030E040E050E061E0FB
:1041E00070E0C6010E94FB5C00E09E012F5F3F4F24
:1041F00041E050E060E070E0C6010E94FB5C86E0B8
:10420000E816F10439F0EA94EF2821F061E0C601E4
:104210000E94452849815A81052E000C660B770BB8
:10422000C6010E94BB2704C085E0E816F10431F402
:1042300018C085E0E816F104B9F6CCCF82E0E816A4
:10424000F104B1F362E0C6010E94452800E020E0DD
:1042500030E040E050E062E070E0C6010E94FB5CAC
:10426000E7CF0F900F90DF91CF911F910F91FF90AB
:10427000EF90DF90CF90BF90AF909F908F90089578
:10428000CF92DF92EF92FF920F93CF93DF9300D004
:1042900000D0CDB7DEB77C0161E00E946A2885FFBF
:1042A00040C0C82ED12CC7010E94F327382F292FD8
:1042B000F701808590E08A30910528F5FC01882778
:1042C000E654FF4F8F4F0C941A7469837A83832FBF
:1042D000330F990B9C838B83822F220F990B9E8324
:1042E0008D8300E09E012F5F3F4F43E050E008C008
:1042F0007A83698300E09E012F5F3F4F41E050E0E9
:1043000060E070E006C000E020E030E040E050E017
:10431000B601C7010E94FB5CB6016F7DC7010E9418
:10432000452826960FB6F894DEBF0FBECDBFDF91AD
:10433000CF910F91FF90EF90DF90CF9008958F92E3
:104340009F92AF92BF92EF92FF920F931F93CF93E2
:10435000DF938C017B0149015A010E943435EC0145
:10436000892BF9F083E0888789869A86AB86BC869C
:1043700088819981009711F00E94E069C7010E942D
:10438000057899838883BE01C801DF91CF911F9181
:104390000F91FF90EF90BF90AF909F908F900C94F3
:1043A000D83EDF91CF911F910F91FF90EF90BF907A
:1043B000AF909F908F900895FB0101900020E9F746
:1043C0003197AF01461B570B20E00C94E71F0F936A
:1043D0001F93CF93DF93EC012097F9F00A811B81A3
:1043E000888587FD06C08E819F81009711F00E940D
:1043F000E7218885843031F489859A85009711F00A
:104400000E94E06988819981009711F00E94E0691B
:10441000CE010E94E069E801DFCFDF91CF911F91CB
:104420000F9108950F931F93CF93DF93009791F00F
:104430008C010E943435EC01892B61F0C8010E9487
:104440005B34BE01C8010E94151B019631F4CE01F8
:104450000E94E72180E090E001C0CE01DF91CF9182
:104460001F910F910895CF93C82F462F61E070E000
:104470000E94CB4361E070E08C2F0E94A144811127
:10448000F9CFCF91089520E5FC0120831182089592
:10449000FC018485843011F00C94314680E008954D
:1044A0008F929F92AF92BF92CF92DF92EF92FF9244
:1044B0000F931F93CF93DF936B017C01142F9B010C
:1044C000AC010E94C676882319F063E474E027C02B
:1044D00046015701E894B7F82FEF3FEF4FE75FE74A
:1044E000C501B4010E94C67681110DC02FEF3FEFC8
:1044F0004FE75FE7C501B4010E94A57418161CF4CC
:1045000067E474E00CC02FEF3FEF4FE75FE4C701B3
:10451000B6010E940476181694F46BE474E087EAFE
:1045200097E0DF91CF911F910F91FF90EF90DF9077
:10453000CF90BF90AF909F908F900C9452582FEFD8
:104540003FEF4FE75FECC701B6010E94A57487FDFE
:10455000E4CF20E030E0A901C701B6010E94A574B4
:1045600087FF0BC06DE287EA97E00E94E957EC01F4
:10457000F7FAF094F7F8F09402C0C0E0D0E000E061
:1045800060E070E080E09FE3101741F020E030E051
:1045900040E251E40E94AA740F5FF6CFA701960192
:1045A0000E9439746B017C010E9423754B015C01F0
:1045B0002AE0AB01BC0187EA97E00E946758C80F68
:1045C000D91F1123C9F1C501B4010E9452759B0185
:1045D000AC01C701B6010E9438746B017C016EE228
:1045E00087EA97E00E94E957C80FD91F20E030E022
:1045F00040E251E4C701B6010E9409764B015C011B
:104600000E9423756B01E12CF12C2AE0B701A60171
:1046100087EA97E00E946758C80FD91FC701B60103
:104620000E9452759B01AC01C501B4010E9438740F
:104630006B017C011150D1F6CE01DF91CF911F911A
:104640000F91FF90EF90DF90CF90BF90AF909F9031
:104650008F900895BC018230910508F40895613E61
:104660008EE1780748F49B0195E0369527959A9559
:10467000E1F748E0420F01C04FEF91E0242F30E016
:10468000290F311D35952795229FF001239FF00DAD
:10469000F00D11246E177F0718F44FEF420F04C07E
:1046A0002F3F39F091E0920F491740F78FEF890FB4
:1046B00008958FEF0895CF93DF93009709F447C0D3
:1046C000FC012081222309F442C0EC0161ED79E074
:1046D0000E943F6C892BF1F16CEC79E0CE010E94D5
:1046E0003F6C892BD1F167EC79E0CE010E943F6CE1
:1046F000892BB1F16EEB79E0CE010E943F6C892BE2
:1047000091F168EB79E0CE010E943F6C892B71F149
:1047100064EB79E0CE010E943F6C892B51F16FEA86
:1047200079E0CE010E943F6C892B31F16BEA79E090
:10473000CE010E943F6C892B11F167EA79E0CE012E
:104740000E943F6C892BF1F489E090E01DC080E06D
:1047500090E01AC081E090E017C082E090E014C0C1
:1047600083E090E011C084E090E00EC085E090E02E
:104770000BC086E090E008C087E090E005C088E0CC
:1047800090E002C08FEF9FEFDF91CF9108952F92BD
:104790003F924F925F926F927F928F929F92AF92D1
:1047A000BF92CF92DF92EF92FF920F931F93CF931E
:1047B000DF93CDB7DEB72A970FB6F894DEBF0FBEF2
:1047C000CDBF5C016B01042F7901672B09F487C011
:1047D00021153105F9F0D9018C918823D9F06FE2C8
:1047E00070E0C9010E945C78009739F0FC011192D9
:1047F000CF010E945B234C0102C0812C912CC70188
:104800000E945B237C01019739F08A94892809F082
:1048100065C002C0E12CF12C66E27AE0C6010E947C
:104820003F6C892B09F40BC262E27AE0C6010E9458
:104830003F6C892B09F41FC26DE17AE0C6010E942A
:104840003F6C892B09F408C266E17AE0C6010E9438
:104850003F6C892B09F403C261E17AE0C6010E9432
:104860003F6C892B09F4FEC16DE07AE0C6010E941D
:104870003F6C892B09F4F9C168E07AE0C6010E9417
:104880003F6C892B09F4F4C163E07AE0C6010E9411
:104890003F6C892B09F4D3C16DEF79E0C6010E940A
:1048A0003F6C892B09F4E7C164EF79E0C6010E94EF
:1048B0003F6C892B09F4E2C16BEE79E0C6010E94DE
:1048C0003F6C892B09F4DDC1D6018C918D3251F0FA
:1048D00090ED980F9A3030F08332B9F1E0C180E06A
:1048E00090E0DDC1FE0131964F01412C512C1E2F6D
:1048F0009A8632012FEF621A720A2301C6010E94C2
:10490000186C1C016CE270E0C6010E945C786C01BE
:10491000892B19F03FEFC31AD30AD4012D923D928F
:104920004D01C114D10439F0F3E06F16710409F799
:1049300043E0442E512CD501ED91FC910190F08182
:10494000E02D212F3A85A20175C0CE0107969E0168
:10495000275F3F4F3F932F93215031093F932F9370
:104960009F938F938FE494E09F938F93DF92CF92E6
:104970000E9410790FB6F894DEBF0FBECDBF03972B
:1049800009F0ACCF1F8188849984812F811608F4A7
:10499000882DC92C891508F4C82E1C198C189C1850
:1049A0009C2D90959F3F09F448C080E090950E940F
:1049B0002A23D82ED094882D90E0810F911D890D47
:1049C000911D892BE9F5CD2CC094D12C10E0212F1D
:1049D00030E0ADE6B1E00E940B74412C512C320165
:1049E0004A94A30192010E94D9733A8329832D2D01
:1049F00030E0A4E6B0E00E940B74A30192010E9493
:104A0000D9733C832B832C2D30E0A4E6B0E00E94C8
:104A10000B74A30192010E94D9733E832D83D501AB
:104A2000ED91FC910190F081E02D9E012F5F3F4FB1
:104A300043E050E060E070E030C1DD24DA94BBCFA9
:104A4000BFEFDB16F9F0D11002C0DD24D3944D2C5A
:104A5000512C612C712C6FEF7FEF80E090E0A3016F
:104A600092010E94D973A12FB0E00E94F873172F12
:104A7000A82DB0E00E94F873872EA92DB0E00E9407
:104A8000F873972E682C712C610E711C690C711CC7
:104A9000EFEF6E167104FCF46114710419F46624CE
:104AA0006394712C930140E050E06FEF7FEF80E062
:104AB00090E00E94D973A12FB0E00E94F873172FE5
:104AC000A82DB0E00E94F873872EA92DB0E00E94B7
:104AD000F873972E05C0FFEF6F16710409F06CF4A0
:104AE0002C2D362D230F08F42FEF922F2F3F29F076
:104AF00080E00E942A23C82E02C0CC24CA94892DAB
:104B0000911608F4812F881508F4882D81132FC081
:104B100081100DC0182F20E8121B08F410E020E6C9
:104B2000129F010E10E0111D1124105386C0282D74
:104B300030E0482F50E0421B530B2417350744F454
:104B4000182D20E6129F010E10E0111D112475C0D2
:104B500016E5180D181B24E0121B08F410E020E6DF
:104B6000129F010E10E0111D1124105E66C0881105
:104B700039C091101AC03BEA232F211B08F420E012
:104B80004FE2249F020E20E0211D1124482F431BD9
:104B900008F440E0142F30E6139F010E10E0111DC1
:104BA0001124120F1695105C48C0292D30E090E0BA
:104BB000821B930B192D2817390744F420E6129F06
:104BC000010E10E0111D1124105A37C025E5121BEB
:104BD00008F410E020E3129F010E10E0111D1124D3
:104BE00010582BC011110DC0192D20E8121B08F40C
:104BF00010E020E3129F010E10E0111D1124185740
:104C00001CC0212F30E0892D90E0821B930B2817C8
:104C1000390744F420E6129F010E10E0111D112403
:104C200010560BC025E5121B08F410E020E6129F79
:104C3000010E10E0111D112410541F5FC8CED501C4
:104C4000ED91FC910190F081E02D20E030E040E01A
:104C500050E061E070E021C063E070E014C064E007
:104C600070E011C065E070E00EC066E070E00BC05F
:104C700067E070E008C062E070E005C068E070E0E6
:104C800002C069E070E0D501ED91FC910190F081E6
:104C9000E02D20E030E040E050E0C50119952A9673
:104CA0000FB6F894DEBF0FBECDBFDF91CF911F913D
:104CB0000F91FF90EF90DF90CF90BF90AF909F90BB
:104CC0008F907F906F905F904F903F902F900895BE
:104CD0008F929F92AF92BF92CF92DF92EF92FF920C
:104CE0000F931F93CF93DF93E091EE05F091EF05C3
:104CF000309709F468C0812EC02F932EC22EA52EA6
:104D0000D42EB72ED62FBC01CF010E94B63E8C0107
:104D1000009709F45BC0DC0118968C91853009F08E
:104D200055C060E0C8010E94A93E7C0161E0C80155
:104D30000E94A93EFC0101851285D70119962D918B
:104D40003C911A972130310569F02CF4232BF1F5B1
:104D50006C2FC80118C02230310549F027303105C9
:104D6000A9F034C06C2FC80103960E94E5546D2F42
:104D7000C8010E94E5546D2DC80101960E94E554BA
:104D80006C2DC80102960E94E55420C0892BF1F0D9
:104D900080858530D9F4E680F780E114F104B1F024
:104DA0000C2F182D2C2D392D4D2D5A2D6D2F7B2D7F
:104DB000F701818592850E946826D7011296ED90B1
:104DC000FC901397EACF80E090E002C081E090E091
:104DD000DF91CF911F910F91FF90EF90DF90CF90D7
:104DE000BF90AF909F908F900895CF92DF92EF92F7
:104DF000FF920F931F93CF93DF93E091850AF09179
:104E0000860A3097A1F09085953089F469017A017E
:104E1000EB01682FCF010E94A93EFC01818592859C
:104E2000009729F09601A701BE010E946826DF9134
:104E3000CF911F910F91FF90EF90DF90CF90089549
:104E4000AF92BF92CF92DF92EF92FF920F931F9398
:104E5000CF93DF938091800A9091810A892B09F486
:104E600072C0E1E0F0E0C0E0D0E0CC24C394D12CEB
:104E7000B6010C2E02C0660F771F0A94E2F740912C
:104E8000F4055091F5057F0184E0E80EF11CCF0197
:104E9000B12C9C01A0910602B0910702A817B90796
:104EA00020F42091060230910702A091A60AB09149
:104EB000A70AA20FB31FAC90A091800AB091810AFB
:104EC0009C0121503109A20FB31F0A2D10E02C9133
:104ED00030E00217130729F0462B572BAC92BB2466
:104EE000B3940196E816F906A1F65093F5054093A0
:104EF000F405BB2011F18091800A9091810AE80F9E
:104F0000F91F028110E0218130E0408150E03197AB
:104F1000608170E0CE010E94F5260E947E5FDC0178
:104F2000CB01845D9E4FAF4FBF4F8093F0059093B0
:104F3000F105A093F205B093F3052196F701C43073
:104F4000D10509F095CFDF91CF911F910F91FF907F
:104F5000EF90DF90CF90BF90AF900895DC01129654
:104F6000ED91FC911397309721F081E09085953079
:104F700009F080E00895CF92DF92EF92FF92CF93F5
:104F8000DF93DC011696ED91FC911797309721F194
:104F90002085223009F56A017B01EC0163EE79E09E
:104FA00087EA97E00E942E586DED79E087EA97E056
:104FB0000E942E582AE030E0B701A60187EA97E068
:104FC0000E94B05887EA97E00E94F858EE81FF816E
:104FD000C186D286E386F486DF91CF91FF90EF9071
:104FE000DF90CF900895FC0186819781009789F02A
:104FF000FC012085223041F0253079F460E00E94E8
:10500000A93E009779F0FC016185728583859485BE
:1050100008956FEF7FEFCB0108956EEF7FEF8FEF75
:105020009FEF08956DEF7FEF8FEF9FEF08950F9340
:105030001F93CF93DF93FC01C481D581209799F012
:105040008885823029F4672B71F489859A8518C088
:10505000853061F48B01CE010E944B4290E008172D
:1050600019073CF003C08FEF9FEF0AC08EEF9FEF50
:1050700007C0602FCE010E94A93EFC018185928568
:10508000DF91CF911F910F910895CF93C62F63E0C9
:10509000FC01828193810E94A93E0097C9F04C2FA8
:1050A00050E060E070E0FC014187528763877487BD
:1050B00065ED79E087EA97E00E942E586C2F87EA29
:1050C00097E00E94D13E87EA97E0CF910C94F85880
:1050D000CF910895CF93C62F63E0FC018281938125
:1050E0000E94A93E009731F0FC018185C11103C0E7
:1050F0008F7001C08FEFCF910895BF92CF92DF9252
:10510000EF92FF920F931F93CF93DF93EC010E94D6
:10511000AE27882309F441C08A819B810E944B42BB
:10512000082F10E0C801880F991F9C0123593D4F9B
:10513000790132E0B32E04301105D4F4F701C190A7
:10514000D1907F010E943435009751F0FC01B08668
:10515000A601DD0C660B770B418752876387748746
:10516000BC018A819B810E94D83E0F5F1F4FE3CF15
:105170000A811B8160E0C8010E94A93EFC01818573
:10518000888761E0C8010E94A93E9D838C8362E00C
:10519000C8010E94A93E9F838E83DF91CF911F910A
:1051A0000F91FF90EF90DF90CF90BF900895CF9335
:1051B000DF93EC01FB0124813581408151816281C3
:1051C00073810E94B058CE01DF91CF9108958F92E4
:1051D0009F92AF92BF92CF92DF92EF92FF920F9386
:1051E0001F93CF93DF93CDB7DEB7C054D1090FB66D
:1051F000F894DEBF0FBECDBF8C015B01FC01F380D4
:1052000063EA79E087EA97E00E942E586F2D87EADB
:1052100097E00E94D13E61EA79E087EA97E00E9438
:105220002E58B50187EA97E00E948F3E87EA97E003
:105230000E94F858F801C080D1806AE574E0C60188
:105240000E94B63E4C016FE574E0C6010E94B63E76
:105250007C0164E674E0C6010E94B63E8C0169E6FA
:1052600074E0C6010E94B63E6C010097B9F1FC01E2
:105270006185728540E450E0CE0101960E949578E8
:105280006FE270E0CE0101960E945C78892B51F4A8
:10529000F6012185328543E050E060E4CE010196BD
:1052A0000E946C55A114B10441F0E114F10419F409
:1052B0006EE674E00FC0F70107C00115110519F47F
:1052C00061E774E007C0F80161857285FB018081A8
:1052D000882321F0CE0101960E9437208114910489
:1052E000E9F1F40161857285CE0101960E94241EC8
:1052F000CE0101960E94AE27882381F1AB2879F078
:10530000E114F10451F4E12CF12C01E020E030E053
:1053100040E050E061E070E00EC0F70112C00115FE
:10532000110571F4E12CF12C01E020E030E040E0C7
:1053300050E062E070E0CE0101960E94BF080EC00E
:10534000F80161857285FB018081882339F020E0B6
:1053500030E041E0CE0101960E94C723C05CDF4FE0
:105360000FB6F894DEBF0FBECDBFDF91CF911F9176
:105370000F91FF90EF90DF90CF90BF90AF909F90F4
:105380008F900895EF92FF920F931F93CF93DF9327
:105390008091F4059091F505C4E0D0E021E030E083
:1053A000AC0142235323452B29F0A9014095509588
:1053B00084239523220F331F219791F79093F505AE
:1053C0008093F4050E947E5F0091F0051091F10535
:1053D0002091F2053091F30560177107820793075A
:1053E00008F457C0012B022B032B09F452C0109272
:1053F000F0051092F1051092F2051092F305E12CE0
:10540000F12CE091800AF091810AEC0FFD1F0381DD
:1054100010E0228130E0418150E0608170E0C701FE
:105420000E94F5268FEFE81AF80A249684E0E81621
:10543000F10439F7C1E0D0E08091060290910702B3
:105440008C179D0728F4809106029091070201C0F5
:10545000CE012091A60A3091A70AF901E80FF91FA1
:10546000608187EA97E00E94D13E65E774E087EAB1
:1054700097E00E94FC582196C131D105E9F687EAF0
:1054800097E0DF91CF911F910F91FF90EF900C94D7
:10549000F858DF91CF911F910F91FF90EF900895F1
:1054A00060E08DE00C94B03C61E08DE00C94B03C89
:1054B0000F931F93CF93DF93EB0187E097E09F93C8
:1054C0008F9386E097E09F938F9385E097E09F937B
:1054D0008F9384E097E09F938F9383E097E09F936F
:1054E0008F9382E097E09F938F9387E794E09F9359
:1054F0008F938B818F938A818F930E9410792DB720
:105500003EB7205F3F4F0FB6F8943EBF0FBE2DBF92
:10551000069794F40A80DB81C02D69E27AE087EA7D
:1055200097E00E942E58BE0187EA97E0DF91CF9165
:105530001F910F910C94FC580E94A15C02E017E0AF
:10554000C0E0D0E0F80161918F01CE010E94997313
:105550002196C630D105B1F76BE37AE087EA97E090
:10556000DF91CF911F910F910C942E582F923F9263
:105570004F925F926F927F928F929F92AF92BF9263
:10558000CF92DF92EF92FF920F931F93CF93DF930F
:10559000CDB7DEB7CD55D1090FB6F894DEBF0FBE3B
:1055A000CDBF0091FC051091FD050115110509F411
:1055B000A9C20E947E5FC090FE05D090FF05E090DA
:1055C0000006F0900106C616D706E806F90608F0B0
:1055D00099C2F801A680B780A114B10409F459C199
:1055E000F5018085863009F050C16396BFAEAEAE3E
:1055F000639767961FAE1EAE679764961FAE64975B
:1056000065961FAE65976CE874E0C5010E94B63ED2
:10561000009729F0FC01818564968FAF6497F501AE
:10562000808191810E94186C182F65968FAF6597C5
:105630006EE874E0C5010E94B63E009789F5649655
:105640000FAD64976BE77CE087EA97E00E942E58E5
:10565000612F87EA97E00E94D13E69E77CE087EA04
:1056600097E00E942E58602F87EA97E00E94D13E73
:1056700087EA97E00E94F85840E050E06EE874E056
:1056800063968EAD9FAD63970E94F53E6EE874E021
:1056900063968EAD9FAD63970E94B63E009729F04A
:1056A000099667969FAF8EAF67976596FFAC659733
:1056B000FF2009F4EAC067968EAD9FAD6797892BEE
:1056C00009F4E3C064968FAD6497F82FF270DF2E73
:1056D00086FF06C160E974E063968EAD9FAD639767
:1056E0000E94B63E8C01D110E4C062E08F2D0E9472
:1056F000085F65968FAD6597863308F08653909165
:105700007B00282F2870977F922B90937B008770C7
:10571000806480937C0080917A00806480937A001A
:1057200080917A0086FDFCCFC0907800809179004E
:10573000D12CD82A0115110509F4C7C1F8018085BB
:10574000853009F0C2C1C8010E944B426E968FAFEE
:105750006E97843008F4AFC063E0C8010E94A93E90
:10576000FC018184928462E0C8010E94A93EFC0190
:10577000418452846384748461E0C8010E94A93E1C
:105780001C0160E0C8010E94A93EFC012185328510
:10579000438554856D962CAF3DAF4EAF5FAF6D978F
:1057A000C601DD0CAA0BBB0B9C01AD016D96CCAC08
:1057B000DDACEEACFFAC6D972C193D094E095F09CD
:1057C000C401092C000CAA0BBB0BBC01CD01641950
:1057D0007509860997090E94A773F1012185328511
:1057E000438554852C193D094E095F090E94D973E0
:1057F000420E531E641E751E62016E96FFAD6E97BB
:10580000F53009F058C064E0C8010E94A93EFC01CF
:10581000818592858C149D040CF464016E96FFAD15
:105820006E97F23009F053C10D2C000CEE08FF0802
:1058300060E0C8010E94A93EFC0181859285A38594
:10584000B485C816D906EA06FB06C4F5C12CD12CCE
:105850006796EEADFFAD6797828193818C159D05AC
:1058600061F0B601CE018F5A9F4F0E94E7286796DC
:10587000EEADFFAD6797D382C2826796EEADFFAD06
:105880006797818185300CF496C0F501A280B380C2
:10589000A3CE0E947E5FDC01CB01C296A11DB11D8B
:1058A0008093FE059093FF05A0930006B093010638
:1058B00029C160E01BCF81E090E0ACCF61E0C8017E
:1058C0000E94A93EFC0181859285A385B4858C1533
:1058D0009D05AE05BF05CCF6CC24C394D12CB8CF22
:1058E000D11003C010E062E002C011E060E08F2D33
:1058F0000E94085F65962FAD659730E0F901E65686
:10590000F34F8491F901E650F34F0491F901E05C03
:10591000F24FF490FF20A1F081110E94B25EEF2DB2
:10592000F0E0EE0FFF1FE75AF34FA591B491EC9111
:105930000E2331E020E009F430E0832F922F02C0E3
:1059400080E090E0212F30E051E02817390709F07E
:1059500050E0052F10E06796EEADFFAD67976281CE
:1059600073810617170719F14181442319F041503B
:1059700041838BCF64964FAD649740FF0AC02817D0
:10598000390771F461E08081811160E0608370E02B
:1059900002C05083B801CE018F5A9F4F0E94E72862
:1059A0006796EEADFFAD6797138302836ECF93E0EA
:1059B000C92EC1826ACF828193818C159D0509F41D
:1059C00064CF6996DFAECEAE699765961FAD6597D9
:1059D00065E77CE087EA97E00E942E58612F87EA0E
:1059E00097E00E94D13E63E77CE087EA97E00E945F
:1059F0002E58B60187EA97E00E948F3E87EA97E02B
:105A00000E94F85863960EAD1FAD63976AE574E087
:105A1000C8010E94B63E3C0169E674E0C8010E94DC
:105A2000B63E8C01009761F1FC016185728540E40E
:105A300050E0CE0101960E9495786FE270E0CE01B1
:105A400001960E945C78892B51F4F80121853285FA
:105A500043E050E060E4CE0101960E946C554AE0BC
:105A6000BE016F5B7F4F69968EAD9FAD69970E94B7
:105A7000926CBE016F5B7F4FCE0101960E94372072
:105A800061147104D9F0F30161857285CE0101962C
:105A90000E94241ECE0101960E94AE27882371F039
:105AA000E12CF12C01E09E01295A3F4F41E050E0EA
:105AB00060E070E0CE0101960E94BF086796EEADEF
:105AC000FFAD6797D382C282E0CE81E090E0679617
:105AD000EEADFFAD6797228133817601E21AF30ABA
:105AE0009701F7FE03C0319521953109821793077D
:105AF00014F41182C2CE818186300CF0BECE8F5F4D
:105B00008183BBCEC35ADF4F0FB6F894DEBF0FBE02
:105B1000CDBFDF91CF911F910F91FF90EF90DF905C
:105B2000CF90BF90AF909F908F907F906F905F903D
:105B30004F903F902F900895A8950E943F11029793
:105B400024F00E943F4D0E94B62A0C94C22967E3BC
:105B50007CE087EA97E00E942E5864E27CE087EAC6
:105B600097E00E942E5866E17CE087EA97E00E9469
:105B70002E586EE07CE087EA97E00E942E5887EA74
:105B800097E00E94F85861E07CE087EA97E00E9485
:105B90002E5861EF7BE087EA97E00E942E5865EE71
:105BA0007BE087EA97E00E942E586EEC7BE087EA64
:105BB00097E00E942E586CEB7BE087EA97E00E940A
:105BC0002E5867EA7BE087EA97E00E942E5868E942
:105BD0007BE087EA97E00E942E5860E97BE087EA45
:105BE00097E00E942E5865E87BE087EA97E00E94E4
:105BF0002E586BE77BE087EA97E00E942E5863E718
:105C00007BE087EA97E00E942E5867E67BE087EA10
:105C100097E00E942E586DE47BE087EA97E00E94AF
:105C20002E586EE27BE087EA97E00E942E5887EAC2
:105C300097E00C94F858AF92BF92CF92DF92EF9218
:105C4000FF920F931F93CF93DF936C017B018A0127
:105C50000E94917381508E3FA0F45701C0E0D0E0C4
:105C600001501109C017D1077CF4C6018C0F9D1F8C
:105C70000E949173F50181935F01882329F0219699
:105C8000F1CF80E090E005C0CE0DDF1D188281E0ED
:105C900090E0DF91CF911F910F91FF90EF90DF90F7
:105CA000CF90BF90AF900895CF92DF92EF92FF9286
:105CB0000F931F93CF93DF936C01EB0109900020AA
:105CC000E9F72197C61BD70BC032D10514F0CFE1FD
:105CD000D0E08B01E12CF12CEC16FD0664F4F80108
:105CE00061918F01C7018C0D9D1D0E949973FFEF7B
:105CF000EF1AFF0AF1CF60E0C6018C0F9D1FDF9104
:105D0000CF911F910F91FF90EF90DF90CF900C9467
:105D10009973882319F064E47AE002C066E47AE0BB
:105D200087EA97E00C942E58AF92BF92CF92DF9201
:105D3000EF92FF920F931F93CF93DF93CDB7DEB710
:105D4000C856D1090FB6F894DEBF0FBECDBF1AA654
:105D500019A6FE01BB962EE1DF011D922A95E9F7F7
:105D60008E01075D1F4F029774F0FB016281738102
:105D70004FE150E0C8010E949578B80186E190E0BB
:105D80000E94542E10C040E250E0B80186E190E03D
:105D90000E941B2E892B39F440E250E062E27BE046
:105DA000C8010E94586C809107071F928F938091C1
:105DB00006071F928F93809105071F928F93809102
:105DC00004071F928F93809103071F928F938091F6
:105DD00002071F928F9384E994E09F938F931F9201
:105DE00088E28F93CE0101966C019F938F930E945E
:105DF000A4786EE07BE087EA97E00E942E58B80115
:105E000087EA97E00E94FC58B60187EA97E00E9473
:105E1000FC5887EA97E00E94F8580FB6F894A895C6
:105E200080916000886180936000109260000FBED6
:105E30007E0199E4E90EF11CD70113961C921E9283
:105E4000129788EE93E0A0E0B0E0F7018483958399
:105E5000A683B78384E0848789EE92E09183808370
:105E600016870587108A178680E590E0928B818BD4
:105E7000158A6BEA72E387E695E30E94D66C8C0183
:105E80000FB6F894DEBF0FBECDBF892BE1F183E0E2
:105E900090E00E944869D8011D969C938E931C97B0
:105EA000FC01F182E0821282C7010E94EB4288234A
:105EB00019F0C7010E945244D7011F966D917C9141
:105EC00050975196AD90BC9052976115710569F04D
:105ED000CE01815A9F4F0E94FE58A501BE01615A12
:105EE0007F4FC7010E94345307C0F701658576854F
:105EF000A501C7010E94FD55181619060CF49EC095
:105F0000C8010E94403500E010E0F701E388F48802
:105F100099E288E10FB6F894A895809360000FBECF
:105F2000909360000115110509F469C0F8ECEF16B3
:105F3000F10409F058C062E07BE087EA97E00E9434
:105F40002E58A3961FAE1EAEA397A5961FAE1EAEEB
:105F5000A5978FEF9FEFA7969FAF8EAFA79789E783
:105F600092E0A1969FAF8EAFA197A9961FAF0EAFFB
:105F7000A997F8948091FA059091FB050E94E7217A
:105F8000CE01815A9F4F0E9412229093FB0580936D
:105F9000FA057894C8010E9440358091FA059091E5
:105FA000FB05892B79F46BEE7AE087EA97E00E9493
:105FB0002E580E947E5FDC01CB018856954CAF4F76
:105FC000BF4F31C060EE7AE087EA97E00E942E581A
:105FD0000E94834969ED7AE087EA97E00E942E5893
:105FE00082E090E0CBC061EC7AE087EA97E00E9423
:105FF0002E58B70187EA97E00E948F3E0CC06FEAE7
:106000007AE087EA97E00E942E5866E97AE087EA0C
:1060100097E00E942E580E947E5FDC01CB018857DA
:106020009C4EAF4FBF4F8093F6059093F705A0931A
:10603000F805B093F90585EF9FEFA0C0D7011D9635
:10604000BC901D971E96AC90DF92CF9282E99AE0A9
:106050009F938F931F930F930E945F6DDF92CF9258
:106060008DE89AE09F938F931F930F930E945F6D2B
:10607000D8011C96ED91FC911D9781E08283DF92FF
:10608000CF928AE89AE09F938F931F930F930E9479
:106090005F6DD8011C96ED91FC911D971282AF9215
:1060A000BF9284E59AE09F938F931F930F930E9472
:1060B0005F6D8FE89AE09F938F931F930F930E94D9
:1060C0005F6DF701148A138AD8011C96ED91FC913B
:1060D0001D97A080B1800FB6F894DEBF0FBECDBF74
:1060E00083E3C82ED12CD501ED91FC910084F1857C
:1060F000E02DC501199541975CF4B1E0CB1AD108A8
:1061000039F064E170E080E090E00E94445FEBCF02
:106110006E01FFE5CF0ED11CDF92CF9288E49AE0AA
:106120009F938F931F930F930E947C6D0F900F90FE
:106130000F900F900F900F90019709F0E6CEF601A7
:1061400080819181D70154969C938E935397D12C43
:1061500080E08A3039F4BAE0DB1609F4D6CE9AE052
:10616000D92E03C08D3009F0D82EC8010E94216DB0
:106170008F3F79F7C8010E944035C7CEC859DF4F1D
:106180000FB6F894DEBF0FBECDBFDF91CF911F9148
:106190000F91FF90EF90DF90CF90BF90AF90089558
:1061A0000E94942E90939605809395058DE09AE039
:1061B0000C945244CF93DF93EC01E881F98102847F
:1061C000F385E02DCE0119950196B9F7DF91CF91B6
:1061D0000895FC01A285B3851097A9F0868597855F
:1061E000029788F0CD010196938782876C9386850C
:1061F00097850197978786870284F385E02D108223
:1062000081E090E0089580E090E00895FC018681AF
:1062100097818F3F2FEF920729F02FEF3FEF3783C2
:1062200026830895A085B185109789F0248535854A
:106230002115310561F0CD010196918780878C9100
:106240002150310935872487082E000C990B0895B9
:10625000FC0186819781019639F481E0248535859A
:10626000232B19F480E0089581E00895CF92DF9206
:10627000EF92FF920F931F93CF93DF937C016A01FC
:106280008B01C0E0D0E0CC15DD0589F0D701ED91A0
:10629000FC910284F385E02DC70119958F3FBFEF74
:1062A0009B0729F0F80181938F012196ECCFCE0155
:1062B000DF91CF911F910F91FF90EF90DF90CF90E2
:1062C0000895CF93C62FDC01ED91FC910088F189F0
:1062D000E02D1995DC01ED91FC910190F081E02D0C
:1062E0006C2FCF911994CF93DF93EC018E819F8116
:1062F0000196D9F4288539858A859B85820F931F5D
:1063000081159041A0F4E881F9810284F385E02DA4
:10631000CE011995813291056CF3E881F9810684EB
:10632000F785E02D682FCE01199581E001C080E04E
:10633000DF91CF910895062E000C770BFC01778337
:1063400066830895CF93DF93EC018E819F81019640
:1063500011F5E881F9810088F189E02DCE011995C8
:10636000DC01ED91FC910084F185E02D1995892BDC
:10637000A1F0E881F9810284F385E02DCE01199521
:106380008132910534F3E881F9810684F785E02DA7
:10639000682FCE01199581E001C080E0DF91CF9197
:1063A00008950F931F93CF93DF93EC018B016FEB55
:1063B00074E00E94FC5801151105B9F1F8016191D2
:1063C0008F01662391F1603220F0623211F06C355A
:1063D00041F56CE5CE010E94E957F80131978081C3
:1063E0008C30D1F044F48930D9F08A30B9F088305B
:1063F00029F762E616C0823259F024F48D30F1F6A6
:1064000062E70FC08F3231F08C35C1F66CE509C000
:1064100062E207C06FE205C066E603C06EE601C037
:1064200064E7CE010E94E957C9CF62E2CE010E9423
:10643000E95780E090E0DF91CF911F910F9108958F
:10644000FC012085318582859385AC014F5F5F4FCC
:1064500053874287820F931F0E94997381E090E0D7
:106460000895FC01868197818F3F2FEF920729F0D5
:106470002FEF3FEF3783268308952085318582856E
:106480009385AC014F5F5F4F53874287820F931F05
:106490000E949173082E000C990B0895FC018681CF
:1064A00097818F3F2FEF920729F02FEF3FEF378330
:1064B00026830895808591850C94216DCF92DF927B
:1064C000EF92FF92CF93DF93EC018E819F818F3FFC
:1064D0002FEF920759F02FEF3FEF3F832E83DF918D
:1064E000CF91FF90EF90DF90CF9008950E947E5F54
:1064F0006B017C01A4EFCA0EA1E0DA1EE11CF11CC5
:10650000E881F9810088F189E02DCE011995DC013F
:10651000ED91FC910084F185E02D1995892B39F4DA
:106520000E947E5F6C157D058E059F0548F3E8810E
:10653000F9810088F189E02DCE011995DC01ED91FA
:10654000FC910284F385E02DDF91CF91FF90EF90D5
:10655000DF90CF901994EF92FF920F931F93CF93F8
:10656000DF93009719F48FEF9FEF80C0FC01E48464
:10657000F584D7010D911C91D801ED91FC9106880D
:10658000F789E02DC8011995882369F3D801ED91A9
:10659000FC910084F185E02DC8011995D801ED9199
:1065A000FC91892B61F30284F385E02DC8011995D4
:1065B000EC010196C1F2F8018589882329F06C2F3E
:1065C00087EA97E00E94D13ED70112968C918823EA
:1065D00009F44BC0C532D10509F047C0D801ED918F
:1065E000FC910084F185E02DC801199502975CF0BB
:1065F000D801ED91FC910688F789E02DC801199525
:106600008111ECCFB0CFD1E0C0E0D801ED91FC9189
:106610000284F385E02DC80119958F3FBFEF9B07DA
:1066200009F4A1CF9C01215431092A31310530F000
:106630009C01215631092A31310538F48D2F82957C
:10664000807F829FC00D11240AC0C0978A309105B7
:1066500030F49D2F9295907F989FC00D1124D150BA
:10666000A0F68C2FCC0F990B01C0CE01DF91CF91FA
:106670001F910F91FF90EF9008958F929F92AF928C
:10668000BF92CF92DF92EF92FF920F931F93CF931F
:10669000DF936115710509F4FFC0FB010085002E31
:1066A000000C110B220B330B0730110508F0F4C05E
:1066B000DB01EC01F8018827EC53FF4F8F4F0C945E
:1066C0001A7463E374E006C019968C91882389F0EC
:1066D0006EE374E0CE01DF91CF911F910F91FF9097
:1066E000EF90DF90CF90BF90AF909F908F900C94E1
:1066F000525868E374E0EECF19964D915D916D911B
:106700007C911C972AE030E0CE01DF91CF911F9160
:106710000F91FF90EF90DF90CF90BF90AF909F9040
:106720008F900C94B0581996CD90DD90ED90FC9020
:106730001C9720E030E0A901C701B6010E94A574B2
:1067400087FF09C061EC74E0CE010E94FC58F7FAA3
:10675000F094F7F8F094C701B6010E9423754B013D
:106760005C012AE0AB01BC01CE010E94675863ECDA
:1067700074E0CE010E94FC58C501B4010E9452751C
:106780009B01AC01C701B6010E9438742DEC3CECB2
:106790004CE45DE30E94397420E030E040E251E4D3
:1067A0000E9409760E942375AB0160E070E02AE048
:1067B000CE010E94675870C019966D917C911A970E
:1067C000CE01DF91CF911F910F91FF90EF90DF905D
:1067D000CF90BF90AF909F908F900C94D131169630
:1067E0000D911C9117976BE5CE010E94E957019618
:1067F00019F48FEF9FEF52C00115110571F0B80128
:10680000CE010E943D330196A1F3F801028113816C
:106810000115110589F36CE2E7CF6DE52FC01696DF
:106820000D911C9117976BE7CE010E94E9570196D5
:1068300001F30115110509F1F80160817181CE01A3
:106840000E94D1310196A9F26AE3CE010E94E95774
:10685000019679F2B801CE010E943D33019649F2CA
:10686000F801028113810115110519F36CE2CE01C3
:106870000E94E9570196E9F6BCCF6DE7CE010E9470
:10688000E95721E030E0019611F020E030E0882760
:106890009927821B930B02C080E090E0DF91CF919B
:1068A0001F910F91FF90EF90DF90CF90BF90AF902E
:1068B0009F908F900895CF93DF93EC01E881F98149
:1068C0000284F385E02DCE0119958F3F2FEF9207BB
:1068D00071F0E881F9818132910594F30684F7859E
:1068E000E02D682FCE01199580E090E002C08FEF77
:1068F0009FEFDF91CF910895EF92FF920F931F9337
:10690000CF93DF938C017B01DC01ED91FC9102843C
:10691000F385E02D1995829709F078C084E0F7019E
:10692000808786E090E00E944869EC01892B09F499
:106930006DC0E2E0F6E0F983E88380E091E0DF01FA
:106940009C011D9221503040E1F79B838A831D8278
:106950001C82D801ED91FC910284F385E02DC801E1
:1069600019958F3FBFEF9B0709F44DC08232910507
:1069700009F44FC0803291050CF44BC08C35910561
:1069800011F0BE013DC0D801ED91FC910284F38568
:10699000E02DC80119958F3FBFEF9B07A1F182360B
:1069A000910531F15CF48F329105F9F08C35910548
:1069B000C9F0829771F6BE0182E222C08E3691053F
:1069C000D1F034F48636910521F6BE018CE018C072
:1069D0008237910599F08437910509F0BACFBE014D
:1069E00089E00EC0BE018CE50BC0BE018FE208C07D
:1069F000BE0188E005C0BE018AE002C0BE018DE094
:106A00000E949F5BA6CFCE010E94E0698FEF9FEFAF
:106A100024C08C819D81009749F0E881F9818E0F17
:106A20009F1FFC0131978081882321F0BE0180E007
:106A30000E949F5B8C819D810E9448698C01009718
:106A400039F062E076E00E947078CE010E94E06941
:106A5000F7011287018780E090E0DF91CF911F91CD
:106A60000F91FF90EF9008958DE090E00E944869AB
:106A7000009729F02DE0FC0111922A95E9F708957D
:106A80000F931F93CF93DF930097E1F0EC010C85F8
:106A90001D850115110579F0D8018D919C91009704
:106AA00039F0DC01ED91FC910488F589E02D199510
:106AB000C8010E94E069CE01DF91CF911F910F9133
:106AC0000C94BF6CDF91CF911F910F910895AF92FD
:106AD000BF92CF92DF92EF92FF920F931F93CF93CB
:106AE000DF9300D01F92CDB7DEB76115710509F4B1
:106AF00096C06B01182FDB011C96AD90BC901D97C2
:106B0000F501E080F180D701ED91FC910688F789CD
:106B1000E02DC7011995811104C0C6010E944035BE
:106B20007EC0F5019281911114C0D701ED91FC91C5
:106B30000190F081E02D612FC7011995F70185893A
:106B4000882309F469C0612F87EA97E00E94E9571A
:106B500063C0812F8F7D81548A3138F380ED810F9E
:106B60008A3018F383ED810F8230F8F21F35E9F295
:106B70001E37D9F21132B1F086EC810F823090F0DD
:106B80008AED810F873070F01D3361F0812F8F7E89
:106B90008F3241F08DED810F823020F01B3511F0E6
:106BA0001D3511F491FFC1CF19821A821B821C82FC
:106BB000812F012E000C990B9F931F9385EC94E07D
:106BC0009F938F938E010F5F1F4F1F930F930E9410
:106BD000E1786E01F4E0CF0ED11C0F900F900F9072
:106BE0000F900F900F90D701ED91FC910190F081E3
:106BF000E02DD8016C91C7011995F701858988238B
:106C000031F0D8016C9187EA97E00E94E9570F5F55
:106C10001F4F0C151D0539F780E090E002C08FEF83
:106C20009FEF0F900F900F900F90DF91CF911F91DA
:106C30000F91FF90EF90DF90CF90BF90AF900895AD
:106C40002C9A08952C980895CF92DF92EF92FF929C
:106C50000F931F93CF93DF93EC017A018B016C01AB
:106C6000C40ED51ECC15DD05A9F00E9422368FE09A
:106C70000E940F438D2F0E940F438C2F0E940F43C1
:106C8000219680E00E940F43F80181938F010E94BA
:106C90002036E8CFC701DF91CF911F910F91FF9070
:106CA000EF90DF90CF900895CF92DF92EF92FF9216
:106CB0000F931F93CF93DF93EC017A018B016C014B
:106CC000C40ED51ECC15DD05A1F00E94223680EF42
:106CD0000E940F438D2F0E940F438C2F0E940F4361
:106CE0002196F80181918F010E940F430E94203666
:106CF000E9CFC701DF91CF911F910F91FF90EF90E6
:106D0000DF90CF9008951F93CF93DF93D82F192F43
:106D1000C62F0E94223680EF0E940F43812F0E94CF
:106D20000F438D2F0E940F438C2F0E940F430E9410
:106D3000203681E0DF91CF911F9108951F93CF936B
:106D4000DF93182F66E270E00E94A144C82FD0E0C4
:106D500067E270E0812F0E94A144DC2FCC279E01C6
:106D6000282BC901DF91CF911F9108951F93CF93D5
:106D7000DF93182F60E270E00E94A144C82FD0E09A
:106D800061E270E0812F0E94A144DC2FCC279E019C
:106D9000282BC901DF91CF911F9108957F928F9287
:106DA0009F92AF92BF92CF92DF92EF92FF920F939A
:106DB0001F93CF93DF93CDB7DEB7A6970FB6F894A6
:106DC000DEBF0FBECDBF8C01762E942E852E20E225
:106DD000B22ECE0101967C01FC012B2D11922A9539
:106DE000E9F78FE093E09AA389A38FEF8BA38CA39D
:106DF0008DA38EA3680183E4C80ED11C43E450E048
:106E0000BE016F5D7F4FC6010E945047019609F495
:106E1000B9C081E089838A8386E0A82EAB821C8278
:106E2000F80164817581868197810E9422746D8347
:106E30007E838F83988789869A8680E890E09C87F6
:106E40008B874CE150E0B701C6010E94A542F701D3
:106E50002B2D11922A95E9F7480188E0880E911CA4
:106E6000F401D70101900D92AA94E1F740E150E0BE
:106E7000B701C6010E94A542F7011192BA94E9F741
:106E800096E0A92EB12C40E250E0B701C6010E9465
:106E9000A542F1E0AF1AB108B1F783E6898392E821
:106EA0009A8393E59B838C8385E38D8381E08E8336
:106EB0007F829DE3988797E099878A8786E0F4012F
:106EC000DE011B9601900D928A95E1F78CE0898B8B
:106ED0008A8B6BEC74E0CE0143960E947078F801C7
:106EE0006385CE0149960E941E50F8016485CE014B
:106EF0004B960E941E50F8016585CE014D960E946A
:106F00001E504EE150E0B701C6010E94A542F3E0D9
:106F10007F121EC082E3898384E08A83F80196850C
:106F20009B8397859C8390899D8391899E8396E31B
:106F30009F838887828D8987838D8A87848D8B87BD
:106F4000858D8C874CE050E0B701C6010E94A542B8
:106F500087E3898386E08A8391E09B8393E09C8327
:106F60008D838FE08E838AE38F838BE388878FEF17
:106F7000898749E050E0B701C6010E94A542C601D9
:106F80000E947D46A6960FB6F894DEBF0FBECDBF19
:106F9000DF91CF911F910F91FF90EF90DF90CF90F5
:106FA000BF90AF909F908F907F9008952F923F92C7
:106FB0004F925F926F927F928F929F92AF92BF9209
:106FC000CF92DF92EF92FF920F931F93CF93DF93B5
:106FD00000D000D0CDB7DEB78C010E94B46A2FEC90
:106FE00037E040E050E00E94D973DC01CB0101960C
:106FF000A11DB11DF80184839583A683B783808387
:107000009183A283B3835801F3E4AF0EB11CC50191
:107010000E94444464E470E0C5010E945046882305
:1070200009F436C10E947E5F2B013C01812C912C1A
:10703000C8018E5B9F4F9E838D8348EEC42E43E034
:10704000D42EE12CF12C52E0252EAD81BE818C9105
:10705000833009F404C1811120C0F8018481958135
:10706000A681B7810196A11DB11D84839583A68356
:10707000B7830E947E5F6419750986099709A70185
:1070800096010E94B773A90161E0C8010E94CE3643
:1070900081E0AD81BE818C93CAC08430F9F4F801DF
:1070A00084819581A681B7810196A11DB11D84833C
:1070B0009583A683B7830E947E5F6419750986094C
:1070C0009709A70196010E94B773A90163E0C8015F
:1070D0000E94CE36AD81BE812C92A9C0813059F577
:1070E000F80142AD53AD64AD75AD9E012F5F3F4FCA
:1070F000C8010E943350382EF2E08F1392C089816C
:107100009A81AB81BC81F80184839583A683B78380
:107110000E947E5F6419750986099709A701960187
:107120000E94B773A90163E0C8010E94CE36AD8109
:10713000BE813C927CC0823009F079C0F80142AD3A
:1071400053AD64AD75AD9E012F5F3F4FC8010E94E6
:107150003350382EF5E08F135DC0E3E0AD81BE8182
:10716000EC93F80182A193A1A4A1B5A1892B8A2B4C
:107170008B2B41F484E893E0A0E0B0E082A393A3DA
:10718000A4A3B5A3F80186A197A1A0A5B1A5892BB9
:107190008A2B8B2B61F482A193A1A4A1B5A1B695F2
:1071A000A7959795879586A397A3A0A7B1A7F80160
:1071B00082A593A5A4A5B5A5892B8A2B8B2BA9F411
:1071C00082A193A1A4A1B5A1AC01BD0123E0769554
:1071D0006795579547952A95D1F7841B950BA60B74
:1071E000B70B82A793A7A4A7B5A7F80186A197A17B
:1071F000A0A5B1A586A797A7A0ABB1AB82A593A583
:10720000A4A5B5A582AB93ABA4ABB5AB88248394FE
:10721000912C0DC0F6E08F1304C0AD81BE811C928D
:1072200006C0BFEF3B1203C0ED81FE811082F1E08A
:107230008F16910409F409CF0E947E5FDC01CB0117
:1072400084199509A609B709F80126A937A940ADFF
:1072500051AD281739074A075B0708F0F6CEC5017C
:107260000E944444F80184819581A681B7810196EA
:10727000A11DB11D84839583A683B7830E947E5F81
:10728000F801FE966083718382839383C40102C0F8
:1072900080E090E026960FB6F894DEBF0FBECDBF1B
:1072A000DF91CF911F910F91FF90EF90DF90CF90E2
:1072B000BF90AF909F908F907F906F905F904F9016
:1072C0003F902F900895CF93DF93FC010190002011
:1072D000E9F79F01281B390B285F3F4F2138310503
:1072E00070F5EC010E94AE1F882349F18091D80807
:1072F0009091D908019611F481E090E09093D9081B
:107300008093D8088091D8089091D90890935D080F
:1073100080935E0847E050E068E578E0CE010E9487
:10732000251FFC01EE5AF74F1682AC01445051095B
:1073300068E578E082E8DF91CF910C94451F80E00A
:10734000DF91CF910895CF92DF92EF92FF920F934A
:107350001F93CF93DF936C018B017B0182E0E80EDA
:10736000F11CC0E0D0E0C6018C0F9D1F0E949173FC
:10737000F70181937F012196C430D105A1F7F8016F
:107380009281992319F081E09F3F09F480E090E019
:10739000DF91CF911F910F91FF90EF90DF90CF90F1
:1073A0000895EF92FF920F931F93CF93DF937C0189
:1073B0008B010E5F1F4FC0E0D0E0F80161918F019B
:1073C000C7018C0F9D1F0E9499732196C430D1056F
:1073D000A1F7DF91CF911F910F91FF90EF9008954A
:1073E000FC01DC018D918111FDCF40E050E020E0F7
:1073F00030E08AE09191992301F1243031055CF568
:107400009E3271F44F3F510509F02CF5DB01A20FBC
:10741000B31F12964C932F5F3F4F40E050E0EACFEE
:10742000849FD001859FB00D1124492F990F550BD2
:10743000405351094A0F5B1FDDCF4F3F510509F003
:1074400054F4243031053CF4FB01E20FF31F428376
:1074500081E090E0089580E090E008954F925F927F
:107460006F927F928F929F92AF92BF92CF92DF9254
:10747000EF92FF920F931F93CF93DF93CDB7DEB7B9
:1074800063970FB6F894DEBF0FBECDBF7C015B01E2
:107490003A01FB0120E080E090E06AE03191332383
:1074A00009F140ED430F4A3080F4689FA001699FC5
:1074B000500D1124CA01C097830F911D37FD9A9575
:1074C0008F3F910559F350F313C03E3289F42330B6
:1074D00079F0D301A20FB11D12968C932F5F80E03B
:1074E00090E0DCCF233021F4F301858381E021C0DB
:1074F000F7014281538164817581809146089091A2
:107500004708A0914808B0914908481759076A07E9
:107510007B0709F49BC10E947E5F8701085F1F4FB4
:107520006F7077277C5FC8010E945046813019F048
:1075300080E090E0FEC18FE093E09A838983F701B9
:1075400082819381A481B5818B839C83AD83BE832B
:1075500045E350E0BE016F5F7F4FC8010E94504776
:10756000892B19F4C12CD12C6CC10E947E5FF701CC
:10757000778366837627672776277A83698342E055
:1075800050E0BE016F5F7F4FC8010E94A54281E0BD
:1075900090E09E878D8742E050E0BE01635F7F4FA1
:1075A000C8010E94A54280E091E09E878D8742E05D
:1075B00050E0BE01635F7F4FC8010E94A5421E8656
:1075C0001D8642E050E0BE01635F7F4FC8010E940C
:1075D000A54242E050E0BE01635F7F4FC8010E94B8
:1075E000A54242E050E0BE01635F7F4FC8010E94A8
:1075F000A5424501F5018081882301F1640156010E
:10760000F60181912F01882321F08E3211F0620161
:10761000F6CFC818D9081C141D0474F4CF8641E0B5
:1076200050E0BE01615F7F4FC8010E94A542A601E4
:10763000B401C8010E94A5424201DCCF1F8641E08F
:1076400050E0BE01615F7F4FC8010E94A542C12C7E
:10765000DD24D394DE86CD8642E050E0BE01635F38
:107660007F4FC8010E94A542DE86CD8642E050E0F1
:10767000BE01635F7F4FC8010E94A542C8010E94FE
:107680007D46892B09F46ECFE3E0AE2EB12C2301A9
:1076900022E0420E511C0E947E5F3B014C01C8015A
:1076A0000E94D74518161906BCF00E947E5FDC01C7
:1076B000CB0186199709A809B909813A9F40A1050C
:1076C000B105E8F4A8950E94B62A61E070E080E078
:1076D00090E00E94445FE3CFF701428153816481CF
:1076E0007581808D918DA28DB38D481759076A07DA
:1076F0007B0749F4848D958DC59729F409C0CC2466
:10770000CA94DC2C92C05EEFC52EDD24DA948DC0C5
:10771000F70181A192A10C970CF4A0C04CE050E0BD
:10772000BE016F5F7F4FC8010E948F458B819C8196
:107730009827892798279A8B898B29813A81322724
:1077400023273227F701468157812417350709F08F
:1077500080C097FF7EC08F709270892B09F0E4C0C3
:107760006F8078847624672476246114710409F488
:10777000D6C0C12CD12C8D819E819827892798272E
:10778000C816D90608F46FC0812C912C41E050E056
:10779000BE016D5E7F4FC8010E948F458B89982F77
:1077A000907C09F092C0811186C042E050E0BE0199
:1077B000615F7F4FC8010E948F4542E050E0BE01EB
:1077C000635F7F4FC8010E948F45C8010E94AE458C
:1077D000C8010E94AE45C8010E94AE45C8010E9482
:1077E000AE4542E050E0BE016F5E7F4FC8010E948F
:1077F0008F458F8598898115914009F06EC0CD84A1
:10780000DE84DC24CD24DC2481E0C816D10409F018
:1078100064C089899A898115944009F07BC044E04D
:1078200050E0B201C8010E948F45A8950E94B62A77
:1078300081E0A81AB10829F0FFEFCF16DF0609F49E
:107840002ACFC8010E944444C60173C08EEF9FEF47
:1078500070C04CEFC42EDD24DA94E7CF9DEFC92E23
:10786000DD24DA94E2CF41E050E0BE01635F7F4F58
:10787000C8010E948F458D85882351F08D859FEF2B
:10788000980F9D87882321F0C8010E94AE45F6CF4E
:107890008D858111E8CFC8010E94AE45C8010E94C4
:1078A000AE45C8010E94AE45C8010E94AE45FFEF3B
:1078B000CF1ADF0A60CF8B899FEF980F9B8B8823AD
:1078C00041F0C8010E94AE45F6CFC8010E94AE4506
:1078D0001B8A8B8981115ACF68CFC12CD12C898901
:1078E0009A89982789279827C816D90638F4C80195
:1078F0000E94AE45FFEFCF1ADF0AF1CF2FEF821AB9
:10790000920A6814790409F041CF26EFC22EDD24D3
:10791000DA948BCF77EFC72EDD24DA9486CF3AEF57
:10792000C32EDD24DA9481CF8BEFC82EDD24DA94C8
:107930007CCF63960FB6F894DEBF0FBECDBFDF914C
:10794000CF911F910F91FF90EF90DF90CF90BF905C
:10795000AF909F908F907F906F905F904F90089521
:107960001F93CF93DF93282F30E0F901E656F34FB2
:107970008491F901E650F34FD491F901E05CF24FA4
:10798000C491CC23C1F0162F81110E94B25EEC2F5E
:10799000F0E0EE0FFF1FE058F34FA591B4919FB7B1
:1079A000F894111104C08C91D095D82302C0EC91A9
:1079B000DE2BDC939FBFDF91CF911F9108951F9322
:1079C000CF93DF931F921F92CDB7DEB76CE271E0C9
:1079D00080E090E00E94445F1FB7F8948091080710
:1079E000811127C0E5E7FDE08491EFE2FDE094918D
:1079F000E82FF0E0EE0FFF1FE052F34FA591B49196
:107A0000EC91E92321F461E085E30E94B03C61E060
:107A100085E30E94085F8CB580618CBD8CB5806465
:107A20008CBD61E084E30E94085F61E083E30E9413
:107A3000085F809108078F5F809308071FBF249A13
:107A4000CE0101960E94432289819A810E94A6520A
:107A500067E080E090E00E94833665E58BE190E08E
:107A60000E94833665E58AE190E00E9483360E9499
:107A7000A55280E090E49093DD058093DC0580E0E2
:107A800090E69093E5058093E40580E098E4909378
:107A9000DF058093DE0580E098E69093E70580930C
:107AA000E60580E090E59093E1058093E00580E0B5
:107AB00090E79093E9058093E80580E098E590933E
:107AC000E3058093E20580E098E79093EB058093CF
:107AD000EA050F900F90DF91CF911F910895AF921B
:107AE000BF92CF92DF92EF92FF920F931F93CF93AB
:107AF000DF931F921F92CDB7DEB75C018B016A0145
:107B000079010E94DF3CCE0101960E9443228981C7
:107B10009A810E94A65246E050E062E077E089E058
:107B200090E00E945436C50102960E949052C60110
:107B300002960E949E52C70102960E9497520E948E
:107B4000A552F80182819381A481B58180934C086C
:107B500090934D08A0934E08B0934F080F900F904C
:107B6000DF91CF911F910F91FF90EF90DF90CF9019
:107B7000BF90AF900895CF92DF92EF92FF92CF9394
:107B8000DF93CDB7DEB768970FB6F894DEBF0FBEB0
:107B9000CDBFFA012FE033E03A8329835FEF5B83A7
:107BA0005C835D831E8238872F83C280D380E4800C
:107BB000F580C986DA86EB86FC863E872D87FB0139
:107BC00042815381648175814F87588B698B7A8B91
:107BD0003C8B2B8BFC0182819381A481B5818D8BA1
:107BE0009E8BAF8BB88F9E012F5F3F4FAE01495FD9
:107BF0005F4FBE01635F7F4FCE0143960E946F3D92
:107C000068960FB6F894DEBF0FBECDBFDF91CF915F
:107C1000FF90EF90DF90CF9008950F931F93CF9335
:107C2000DF93CDB7DEB768970FB6F894DEBF0FBE0F
:107C3000CDBFFB01DC0112964D915D916D917C9160
:107C400015974D8B5E8B6F8B788F8FE093E09A83C7
:107C5000898321E0288F0D891E892F89388D0B8318
:107C60001C832D833E8398878F8302811381248117
:107C7000358109871A872B873C879E878D874F8799
:107C8000588B698B7A8BAE014F5F5F4FBE01695F86
:107C90007F4FCE010D960E94BB3D68960FB6F894BB
:107CA000DEBF0FBECDBFDF91CF911F910F91089521
:107CB000CF93DF93CDB7DEB762970FB6F894DEBFF0
:107CC0000FBECDBFFC0182819381A481B5818F87D6
:107CD000988BA98BBA8B2FE033E03A83298341E05C
:107CE0004A8B4F85588969897A894B835C836D8378
:107CF0007E8338872F8389879A87AB87BC87BE01AD
:107D00006F5F7F4FCE0107960E940D3E62960FB6C1
:107D1000F894DEBF0FBECDBFDF91CF910895AB01C8
:107D2000770F660B770B2AE030E00C94B0580F9376
:107D30001F93CF93DF93EC010E942E588C01CE014C
:107D40000E94F858800F911FDF91CF911F910F91E2
:107D50000895FC0186819781009739F0662329F008
:107D60006150FC0182819381F7CF08950F931F9397
:107D7000CF93DF938B01FC01C681D781209759F007
:107D8000B801888199810E943E78892B21F00A8070
:107D9000DB81C02DF3CFCE01DF91CF911F910F91E9
:107DA0000895462F50E060E070E02AE00C94675898
:107DB000DC011696ED91FC91179761157105A1F004
:107DC000309729F417967C936E93169708958281C5
:107DD0009381009711F0FC01FACF73836283DB017A
:107DE0001596FC93EE9314970895CF92DF92EF923D
:107DF000FF920F931F93CF93DF938C017B016A0156
:107E00000E943435EC01892B09F182E08887A601B4
:107E1000DD0C660B770B49875A876B877C878881D7
:107E20009981009711F00E94E069C7010E940578CE
:107E300099838883BE01C801DF91CF911F910F9173
:107E4000FF90EF90DF90CF900C94D83EDF91CF91D0
:107E50001F910F91FF90EF90DF90CF900895CF92F8
:107E6000DF92EF92FF921F93CF93DF93EC016A01B1
:107E70007B01122FE889F98982E080834115514EF8
:107E800061057105B1F060E079E08DE390E0A70154
:107E900096010E94B773DA01C9010197A109B109DE
:107EA000B695A795979587959C01211580E1380790
:107EB000A8F0E889F989108260E874E88EE190E022
:107EC000A70196010E94B773DA01C9010197A109C0
:107ED000B109B695A795979587959C01EC85FD8589
:107EE0003083EE85FF852083188EEC89FD89108311
:107EF000EA89FB89808180618083EA89FB898081AE
:107F000088608083EA89FB89808180688083EA8930
:107F1000FB8980818F7D8083DF91CF911F91FF90BE
:107F2000EF90DF90CF9008958F929F92AF92BF9283
:107F3000CF92DF92EF92FF920F931F93CF93DF9335
:107F4000CDB7DEB7DA950FB6F894DEBF0FBECDBF62
:107F5000C82E8091F5088983CA8221E0C216A0F05C
:107F600074E07C1518F487E1C8120EC08091F60801
:107F70009091F7089B838C838091F8089091F90881
:107F80009D838E8386E001C082E08E010F5F1F4FCC
:107F900090E19C1528F0AFE0CA1630F49BEF01C0C9
:107FA0009AEE9C0D923078F420917A0990917B0999
:107FB000F801E80FF11D908391E0980FF801E90FA7
:107FC000F11D8E5F2083BFE0CB1641F1BC1558F048
:107FD000E5E0CE16A1F0F6E0CF12B6C020917E0902
:107FE00090917F0910C026E1C21609F48EC077E196
:107FF000C71609F459C090E1C912A6C055C0209116
:108000007C0990917D09F801E80FF11D908391E0C2
:10801000980FF801E90FF11D8E5F95C020917C0942
:1080200030917D09F801E80FF11D308342E0480FDF
:1080300091E0980FF801E90FF11D2083B9016770F5
:108040007727A3E036952795AA95E1F7672B19F0D6
:1080500091E0920F01C0922FB3E0B80FF801E40F46
:10806000F11D90838C5F60E070E0A0E04FEF480F5F
:108070009A1303C08B2F890F67C050E09B01359581
:108080002795400F511F220F331FF901E258F64F79
:10809000A0FD02C0208101C02181FA012083AF5FD1
:1080A0006F5F7F4F8F5FE2CF20917C0930917D0918
:1080B000F801E80FF11D308391E0980FF801E90F06
:1080C000F11D208392E0980FF801E90FF11D8D5FFB
:1080D000922F990F908390E03327E92FF0E0E21779
:1080E000F30794F5EE0FFF1FE258F64F50814181E0
:1080F000F801E80FF11D408341E0480FF801E40F5B
:10810000F11D8E5F50839F5FE8CF90917E09209193
:108110007F09F801E80FF11D208321E0280FF80105
:10812000E20FF11D9083209180099091810932E046
:10813000380FF801E30FF11D908393E0980FF801D9
:10814000E90FF11D8C5F20837801F8012FEF3FEFDD
:10815000D02E9E2F901B9817A0F49191292748E0CC
:1081600050E0B9017695679520FF06C09B0191E02C
:10817000292790EA392701C09B014150510989F70D
:10818000E8CFF801E80FF11D2083B2E0BB2EB80E56
:108190008F5FF801E80FF11D3083F801EB0DF11D41
:1081A00010828091F3089091F408DC01ED91FC912C
:1081B0000284F385E02D1995019699F7E091090A5B
:1081C000F0910A0A309709F019958091F30890917F
:1081D000F4082E2D2D192B1558F4F70161917F010C
:1081E000DC01ED91FC910190F081E02D1995EDCF2E
:1081F000DC01ED91FC910680F781E02D1995E0916D
:108200000B0AF0910C0A309709F019950E947E5FD5
:108210004B015C01A8E0EA2EF12CD12C8091F308EF
:108220009091F408DC01ED91FC910084F185E02D42
:108230001995892BC1F08091F3089091F408DC0125
:10824000ED91FC910284F385E02D19959091F5084C
:10825000891711F0FF2099F1F801EF0DF11D8083CE
:10826000EA94F39407C0E091070AF091080A309766
:1082700009F01995B5E0FB1222C0EA818E2F8F77A5
:1082800090E08C159D0509F0A2C0E7FF04C08B812A
:10829000882381F181C08E2F90E0FC013197E73176
:1082A000F10568F48827E553FF4F8F4F0C941A743B
:1082B000F3E0EF2E04C0EB8002C0E5E0EE2E0E945A
:1082C0007E5FDC01CB0188199909AA09BB09813DB0
:1082D0009740A105B10538F480E0EE2031F0882305
:1082E00009F49CCF59C082EEF8CF811155C0F4E05B
:1082F000FF15C0F58FEF9FEF60E0EF2DF0E09F01DD
:1083000022503109462F50E0D80142175307BCF4E0
:10831000A40FB51F4C91842748E050E0DC01B695CE
:10832000A79580FF06C0CD0171E0872770EA9727E7
:1083300001C0CD014150510989F76F5FE3CFA20F12
:10834000B31F2C9130E0AC0155274217530709F0B9
:1083500040C0892F9927EC0FFD1F208130E0821744
:108360009307B9F58A818530B0F58330B0F5813057
:1083700090F05B81652F70E0759567952091060AF6
:1083800040E0842F90E0861797070CF452C02093AA
:10839000060A50FD6CC080E01092000A1092020A9A
:1083A0001092010A1092050AD3950FB6F894DEBF19
:1083B0000FBECDBFDF91CF911F910F91FF90EF9036
:1083C000DF90CF90BF90AF909F908F90089581EEF7
:1083D000E3CF83EEE1CF8731F1F66B8170E07595E5
:1083E00067952091060A40E0842F90E08617970752
:1083F0001CF02093060ACFCF4034C0F49C012E5FBE
:108400003F4F220F331F880F991FFC01ED50F74F8C
:10841000DE01A20FB31F8C9190E0982F8827D8011E
:10842000A20FB31F2C91822B90878783242F4F5F3D
:10843000DBCF4034C8F4880F991FFC01ED50F74F93
:10844000A5E0B0E0AC0FBD1FA80FB91F2C9130E024
:10845000322F2227A4E0B0E0AC0FBD1FA80FB91F38
:108460008C91282B30872783242F4F5F8ACF40346D
:1084700068F4880F991FFC01ED50F74FDE01A80F3B
:10848000B91F14968C9190E09087878381E0840FC8
:108490008093060A80CFDC011696ED91FC91179728
:1084A00080E0309729F08F5F0280F381E02DF9CFD3
:1084B00008950895CF93DF931F92CDB7DEB76983F8
:1084C000DC01ED91FC910280F381E02D41E050E070
:1084D000BE016F5F7F4F19950F90DF91CF91089587
:1084E000FC01818D928D0895FC0184899589089500
:1084F0002FE033E0FC0131832083FB014089518967
:1085000062897389FC014283538364837583089570
:10851000DC01ED91FC91048CF58DE02D199480E047
:108520000895FC019485FB018485981303C081E0C4
:10853000943009F480E0089521E0FC0184858430C2
:1085400009F420E0822F089508958F929F92AF92B0
:10855000BF92DF92EF92FF920F931F93CF93DF931F
:108560001F921F92CDB7DEB77C014B018A01FC013F
:10857000A688B788D08CCE0101960E9443228981BB
:108580009A810E94A6528D2D0E9402508017910759
:1085900020F48D2D0E9402508C019801A401B50198
:1085A0008D2D0E949D4F0E94A552F70186899789C3
:1085B000800F911F978B868BC8010F900F90DF91D2
:1085C000CF911F910F91FF90EF90DF90BF90AF90F0
:1085D0009F908F900895CF93DF93FC0124852430E2
:1085E000D1F0EC010E944822843181F0882371F09F
:1085F000883161F08C3161F4E881F9810084F18582
:10860000E02DCE01199521E0892B19F420E001C05D
:1086100021E0822F01C080E0DF91CF9108958EBDCF
:1086200000000DB407FEFDCF8EB50895DF92EF92E6
:10863000FF920F931F93CF93DF931F921F92CDB79B
:10864000DEB7D82ECE0101960E94432289819A81FD
:108650000E94A652E12CF12C8D2D0E949E368C0199
:10866000892B21F08D2D0E949E367C010E151F0551
:1086700099F70E94A552C8010F900F90DF91CF91FA
:108680001F910F91FF90EF90DF900895FC011382EE
:10869000128288EE93E0A0E0B0E084839583A68305
:1086A000B78381E293E0918380838FE093E09787A3
:1086B0008687108A118A128A138A84E0808F08952F
:1086C000AF92BF92CF92DF92EF92FF920F931F93E0
:1086D000CF93DF93CDB7DEB7AF970FB6F894DEBF79
:1086E0000FBECDBF7C015B016A010FE013E01A836E
:1086F00009831B821C821D821E82CE0109960E9464
:1087000046431BA70AA71CA61DA61EA61FA680914E
:108710004C0890914D08A0914E08B0914F088EA33F
:108720009FA3A8A7B9A78B839C83AD83BE8318861C
:108730001F82AE01465D5F4FB501CE0101960E94DA
:108740002E3A81309105B1F4D701ED91FC91048866
:10875000F589E02D1DA30CA38CA59DA5AEA5BFA5F5
:108760008EA39FA3A8A7B9A7A601BE016C5D7F4FEA
:10877000C7011995AF960FB6F894DEBF0FBECDBFF7
:10878000DF91CF911F910F91FF90EF90DF90CF90ED
:10879000BF90AF9008959B0190E00496982F882792
:1087A000642F820F931F0C9483361F93CF93DF9314
:1087B0001F921F92CDB7DEB7182FCE0101960E94EF
:1087C000432289819A810E94A65260E170E0812F44
:1087D0000E9433224FEF62E070E0812F0E94CB4372
:1087E0000E94A5520F900F90DF91CF911F91089595
:1087F000DF92EF92FF920F931F93CF93DF931F921D
:108800001F92CDB7DEB7182FD62E7A01022F0E9405
:10881000D543CE0101960E94432289819A810E940C
:10882000A6524D2D402B60E070E0812F0E94CB437B
:10883000E114F10459F4E0907D0AF0907E0A8FEF84
:10884000E81AF80AF0927E0AE0927D0A4F2D64E061
:1088500070E0812F0E94CB434E2D65E070E0812FA8
:108860000E94CB4361E070E0812F0E9433220E947E
:10887000A55281E00F900F90DF91CF911F910F9142
:10888000FF90EF90DF900895CF93DF93FC01808DF0
:10889000843029F0EF010E94D54384E0888FDF9176
:1088A000CF910895CF92DF92EF92FF920F931F9393
:1088B000CF93DF931F921F92CDB7DEB7FC01F484F4
:1088C000F4E0FF1699F18C01CE0101960E9443223B
:1088D00089819A810E94A65268E070E08F2D0E94E3
:1088E00033220E94A5520E947E5F6B017C01C80169
:1088F0000E9448228823B9F062E370E080E090E0B3
:108900000E94445F0E947E5FDC01CB018C199D09AF
:10891000AE09BF09883E9340A105B10540F3F801B7
:1089200084850E94D54384E0F80184870F900F90DE
:10893000DF91CF911F910F91FF90EF90DF90CF903B
:108940000895CF93DF9390E00496982F8827EC0149
:10895000C60FD71F0E9422368FE00E940F438D2F33
:108960000E940F438C2F0E940F4380E00E940F4310
:10897000C82F0E9420368C2FDF91CF910895CF927F
:10898000DF92FF920F931F93CF93DF931F921F925B
:10899000CDB7DEB7F82E6B01CE0101960E944322BF
:1089A00089819A810E94A65268E270E08F2D0E9410
:1089B000A144082F10E069E270E08F2D0E94A144CD
:1089C000702F6627682B21E030E0A6018F2D0E94D2
:1089D000554F0E94A55281E090E00F900F90DF91DB
:1089E000CF911F910F91FF90DF90CF900895CF937B
:1089F000DF931F92CDB7DEB7FC01218D328D232B83
:108A000049F0BE016F5F7F4F808D0E94BF44898116
:108A100090E002C08FEF9FEF0F90DF91CF9108950C
:108A20008F929F92BF92CF92DF92EF92FF920F931D
:108A30001F93CF93DF931F921F92CDB7DEB7B82E4F
:108A40006B017A01CE0101960E94432289819A81AD
:108A50000E94A652812C912C8B2D0E949E368C0157
:108A6000892B21F08B2D0E949E364C01081519058B
:108A700099F70115110599F463E070E08B2D0E94C0
:108A8000A1448431D9F18823C9F101E010E08C318F
:108A900011F400E010E01195019511092FC0E016C6
:108AA000F1060CF487011016110644F568E270E037
:108AB0008B2D0E94A144E82EF12C69E270E08B2DF1
:108AC0000E94A144FE2CEE24E82A9801A601B701D9
:108AD0008B2D0E94554FE00EF11E4F2D68E270E085
:108AE0008B2D0E94CB434E2D69E270E08B2D0E94AE
:108AF000CB4360E470E08B2D0E9433220E94A5528C
:108B0000C8010F900F90DF91CF911F910F91FF90AF
:108B1000EF90DF90CF90BF909F908F900895CF936C
:108B2000DF93FC01218D328D2115310519F48FEF72
:108B30009FEF11C0EC014217530708F0A901888D7F
:108B40000E9410451816190694F7298D3A8D281B96
:108B5000390B3A8F298FDF91CF9108950F931F938F
:108B6000CF93DF931F92CDB7DEB7FC01218D328DFD
:108B7000232B61F08C0141E050E0BE016F5F7F4F1D
:108B8000808D0E941045181619061CF08FEF9FEF7C
:108B900008C0F801818D928D0197928F818F898114
:108BA00090E00F90DF91CF911F910F9108950F9357
:108BB0001F93CF93DF93CDB7DEB728970FB6F89406
:108BC000DEBF0FBECDBF8C01D80159968D919C910F
:108BD0005A97892B41F0ED91FC910284F385E02DA9
:108BE000C8011995F1CFF801808D0E94164318161F
:108BF000190654F548E050E0BE016F5F7F4FD80181
:108C000058968C910E94104518161906FCF4D8014C
:108C1000509684E0FE01319601900D928A95E1F71D
:108C20008D8190E0982F88272E81820F911DF80169
:108C3000958B848B8F8190E0982F88272885820FD1
:108C4000911D928F818F02C080E090E028960FB630
:108C5000F894DEBF0FBECDBFDF91CF911F910F9172
:108C600008951F93CF93DF931F921F92CDB7DEB766
:108C7000182FCE0101960E94432289819A810E9479
:108C8000A65263E070E0812F0E94A144182F0E9439
:108C9000A552812F0F900F90DF91CF911F910895D2
:108CA000EF92FF921F93CF93DF93FC01208D24302E
:108CB00011F080E01CC07B01EC0110E0812F0E94CC
:108CC0003146811102C0188F05C08831E1F31F5F62
:108CD0001430A1F7888D843061F3FD86EC861A8EFE
:108CE000198E20E0A70162E00E94F84381E0DF9145
:108CF000CF911F91FF90EF9008951F93CF93DF9333
:108D00001F921F92CDB7DEB7FC01108DCE010196E8
:108D10000E94432289819A810E94A65260E270E0FB
:108D2000812F0E94332262E070E0812F0E94A144D3
:108D300084FD1DC062E070E0812F0E94A14483FF8A
:108D40000BC048E162E070E0812F0E94CB430E949B
:108D5000A55280E090E015C00E94A552CE01019678
:108D60000E94432289819A810E94A652DCCF40E171
:108D700062E070E0812F0E94CB430E94A55281E007
:108D800090E00F900F90DF91CF911F910895CF93B6
:108D9000DF93C82FD62F472F60E170E00E94CB43AE
:108DA0004D2F61E170E08C2FDF91CF910C94CB437C
:108DB00090E0982F882744E050E0845F9B4F0C940C
:108DC0005436BF92CF92DF92EF92FF920F931F9390
:108DD000CF93DF9300D000D0CDB7DEB7FC01208D5C
:108DE000243009F04CC06A017B018C01B12C63E096
:108DF00070E08B2D0E94A144811103C0F801B08E58
:108E000006C08831D9F3B394F4E0BF12F0CFF80173
:108E1000808D8430A1F196E0E7E1F3E0DE01119668
:108E200001900D929A95E1F7F70193819F779C83CA
:108E300094819D8395819E83B7016E5F7F4F0E94D1
:108E4000D846B601F801808D0E94C746F801808D92
:108E500090E0982F882746E050E0BE016F5F7F4F7B
:108E60008A5F9B4F0E945436F801128E118E20E8C3
:108E7000A60162E0808D0E94F84381E001C080E09D
:108E800026960FB6F894DEBF0FBECDBFDF91CF910F
:108E90001F910F91FF90EF90DF90CF90BF900895BA
:108EA000DF92EF92FF920F931F93CF93DF931F9266
:108EB0001F92CDB7DEB7FB01DC0157961C921E92C4
:108EC00056972281211109C02381211106C02481D6
:108ED000211103C025812223F1F041155105D9F05C
:108EE0007A018F01FC01D08CCE0101960E944322B1
:108EF00089819A810E94A652B8016E5F7F4F8D2DA5
:108F00000E94D846B7018D2D0E94C7460E94A552E7
:108F100081E090E002C080E090E00F900F90DF9140
:108F2000CF911F910F91FF90EF90DF9008956DE228
:108F30007FE087EA97E00C942E58CF93DF931F923F
:108F4000CDB7DEB71982892B21F0FB0162817381D5
:108F500003C0BE016F5F7F4F86E390E00E94542EF6
:108F60006EE570E187EA97E00E942E580F90DF913E
:108F7000CF910895CF93DF93C0E0D0E060E0CE01C1
:108F80000E9499732196C11582E0D807B9F76EE463
:108F900070E187EA97E0DF91CF910C942E580F9300
:108FA0001F93CF93DF93CDB7DEB72C970FB6F8940E
:108FB000DEBF0FBECDBF8B012FE033E03A832983A4
:108FC0001B821C821D821E8238872F8319861A8677
:108FD0001B861C8683309105B9F144F481309105DC
:108FE00009F454C0029709F443C057C08430910576
:108FF000B9F0059709F051C0BE01695F7F4FF801D4
:10900000808591850E94F039BE01892B19F0695F36
:109010007F4F02C06F5F7F4F82E190E00E94D139A5
:10902000BE01695F7F4FF801868197810E94F03908
:10903000BE01892B19F0695F7F4F02C06F5F7F4FC0
:109040008EE090E00E94D139BE01695F7F4FF80148
:10905000848195810E94F039BE01892B19F0695FE6
:109060007F4F02C06F5F7F4F8AE090E00E94D1394E
:10907000BE01695F7F4FF801828193810E94F039C0
:10908000BE01892B21F0695F7F4F03C0BE016F5F76
:109090007F4F86E090E00E94D13967E470E187EA73
:1090A00097E00E942E582C960FB6F894DEBF0FBEA4
:1090B000CDBFDF91CF911F910F910895CF93DF9393
:1090C000CDB7DEB72C970FB6F894DEBF0FBECDBF7D
:1090D0001C821B821E821D828FEF9FEF98878F83D9
:1090E0008AE593E09A83898386E490E09A8789876A
:1090F0001C861B866DE270E187EA97E00E942E587D
:109100006091FA057091FB05CE0101960E943D33F6
:109110006FEFCE0101960E9420326DE170E187EA87
:1091200097E00E942E582C960FB6F894DEBF0FBE23
:10913000CDBFDF91CF9108950F931F93CF93DF930E
:10914000CDB7DEB769970FB6F894DEBF0FBECDBFBF
:109150008FE290E09A838983FE01339687E1DF01F5
:109160001D928A95E9F768E070E187EA97E00E942E
:109170002E5822E037E0DE011196AE01435F5F4FCB
:109180008D01F90161919F01862F90E074E0959522
:1091900087957A95E1F78B5B9C4FFC018081119656
:1091A0008C931197E62FEF70F0E0EB5BFC4F808122
:1091B00012968C9312971296A417B50711F71E8674
:1091C00062ED74E0C8010E945178B80187EA97E027
:1091D0000E94FC58C8010E9463391E866AED74E043
:1091E000C8010E945178B80187EA97E00E94FC58B4
:1091F00064EE74E0C8010E94DC2169960FB6F89411
:10920000DEBF0FBECDBFDF91CF911F910F910895AB
:10921000CF93C1E068EE73E080E090E00E94445F8D
:109220006C2F87EA97E00E94D13ECF5FC43191F75F
:10923000CF9108950F931F93CF93DF93CDB7DEB7F0
:1092400028970FB6F894DEBF0FBECDBF0E94A72DA2
:1092500066E87DE087EA97E00E942E58CE010196ED
:109260000E94E74ECE0101960E94914E0FE013E05E
:109270001A8309831B821C821D821E82CE010796DF
:109280000E9443228F8198850E94A65244E050E0BC
:10929000BE016D5F7F4F81E090E00E9424360E9406
:1092A000A552CE0101960E94914E1A8309831B821A
:1092B0001C821D821E82CE0107960E9443228F814E
:1092C00098850E94A65244E050E0BE016D5F7F4F3A
:1092D00085E090E00E9424360E94A552CE010196BE
:1092E0000E94914E6CEA7DE087EA97E00E942E583A
:1092F00028960FB6F894DEBF0FBECDBFDF91CF9199
:109300001F910F9108958F929F92AF92BF92CF922B
:10931000DF92EF92FF920F931F93CF93DF93CDB71E
:10932000DEB729970FB6F894DEBF0FBECDBF809190
:10933000FA059091FB05009709F400C266EE74E00F
:109340000E94B63E9093860A8093850A009709F49E
:10935000A5C00E944B42082F10E00115110509F429
:109360009DC0000F111F000F111F8091800A909166
:10937000810A892B09F083C0C8010E944869909333
:10938000810A8093800A1092A30A1092A20A109276
:10939000880A1092870A1092A10A1092A50A1092C8
:1093A000A40A7801013082E018071CF0E12C22E0C9
:1093B000F22EC70101960E9448699093A70A8093F4
:1093C000A60A9093A00A80939F0A8E0D9F1D9093EA
:1093D0009A0A8093990A0E947E5F60939B0A709319
:1093E0009C0A80939D0A90939E0A80E090E0E09111
:1093F000A60AF091A70AE80FF91F10820196E81655
:10940000F906ACF782E090E09093A30A8093A20A59
:1094100080E98093C9001092C8001092CD0083E0CB
:109420008093CC008EE08093CA00F0920702E09215
:1094300006022091A60A3091A70A80910602909117
:109440000702820F931F90939A0A8093990A232B05
:1094500009F40BC166E57FE087EA97E00E942E5889
:10946000B80187EA97E00E948F3E87EA97E00E9462
:10947000F85880E297E29093980A8093970A65EBF8
:109480007FE087EA97E00E942E58B80187EA97E0CC
:109490000E948F3E87EA97E00E94F8586CEE74E0D5
:1094A0008091FA059091FB050E94B63E8C010097D1
:1094B00091F10E944B42882371F161E0C8010E9442
:1094C000A93EFC010185128590918F0A992359F0DC
:1094D000809170008E7F8093700010928F0A10929E
:1094E00002021092010283E08093000291110E9417
:1094F0008754C8010E94AF5469E97FE087EA97E08A
:109500000E942E58B80187EA97E00E948F3E87EAB2
:1095100097E00E94F858E090FA05F090FB0560EFA4
:1095200074E0C7010E94B63E90938A0A8093890A2C
:1095300067EF74E0C7010E94B63E8C019093EF057F
:109540008093EE056DEF74E0C7010E94B63E9093E4
:109550008E0A80938D0A109294051092930501153E
:10956000110511F1F801E680F78099E6C92E92E025
:10957000D92E0091EE051091EF050115110569F046
:10958000E114F10451F0F70180858530B1F7C7018E
:109590000E944B42823088F36FC0F8018681978128
:1095A00090939405809393050091FA051091FB0523
:1095B00069EE74E0C8010E94B63E9093FD05809369
:1095C000FC0564E075E0C8010E94B63E9093840AF1
:1095D0008093830A63E87FE087EA97E00E942E5831
:1095E0006BE77FE087EA97E00E942E5881E02091A8
:1095F000EE053091EF05232B09F480E00E94892EBF
:1096000062E77FE087EA97E00E942E5881E0209190
:10961000FC053091FD05232B09F480E00E94892E82
:1096200069E67FE087EA97E00E942E5881E020916A
:10963000890A30918A0A232B09F480E00E94892E3E
:1096400062E67FE087EA97E00E942E5881E0209151
:10965000830A3091840A232B09F480E00E94892E2A
:1096600087EA97E00E94F85869C06FE37FE087EAD5
:1096700097E00E94973EFDCEDA82C982FC82EB829F
:10968000CE0101960E947D28CE0101960E94AE2750
:10969000882309F44FC060E070E0CE0101960E947B
:1096A00017288C0160E0CE0101960E946A28A82E3E
:1096B000B12C8985853019F0863049F03BC0A11462
:1096C000B10429F462E0CE0101960E944528C80148
:1096D00017FF03C0919581959109982E092F882E27
:1096E00061E00E94085F11E0AA94AB2809F010E045
:1096F000612F882D0E94B03C64E97FE087EA97E003
:109700000E942E58692D702F87EA97E00E948F3EA5
:1097100062E97FE087EA97E00E942E58612F70E0AF
:1097200087EA97E00E948F3E60E97FE087EA97E052
:109730000E942E58F701E280F3801BCF29960FB6C6
:10974000F894DEBF0FBECDBFDF91CF911F910F9177
:10975000FF90EF90DF90CF90BF90AF909F908F9051
:109760000895CF93DF93CDB7DEB72C970FB6F8945B
:10977000DEBF0FBECDBF69EF7FE087EA97E00E94B2
:109780002E5886E490E00E9491738B37A1F51C82DD
:109790001B821E821D828FEF9FEF98878F838AE541
:1097A00093E09A83898386E490E09A8789871C8670
:1097B0001B868091FA059091FB050E94E721CE015E
:1097C00001960E9412229093FB058093FA05892B43
:1097D00019F468ED7FE011C06FEC7FE087EA97E055
:1097E0000E942E580E9483498DE09AE00E945244C4
:1097F00081E090E008C066EE7FE087EA97E00E9493
:109800002E5880E090E02C960FB6F894DEBF0FBE85
:10981000CDBFDF91CF9108950C94B14BCF92DF92E1
:10982000EF92FF92CF93DF93EC010E947E5F6B017A
:109830007C018091560890915708DC01ED91FC91D4
:109840000084F185E02D1995892B79F40E947E5FC3
:10985000DC01CB018C199D09AE09BF0988399A43F7
:10986000A105B10530F380E00DC0809156089091BC
:109870005708DC01ED91FC910284F385E02D1995E8
:10988000888381E0DF91CF91FF90EF90DF90CF90C0
:1098900008954F925F926F927F928F929F92AF92B4
:1098A000BF92CF92DF92EF92FF920F931F93CF93CD
:1098B000DF931F921F92CDB7DEB75C0188E598E079
:1098C0000E940E4C81113AC036C08C01CE01019627
:1098D0000E940E4C882379F1C80101962981F70175
:1098E00021937F01422F4F7750E0449DB001459D69
:1098F000700D549D700D1124C60ED71E47E0440C08
:10990000551C661C771C4A95D1F727FF27C0853068
:109910009105D9F68FEF9FEF9093F2088093F108AD
:109920008091560890915708DC01ED91FC910488D4
:10993000F589E02D199580E090E08EC09090580850
:10994000198289E5E82E88E0F82E01E010E0C12CAC
:10995000D12C412C512C32014394B8CFF92DF07FFA
:10996000FA832FEF280FD5012C93F03319F5885A7D
:10997000974F0E940E4C8823F1F2C801865A974FE8
:109980000E940E4C8823B9F2C8010396D501EC91D0
:10999000F0E0EE5AF74FE780F12CFE2CEE24208504
:1099A000E20EF11C2091580821FF08C0B2E0EB0E36
:1099B000F11C04C020E0E12CF12C01C022E0422E79
:1099C000512CFC01EE5AF74F4F018C01481A590AED
:1099D0002EEF622E77247A94C801840D951D8C1584
:1099E0009D0578F5CE0101960E940E4C882309F45E
:1099F000A2CF8091EF089091F0080097B1F0FA8122
:109A0000F03399F4D5012C91F301E21BF1099F0188
:109A1000200F311FE216F30640F4DC01ED91FC91BA
:109A20000190F081E02D698119950038110518F435
:109A30008981F40186830F5F1F4FFFEF8F1A9F0A02
:109A4000CBCF8091EF089091F008892B21F4013859
:109A5000110508F070CFC8010F900F90DF91CF91E2
:109A60001F910F91FF90EF90DF90CF90BF90AF903C
:109A70009F908F907F906F905F904F9008952F925E
:109A80003F924F925F926F927F928F929F92AF928E
:109A9000BF92CF92DF92EF92FF920F931F93CF93DB
:109AA000DF931F92CDB7DEB70E94AE1F382E8823FA
:109AB00009F422C10E947E5F2B013C018091DE08E7
:109AC0009091DF08A091E008B091E108A301920114
:109AD000281B390B4A0B5B0BDA01C90189399A4300
:109AE000A105B105A8F48091DA089091DB08A09156
:109AF000DC08B091DD08A3019201281B390B4A0B49
:109B00005B0BDA01C90189399A43A105B105C8F196
:109B10002091E2088091560890915708222371F015
:109B20002CEF3FEF3093F2082093F108DC01ED9128
:109B3000FC910488F589E02D1995DDC020EC209377
:109B4000580810925908DC01ED91FC910280F381D4
:109B5000E02D42E050E068E578E019954092DA089F
:109B60005092DB086092DC087092DD084092DE08BB
:109B70005092DF086092E0087092E10881E08093E3
:109B8000E2088091560890915708DC01ED91FC9114
:109B90000084F185E02D1995892B09F4ADC0CE0123
:109BA00001960E94494C5C01892B09F4A0C04092A7
:109BB000DE085092DF086092E0087092E108809120
:109BC0005808807F803309F076C08091E308909137
:109BD000E408892B09F490C0E980F12CF701EE5AD2
:109BE000F74F078110E0102F00278085080F111D07
:109BF0009701265A374F4901B701655A774FA80197
:109C0000C9010E942C78B8016E0D7F1DDB01AE5A90
:109C1000B74F18961C921897809158088670282E76
:109C2000E091E308F091E40832E0831337C019961D
:109C3000CC901997D12CDC2CCC241A968C91C80E80
:109C4000D11C4BEF5FEF4E195F09401B510B4A0DC2
:109C50005B1D635A774FC401199580E480935808BF
:109C600020925908D0925A08C0925B0880915608F9
:109C700090915708DC01ED91FC910280F381E02D79
:109C800044E050E068E578E019954092DA08509297
:109C9000DB086092DC087092DD082EC04DEF5FEFAC
:109CA0004E195F09401B510B4A0D5B1D655A774FDA
:109CB000C401199521C0803CA9F480ED8093580817
:109CC000109259088091560890915708DC01ED9147
:109CD000FC910280F381E02D42E050E068E578E0FD
:109CE00019950AC0803D41F41092E20805C00E9417
:109CF000AE1F811101C0312C832D0F90DF91CF91C8
:109D00001F910F91FF90EF90DF90CF90BF90AF9099
:109D10009F908F907F906F905F904F903F902F908B
:109D20000895AF92BF92CF92DF92EF92FF921F936E
:109D3000CF93DF9300D000D0CDB7DEB76C017C01AC
:109D400010E08AE0A82EB12C1330A9F0F70182812F
:109D500090E0A0E0B0E089839A83AB83BC83BE82AD
:109D6000AD82BE016F5F7F4F87EA97E00E94D728E0
:109D700063E770E114C0F601858190E0A0E0B0E0F7
:109D800089839A83AB83BC83BE82AD82BE016F5F41
:109D90007F4F87EA97E00E94D72860E770E10E9432
:109DA0002E581F5FFFEFEF1AFF0A143069F6269650
:109DB0000FB6F894DEBF0FBECDBFDF91CF911F91DC
:109DC000FF90EF90DF90CF90BF90AF9008950F93EA
:109DD0001F93CF93DF931F921F92CDB7DEB78C01F5
:109DE0008FE093E0F80191838083128213821482C2
:109DF0001582CE0101960E94432289819A810E9498
:109E0000A652B8016E5F7F4F44E050E08FE090E0D3
:109E10000E9424360E94A552C8010F900F90DF9136
:109E2000CF911F910F910895CF93DF93C2E5D8E0B2
:109E300080EE8E831F828C819D81DC01ED91FC91EF
:109E40000280F381E02D42E050E068E578E019956A
:109E50008FEF9FEF9093F2088093F1088C819D81A2
:109E6000DC01ED91FC910680F781E02D19958C8144
:109E70009D81DC01ED91FC910488F589E02D199517
:109E80000E947E5F6093DA087093DB088093DC08A1
:109E90009093DD086093DE087093DF088093E008FC
:109EA0009093E108DF91CF910895AF92BF92CF9246
:109EB000DF92EF92FF920F931F93CF93DF931F9246
:109EC0001F92CDB7DEB77A836983BA01A901E98110
:109ED000FA81F770082F10E0000F111F0C511A4F74
:109EE000D8018D919C918E0F9F1F9F01240F351FCC
:109EF00021303840A0F07A015B0160E078E06B012E
:109F0000CE1ADF0AA601B5010E942436A7014C191A
:109F10005D09B5016C0D7D1DF801808191810F9067
:109F20000F90DF91CF911F910F91FF90EF90DF90F5
:109F3000CF90BF90AF900C9424369F92AF92BF9277
:109F4000CF92DF92EF92FF920F931F93CF93DF9305
:109F5000982E8B015A01690164E270E00E94A144CD
:109F6000E82EF12C65E270E0892D0E94A144FE2CC0
:109F7000EE24E82AE801CE0DDF1D9E013770E92CA2
:109F8000F12CC701880F991FAC0144525A4F7A0136
:109F9000FA0180819181820F931FA9014C0D5D1DF3
:109FA0004130584090F000E018E0021B130BA8016C
:109FB000B5010E945436A601401B510BB501600F3C
:109FC000711FF7018081918102C0A601B5010E9435
:109FD0005436CC0DDD1D4D2F64E270E0892D0E94BA
:109FE000CB434C2F65E270E0892DDF91CF911F911B
:109FF0000F91FF90EF90DF90CF90BF90AF909F9028
:10A000000C94CB43FF920F931F93CF93DF93F82EC3
:10A0100000E010E08F2D0E94B636EC01892B21F074
:10A020008F2D0E94B6368C01C017D10799F7CE014B
:10A03000DF91CF911F910F91FF90089520E3FC01D4
:10A0400020833296862F82958F7090E1899F6019C8
:10A0500011246A3014F4605D01C0695C6293682F5A
:10A060008111F0CF08952F923F924F925F926F929D
:10A070007F928F929F92AF92BF92CF92DF92EF9298
:10A08000FF920F931F93CF93DF93CDB7DEB7E29785
:10A090000FB6F894DEBF0FBECDBF7C012A013B0195
:10A0A00069010E947E5F4B015C0187010D5B1F4FC0
:10A0B000C8010E94D74518161906A4F00E947E5FB9
:10A0C000DC01CB0188199909AA09BB094816590670
:10A0D0006A067B06D8F062E370E080E090E00E94C0
:10A0E000445FE6CF42E250E0BE016F5F7F4FC801A0
:10A0F0000E948F458981823011F080E060C1F801B3
:10A100008489958983349105C1F702C08FEF57C1C7
:10A110006D817E818F8198850E9422744B015C0144
:10A12000F601608371838283938346E050E0B70138
:10A13000685F7F4FCE014D960E941F78892BE9F60C
:10A14000F70180819181A281B38188169906AA06C0
:10A15000BB0698F284819581A681B78188159905FF
:10A16000AA05BB0550F289899A89AB89BC89868783
:10A170009787A08BB18B8EECC82ED12CC8010E9482
:10A18000AE45F1E0CF1AD108C9F7712CC70182960C
:10A190009AA789A7F701B696FCA7EBA708969EA7F2
:10A1A0008DA73C974F01899698AB8FA73897FAAB4C
:10A1B000E9AB1701F6E12F0E311C27018EE1480EA5
:10A1C000511CF801818D928D181619060CF0F6C0FD
:10A1D000C8010E94AE458333910509F4C9C0F4F467
:10A1E00081309105B9F11CF4892B59F3DBC0833020
:10A1F0009105C1F1069709F0D5C0C8010E94AE458E
:10A200006C0144E050E0B201C8010E948F45A12CCE
:10A21000B12CDD2494E0C91AD1083FC08A339105DE
:10A2200009F47AC03CF48533910561F0C69709F4CE
:10A230003FC0B8C08B33910509F484C08F3F9105AE
:10A2400001F2B0C0C8010E94AE45C8010E94AE45EF
:10A25000782EB7CFC8010E94AE4544E050E069A90E
:10A260007AA93AC0C8010E94AE456C0144E050E0B2
:10A27000B101C8010E948F45A12CB12CDD24F4E06E
:10A28000CF1AD108AC14BD040CF09BCFC8010E94BA
:10A29000AE458FEFA81AB80AF5CFAC14BD040CF088
:10A2A00090CFC8010E94AE45EFEFAE1ABE0AF5CFBF
:10A2B000C8010E94AE45682EF701828D811110C041
:10A2C000838D81110DC0848D81110AC0858D81110E
:10A2D00007C044E050E0B401C8010E948F4571CF2F
:10A2E000EFA5F8A9A080B180C280D380B401CE01CF
:10A2F00083960E94FE588DA19EA1AFA1B8A5A81675
:10A30000B906CA06DB0629F3662009F45ACFC8014C
:10A310000E94AE456A94F8CFC8010E94AE4544E061
:10A3200050E06BA57CA5C8010E948F45F70166A18E
:10A3300077A180A591A50E94227466A377A380A728
:10A3400091A73FCFC8010E94AE4544E050E06DA503
:10A350007EA5C8010E948F45F70162A573A584A55B
:10A3600095A50E94227462A773A784A795A729CFF9
:10A37000C8010E94AE4544E050E069A57AA5C80135
:10A380000E948F45F70162A173A184A195A10E944B
:10A39000227462A373A384A395A366A777A780AB57
:10A3A00091AB0FCFC8010E94AE45D82EDD2009F435
:10A3B00008CFC8010E94AE45DA94F8CF872DE29607
:10A3C0000FB6F894DEBF0FBECDBFDF91CF911F91C6
:10A3D0000F91FF90EF90DF90CF90BF90AF909F9044
:10A3E0008F907F906F905F904F903F902F90089547
:10A3F000CF93DF931F92CDB7DEB76983DC01ED9178
:10A40000FC910280F381E02D41E050E0BE016F5FDE
:10A410007F4F19950F90DF91CF910895DC01ED9159
:10A42000FC91068CF78DE02D199591E08927089510
:10A43000862F089581E086270895CF93DF931F929A
:10A44000CDB7DEB789832091900A3981E091910AD6
:10A45000F091920A822F90E080959095F894008078
:10A46000082200824BE000C05DE000005A95E9F749
:10A47000008008220894379508F4022A00824A9541
:10A4800099F778940F90DF91CF9108950F931F93D0
:10A49000CF93DF931F92CDB7DEB78C01DC01ED9136
:10A4A000FC910084F185E02D1995892B51F0BE01B6
:10A4B0006F5F7F4FF80184850E94BF44898190E0DF
:10A4C00002C08FEF9FEF0F90DF91CF911F910F91FF
:10A4D0000895FC0184850C941045CF93DF931F925F
:10A4E000CDB7DEB741E050E0BE016F5F7F4FFC01AA
:10A4F00084850E941045181619061CF4898190E085
:10A5000002C08FEF9FEF0F90DF91CF910895FC0174
:10A510008485843011F00C94164380E090E0089517
:10A5200044E050E0BC018FE090E00C94543644E0ED
:10A5300050E0BC0185E090E00C94543644E050E0DB
:10A54000BC0181E090E00C94543608958CBD9DBD13
:10A5500008956F927F928F929F92AF92BF92CF9207
:10A56000DF92EF92FF921F93CF93DF931F921F9280
:10A57000CDB7DEB75C013B016A01FC0114851430E4
:10A5800041F481E090E0F5019383828380E090E0E4
:10A590005BC07A014130584018F0E12C88E0F82E79
:10A5A000CE0101960E94432289819A810E94A6527F
:10A5B000812F0E9402504C0163E070E0812F0E94C5
:10A5C000A144873111F08C3121F48E149F0440F3A3
:10A5D00002C0E12CF12CCE0101960E944322898118
:10A5E0009A810E94A6529701A30160E070E0812F3A
:10A5F0000E949D4F60E270E0812F0E94332262E052
:10A6000070E0812F0E94A14484FD14C063E070E0DB
:10A61000812F0E94A144811104C0812F0E94D54343
:10A62000B0CFCE0101960E94432289819A810E9477
:10A63000A652E5CF40E162E070E0812F0E94CB435B
:10A64000EF2809F49ECFC6010F900F90DF91CF91B4
:10A650001F91FF90EF90DF90CF90BF90AF909F90B1
:10A660008F907F906F9008958F929F92AF92BF923C
:10A67000DF92EF92FF920F931F93CF93DF931F927E
:10A680001F92CDB7DEB7FC012485243009F083C0CA
:10A690005A018B017C01D12C8D2D0E9431468111F4
:10A6A00003C0F701D48607C08B7F8831D1F3D394E0
:10A6B000F4E0DF12F1CFF7018485843009F46BC038
:10A6C00020910302309104022F5F3F4F11F420E0EC
:10A6D00030EC309304022093030240910302509126
:10A6E000040220E061E00E94F843F80182818F3F7C
:10A6F00051F483818F3F99F484818F3F81F4858168
:10A700008F3F69F445C081110AC0F801838181112E
:10A7100006C08481811103C085818823C9F1A114F9
:10A72000B104B1F1F701D484CE0101960E94432215
:10A7300089819A810E94A652B8016E5F7F4F8D2D4C
:10A740000E94D846B5018D2D0E94C74664E070E096
:10A750008D2D0E9433220E947E5F4B015C01F4E943
:10A760008F0EF1E19F1EA11CB11CC7010E9448225F
:10A77000873149F161E070E080E090E00E94445F41
:10A78000A8950E94B62AC7010E944822811106C0DE
:10A7900084E0F701848780E090E01DC00E947E5F26
:10A7A00086169706A806B90600F7F70184850E9469
:10A7B000D54384E0F701848760E970E187EA97E098
:10A7C0000E94973EE8CF65E870E187EA97E00E9433
:10A7D000973E81E090E00F900F90DF91CF911F9115
:10A7E0000F91FF90EF90DF90BF90AF909F908F9070
:10A7F000089578941F920F920FB60F9211240BB602
:10A800000F92CF92DF92EF92FF920F931F932F93AD
:10A810003F934F935F936F937F938F939F93AF93E8
:10A82000BF93CF93DF93EF93FF93809170008E7F60
:10A83000809370000FE310E08BE1E82EF12C9BE297
:10A84000C92ED12CC091930AD091940A2097F9F483
:10A850000332110508F43BC003521109E091910A3B
:10A86000F091920A90812091900A822F80959823EE
:10A8700090839BE0D7011197F1F79150D9F7808130
:10A88000822B8083C6010197F1F780E00DC00B3069
:10A890001105E8F00B501109E091950AF091960A24
:10A8A000EC0FFD1F319780810E941D522196D0939D
:10A8B000940AC093930A80910102909102028C172E
:10A8C0009D0708F0BFCF1092940A1092930A8091CE
:10A8D0007000816080937000FF91EF91DF91CF91C4
:10A8E000BF91AF919F918F917F916F915F914F91A8
:10A8F0003F912F911F910F91FF90EF90DF90CF909C
:10A900000F900BBE0F900FBE0F901F90189581E017
:10A9100080938F0A80910002282F30E0F901E05CDB
:10A92000F24FE491F0E0EE0FFF1FE058F34F459136
:10A9300054915093920A4093910AF901E650F34FD3
:10A94000E491E093900A61E00E94085F83E08093C5
:10A95000B100E0E7F0E08081816080830895CF93CB
:10A96000DF931816190644F0809170008E7F809353
:10A97000700010928F0A19C0EC018091950A909195
:10A98000960A0E94E069CE01C130D24014F080E006
:10A9900092E090930202809301020E944869909392
:10A9A000960A8093950A892B29F41092020210923C
:10A9B000010208C080918F0A811104C0DF91CF91FC
:10A9C0000C948754DF91CF910895FF920F931F93BA
:10A9D000CF93DF938C01F62E80918F0A811102C0F4
:10A9E0000E948754E8012197C11582E0D80798F4A6
:10A9F00080910102909102028017910718F4C8011A
:10AA00000E94AF548091950A9091960A009719F090
:10AA1000C80FD91FF882DF91CF911F910F91FF903E
:10AA200008958F929F92AF92BF92CF92DF92EF9252
:10AA3000FF920F931F93CF93DF93CDB7DEB72B9782
:10AA40000FB6F894DEBF0FBECDBF8C01CE010196CC
:10AA50007C016C018AE0882E912CA12CB12CC601BE
:10AA60008E199F09411551056105710581F0CB01D2
:10AA7000BA01A50194010E94B773942F852F605DE0
:10AA8000F60161936F01A901692F782FE8CFFC01CE
:10AA90003197EE0DFF1DD8019E01215031094081F3
:10AAA0004D933197E217F307D1F7F801E80FF91F3B
:10AAB00010822B960FB6F894DEBF0FBECDBFDF918C
:10AAC000CF911F910F91FF90EF90DF90CF90BF90AB
:10AAD000AF909F908F9008958F929F92AF92BF9268
:10AAE000CF92DF92EF92FF920F931F93CF93DF935A
:10AAF0008C014A016901E0908D0AF0908E0AC62F00
:10AB0000660FDD0BE114F10449F1F7018085863011
:10AB100029F569E075E0C7010E94B63E5C01F2E0EC
:10AB20008F16910439F083E08816910451F46EE099
:10AB300075E002C062E175E0C7010E94B63E7C018B
:10AB400002C0E12CF12CA114B10451F0F501618592
:10AB50007285AE01C8010E94957808C0E12CF12CE5
:10AB6000AE016EE770E1C8010E94586CAE0160EB67
:10AB700073E0C8010E947778E114F10421F0F70135
:10AB8000618572850FC0F2E08F169104A1F083E019
:10AB90008816910461F08A94892899F460918B0A4F
:10ABA00070918C0AAE01C8010E9477780AC0AE018C
:10ABB00068E770E103C0AE0165E770E1C8010E947B
:10ABC000486CAE0160EB73E0C8010E947778C11455
:10ABD000D10429F0AE01B601C8010E947778C801FE
:10ABE000DF91CF911F910F91FF90EF90DF90CF9069
:10ABF000BF90AF909F908F900895AF92BF92CF92E9
:10AC0000DF92EF92FF920F931F93CF93DF93CDB715
:10AC1000DEB7AF970FB6F894DEBF0FBECDBF7C0195
:10AC20005B016A010FE013E01A8309831B821C8217
:10AC30001D821E82CE0109960E9446431BA70AA7C9
:10AC40001CA61DA61EA61FA680914C0890914D081B
:10AC5000A0914E08B0914F088EA39FA3A8A7B9A7B3
:10AC60008B839C83AD83BE8318861F82AE01465DB5
:10AC70005F4FB501CE0101960E942E3A81309105B9
:10AC8000B1F4D701ED91FC910684F785E02D1DA369
:10AC90000CA38CA59DA5AEA5BFA58EA39FA3A8A719
:10ACA000B9A7A601BE016C5D7F4FC7011995AF968C
:10ACB0000FB6F894DEBF0FBECDBFDF91CF911F91CD
:10ACC0000F91FF90EF90DF90CF90BF90AF900895DD
:10ACD000CF92DF92EF92FF920F931F93CF93DF9368
:10ACE0006C017A018B01C0E0D0E0CE15DF0581F068
:10ACF000D8016D918D01D601ED91FC910190F0810B
:10AD0000E02DC6011995892B11F02196EECF7E0119
:10AD1000C701DF91CF911F910F91FF90EF90DF90CE
:10AD2000CF900895FC01538D448D252F30E0842F62
:10AD300090E0821B930B541710F0CF960895019763
:10AD40000895FC01918D828D981761F0828DDF014D
:10AD5000A80FB11D5D968C91928D9F5F9F73928F0E
:10AD600090E008958FEF9FEF0895FC01918D828D03
:10AD7000981731F0828DE80FF11D858D90E00895D0
:10AD80008FEF9FEF0895FC01918D228D892F90E028
:10AD9000805C9F4F821B91098F73992708958AE0E9
:10ADA00097E00E94C35621E0892B09F420E0822F0E
:10ADB000089587EA97E00E94C35621E0892B09F4A1
:10ADC00020E0822F0895FC01848DDF01A80FB11DC2
:10ADD000A35ABF4F2C91848D90E001968F739927D1
:10ADE000848FA689B7892C93A089B1898C918370AF
:10ADF00080648C93938D848D981306C00288F389A8
:10AE0000E02D80818F7D80830895EF92FF920F93D4
:10AE10001F93CF93DF93EC0181E0888F9B8D8C8D06
:10AE2000981305C0E889F989808185FD26C0F62E32
:10AE30000B8D10E00F5F1F4F0F731127E02E8C8DCD
:10AE4000E8120CC00FB607FCFACFE889F9898081B7
:10AE500085FFF5CFCE010E94E356F1CF8B8DFE0129
:10AE6000E80FF11DE35AFF4FF0829FB7F8940B8F64
:10AE7000EA89FB89808180620AC09FB7F894EE89D5
:10AE8000FF896083E889F989808183708064808389
:10AE90009FBF81E090E0DF91CF911F910F91FF90D4
:10AEA000EF900895CF93DF93EC01888D8823C9F04C
:10AEB000EA89FB89808185FD05C0A889B9898C91C3
:10AEC00086FD0FC00FB607FCF5CF808185FFF2CF5E
:10AED000A889B9898C9185FFEDCFCE010E94E356F8
:10AEE000E7CFDF91CF91089580E090E0892B21F0AA
:10AEF0000E94D956811121C080E090E0892B41F059
:10AF000080E090E0892B21F00E940000811118C0A0
:10AF100080E090E0892B21F00E94CF56811113C070
:10AF200080E090E0892BA1F080E090E0892B81F017
:10AF30000E94000081110AC008950E940000DCCF29
:10AF40000E940000E5CF0E940000EACF0C940000B0
:10AF500008950E940078EF92FF920F931F93CF9372
:10AF6000DF93EC018B017A010E947E5FFE01E857BE
:10AF7000FF4F60837183828393838C819D81DC0189
:10AF8000ED91FC910280F381E02DA701B801DF91E2
:10AF9000CF911F910F91FF90EF9019941F93CF9332
:10AFA000DF93EC01162F0E947E5FFE01E857FF4FF2
:10AFB00060837183828393838C819D81DC01ED9119
:10AFC000FC910190F081E02D612FDF91CF911F91D5
:10AFD0001994DC01ED91FC910190F081E02D199420
:10AFE0008F929F92AF92BF92CF92DF92EF92FF9299
:10AFF0000F931F93CF93DF937C018B014C0182E071
:10B00000880E911C5701E5E0AE0EB11CC0E0D0E007
:10B01000F40161914F01C8010E94D13E6C016EE2C2
:10B02000C8010E94E9578C0D9D1DC80FD91F8A14B5
:10B030009B0471F7F7016581C8010E94D13E8C0F16
:10B040009D1FDF91CF911F910F91FF90EF90DF90A7
:10B05000CF90BF90AF909F908F900895EF92FF9206
:10B060000F931F93CF93DF938C017B01C0E0D0E05F
:10B07000F701EC0FFD1F6491662361F0D801ED919B
:10B08000FC910190F081E02DC8011995892B11F0F8
:10B090002196EECFCE01DF91CF911F910F91FF90BE
:10B0A000EF9008956115710579F0FB010190002082
:10B0B000E9F73197AF01461B570BDC01ED91FC918D
:10B0C0000280F381E02D199480E090E008958F9242
:10B0D0009F92AF92BF92EF92FF920F931F93CF93E5
:10B0E000DF93CDB7DEB7A1970FB6F894DEBF0FBEE2
:10B0F000CDBF7C01FA01CB0119A2223008F42AE06D
:10B100008E010F5D1F4F822E912CA12CB12CBF01FF
:10B11000A50194010E94B773F901CA0101501109F8
:10B120006A3014F4605D01C0695CD8016C93232B14
:10B13000242B252B61F7B801C7010E945258A19614
:10B140000FB6F894DEBF0FBECDBFDF91CF911F9138
:10B150000F91FF90EF90BF90AF909F908F900895C8
:10B16000CF92DF92EF92FF920F931F93CF93DF93D3
:10B170002115310581F4DC01ED91FC910190F08104
:10B18000E02D642FDF91CF911F910F91FF90EF90F1
:10B19000DF90CF9019942A30310501F577FF1DC05B
:10B1A0006A017B01EC016DE20E94E9578C014427A2
:10B1B0005527BA014C195D096E097F092AE0CE01B5
:10B1C0000E946758800F911FDF91CF911F910F91BF
:10B1D000FF90EF90DF90CF9008952AE0DF91CF911C
:10B1E0001F910F91FF90EF90DF90CF900C946758D4
:10B1F00068EF73E00C9452580C945258DC018FE0C5
:10B2000093E08D939D9384E0FB0101900D928A95CC
:10B21000E1F708951F920F920FB60F9211240BB60B
:10B220000F922F933F934F935F936F937F938F93DF
:10B230009F93AF93BF93EF93FF938AE097E00E94B1
:10B24000E356FF91EF91BF91AF919F918F917F91C5
:10B250006F915F914F913F912F910F900BBE0F9087
:10B260000FBE0F901F9018951F920F920FB60F925E
:10B2700011240BB60F922F938F939F93EF93FF930D
:10B28000E0911A07F0911B078081E0912007F0916F
:10B29000210782FD12C09081809123078F5F8F73F9
:10B2A00020912407821751F0E0912307F0E0E65F38
:10B2B000F84F958F8093230701C08081FF91EF9114
:10B2C0009F918F912F910F900BBE0F900FBE0F90FB
:10B2D0001F9018951F920F920FB60F9211240BB664
:10B2E0000F922F933F934F935F936F937F938F931F
:10B2F0009F93AF93BF93EF93FF9387EA97E00E94EA
:10B30000E356FF91EF91BF91AF919F918F917F9104
:10B310006F915F914F913F912F910F900BBE0F90C6
:10B320000FBE0F901F9018951F920F920FB60F929D
:10B3300011240BB60F922F938F939F93EF93FF934C
:10B34000E091B707F091B8078081E091BD07F091D7
:10B35000BE0782FD12C090818091C0078F5F8F73FE
:10B360002091C107821751F0E091C007F0E0E95544
:10B37000F84F958F8093C00701C08081FF91EF91B6
:10B380009F918F912F910F900BBE0F900FBE0F903A
:10B390001F9018951F920F920FB60F9211240BB6A3
:10B3A0000F922F933F934F935F938F939F93EF93BE
:10B3B000FF932091A60A3091A70A8091A40A909148
:10B3C000A50AAC014F5F5F4F5093A50A4093A40AB2
:10B3D000F901E80FF91F80818093CE008091060269
:10B3E000909107022091A40A3091A50A8217930731
:10B3F00048F48FEF9FEF9093A50A8093A40A88E406
:10B400008093C900FF91EF919F918F915F914F9130
:10B410003F912F910F900BBE0F900FBE0F901F907A
:10B4200018951F920F920FB60F9211242F933F93EE
:10B430008F939F932091A20A3091A30A8091A40A2E
:10B440009091A50A21303105A9F48F3F2FEF920783
:10B4500089F41092C8001092CD0089E08093CC004E
:10B4600086E28093CA001092CE001092A50A109234
:10B47000A40A17C0892BA9F41092C8001092CD001D
:10B4800083E08093CC008EE08093CA0088E28093B2
:10B49000C9001092CE0081E090E09093A50A8093BD
:10B4A000A40A9F918F913F912F910F900FBE0F9003
:10B4B0001F9018951F920F920FB60F9211240BB682
:10B4C0000F922F933F934F935F936F937F938F933D
:10B4D0009F93AF93BF93EF93FF939091C800809198
:10B4E000CE0094FF08C081E08093A10A8091A60A53
:10B4F0009091A70A57C09091A10A913099F48111B7
:10B500000EC082E08093A10A0E947E5F60939B0A36
:10B5100070939C0A80939D0A90939E0A3EC010925D
:10B52000A10A44C0923009F041C0E0919F0AF09115
:10B53000A00A9081891721F091E090930502808301
:10B5400020919F0A3091A00A8091990A90919A0ABD
:10B550002817390711F51092A10A80910502882356
:10B56000D1F08091970A9091980A892BA1F01092BE
:10B57000C900E091970AF091980A199580E98093A3
:10B58000C9001092C8001092CD0083E08093CC00D7
:10B590008EE08093CA001092050280919F0A9091DC
:10B5A000A00A01969093A00A80939F0AFF91EF91C1
:10B5B000BF91AF919F918F917F916F915F914F91CB
:10B5C0003F912F910F900BBE0F900FBE0F901F90C9
:10B5D0001895CF92DF92EF92FF920F931F93CF9324
:10B5E000DF936C018B0186E090E00E944869EC01DA
:10B5F0009093A90A8093A80AF60101900020E9F728
:10B60000CF018C199D090E9448697C01B6010E94F6
:10B610007078F60101900020E9F73197EC19FD09E7
:10B62000EE0DFF1D1082F982E8821B830A83809150
:10B630009105909192059D838C83D0939205C09340
:10B640009105DF91CF911F910F91FF90EF90DF90C7
:10B65000CF900895CF92DF92EF92FF920F931F93B6
:10B66000CF93DF93CDB7DEB7EC970FB6F894DEBF7C
:10B670000FBECDBFDC012C91222309F451C061E340
:10B6800074E00E94676C9A8389837E01B3E0EB0EBD
:10B69000F11C01E010E0D02EC12E61E374E080E0E7
:10B6A00090E00E94676CF701819391937F010E31C6
:10B6B000110539F40091A80A1091A90AE980FA80CD
:10B6C00008C00F5F1F4F892B31F7F4CFF8010481B9
:10B6D000158101151105A1F0D8016D917C91C7016B
:10B6E0000E946778892B91F7D8011296ED91FC9111
:10B6F0001397BE016F5F7F4F8D2D9C2D199506C04E
:10B7000062EA70E187EA97E00E94973E87EA97E055
:10B710000E94F8586EE970E187EA97E00E942E587F
:10B72000EC960FB6F894DEBF0FBECDBFDF91CF9180
:10B730001F910F91FF90EF90DF90CF900895FB0144
:10B7400024813581428153812417350758F4408183
:10B750005181DA01A20FB31F8C93848195810196E8
:10B760009583848380E00895FC0184819581089508
:10B77000089580E090E008958F929F92AF92BF92DB
:10B78000CF92DF92EF92FF920F931F93CF93DF93AD
:10B79000CDB7DEB7C154D1090FB6F894DEBF0FBEE6
:10B7A000CDBF5C016B018A0161E071E187EA97E03E
:10B7B0000E942E58B50187EA97E00E94FC586EEF70
:10B7C00070E187EA97E00E942E58C114D10409F471
:10B7D000A4C00C0D1D1DF80110829E012F5F3F4F6C
:10B7E00079018091B50A9091B60A009711F481EC25
:10B7F0009AE0F701E81BF90BEA3FF1051CF469EF49
:10B8000070E149C046018016910641F0F401619152
:10B810004F0187EA97E00E94E957F5CF87EA97E062
:10B820000E94F858809195059091960520E030E0AF
:10B83000049719F443E050E019C042E050E061E49D
:10B84000C7010E946C55F70101900020E9F731977C
:10B850008F010E191F09A801B701C5010E94877841
:10B860000097A9F020E030E041E050E061E4C7013A
:10B870000E946C55F70101900020E9F731978F0184
:10B880000E191F09A801B701C5010E948778892BED
:10B8900039F06EEE70E187EA97E00E942E583DC0C5
:10B8A0000A0D1B1D67E175E0C8010E946778892BAE
:10B8B00021F4C6010E942A5B30C06FE270E0C8012B
:10B8C0000E945C785C01009741F0FC01108281814C
:10B8D000843219F1FFEFAF1ABF0AF8018081843278
:10B8E000E1F0B801C7010E94241EC7010E94AE27E3
:10B8F000882399F0298580919505909196052730A8
:10B9000019F48430910549F041E0049709F440E0CE
:10B910009501B601C7010E94C723CF5BDF4F0FB669
:10B92000F894DEBF0FBECDBFDF91CF911F910F9175
:10B93000FF90EF90DF90CF90BF90AF909F908F904F
:10B940000895CF92DF92EF92FF921F93CF93DF93F0
:10B9500000D000D0CDB7DEB766E071E187EA97E0AE
:10B960000E942E5882E0E82E87E0F82E10E090E149
:10B97000C92ED12C1530B9F0F701808190E0A0E0FC
:10B98000B0E089839A83AB83BC83DE82CD82BE0123
:10B990006F5F7F4F87EA97E00E94D72864E071E1EC
:10B9A0000E942E5814C08091070790E0A0E0B0E0FC
:10B9B00089839A83AB83BC83DE82CD82BE016F5FB5
:10B9C0007F4F87EA97E00E94D7280E94F8581F5FB0
:10B9D000FFEFEF1AFF0A163069F626960FB6F894B5
:10B9E000DEBF0FBECDBFDF91CF911F91FF90EF90D3
:10B9F000DF90CF9008955F926F927F928F929F9287
:10BA0000AF92BF92CF92DF92EF92FF920F931F936C
:10BA1000CF93DF93CDB7DEB7E4970FB6F894DEBFD0
:10BA20000FBECDBF6C017B013A01590161E00E945C
:10BA30006A28002361F0682F6062C6010E944528D1
:10BA40006DED70E187EA97E00E942E58B8C01AA207
:10BA500019A2FE01B3968EE0DF011D928A95E9F7E7
:10BA600020E030E043E050E060E2CE0101960E9429
:10BA70006C55D6011296ED91FC91139760817181FE
:10BA800040E250E0CE0101960E947778B2E0EB16DA
:10BA9000F104C9F03CF4E114F104E1F0EA94EF2878
:10BAA00079F05FC086E0E816F10451F09EE0E916F7
:10BAB000F10481F0A5E0EA16F10409F052C003C0D8
:10BAC0006EE674E002C061E774E0CE0181960E94E8
:10BAD000707850C0A114B10409F44CC08501C12C88
:10BAE000D12C80E2A82E85E0B82E94E0592E7E015C
:10BAF000B1E3EB0EF11C4301E1E08E1A9108C6148C
:10BB0000D704C4F5D8018C9111969C910E5F1F4FFC
:10BB10009F938F93BF92AF921F925F92FF92EF928B
:10BB20000E94A47840E150E0B701CE0181960E94C6
:10BB300077780FB6F894DEBF0FBECDBFC814D90416
:10BB400061F063E275E0C7010E94707840E150E067
:10BB5000B701CE0181960E947778FFEFCF1ADF0AF6
:10BB6000CECF6FEC70E187EA97E00E942E588FEFFE
:10BB70009FEF27C069EC70E187EA97E00E942E589A
:10BB8000BE016F5F7F4F87EA97E00E94FC5866EC2A
:10BB900070E187EA97E00E942E58BE016F5D7F4FEB
:10BBA00087EA97E00E94FC5887EA97E00E94F858DD
:10BBB000BE016F5D7F4FCE0101960E94372080E06D
:10BBC00090E0E4960FB6F894DEBF0FBECDBFDF91D4
:10BBD000CF911F910F91FF90EF90DF90CF90BF908A
:10BBE000AF909F908F907F906F905F900895FF929D
:10BBF0000F931F93CF93DF93CDB7DEB729970FB67F
:10BC0000F894DEBF0FBECDBF8C010E94AE27882303
:10BC100009F46BC060E0C8010E946A28D801189638
:10BC2000FC90B7E0FB1671F0823009F45CC020F4A0
:10BC3000813009F45DC006C0853009F454C08630F7
:10BC400009F456C0C8010E94F327362F272F4F2D25
:10BC500050E04A30510508F046C0FA018827EE51FD
:10BC6000FF4F8F4F0C941A74D8011496ED91FC91EC
:10BC7000159780858530B9F56AEB70E187EA97E022
:10BC80000E942E58D8011496ED91FC9115970681CB
:10BC900017810115110539F1F80161857285CE0111
:10BCA00001960E94241ECE0101960E94AE27882391
:10BCB00011F1CE0101960E94F75D892BE1F062EB54
:10BCC00070E187EA97E00E942E5812C0292F990F41
:10BCD000330B03C0832F922F9C0181E090E0232B34
:10BCE00081F480E00EC080E004C08FEF9FEF09C0B8
:10BCF00081E090E006C0D80112960D911C91139737
:10BD0000C8CF29960FB6F894DEBF0FBECDBFDF9126
:10BD1000CF911F910F91FF9008953FB7F8948091B4
:10BD2000AF0A9091B00AA091B10AB091B20A26B5BB
:10BD3000A89B05C02F3F19F00196A11DB11D3FBF63
:10BD4000BA2FA92F982F8827820F911DA11DB11DF1
:10BD5000BC01CD0142E0660F771F881F991F4A95ED
:10BD6000D1F7089590E0FC013197E231F10508F038
:10BD70004EC08827E451FF4F8F4F0C941A74809166
:10BD800080008F7703C0809180008F7D809380003A
:10BD9000089580918000877FF9CF84B58F7702C0A6
:10BDA00084B58F7D84BD08958091B0008F7703C0E6
:10BDB0008091B0008F7D8093B000089580919000B5
:10BDC0008F7707C0809190008F7D03C08091900095
:10BDD000877F8093900008958091A0008F7707C09F
:10BDE0008091A0008F7D03C08091A000877F809309
:10BDF000A0000895809120018F7707C080912001D5
:10BE00008F7D03C080912001877F8093200108955A
:10BE1000CF93DF9390E0FC01E650F34F2491FC01B7
:10BE2000E05CF24F8491882361F190E0880F991FC4
:10BE3000FC01E052F34FC591D491FC01E058F34F5F
:10BE4000A591B491611109C09FB7F894888120959C
:10BE500082238883EC912E230BC0623061F49FB75C
:10BE6000F8948881322F309583238883EC912E2B90
:10BE70002C939FBF06C08FB7F894E8812E2B2883A0
:10BE80008FBFDF91CF9108958F929F92AF92BF9213
:10BE9000CF92DF92EF92FF926B017C010E948D5E48
:10BEA0004B015C01C114D104E104F104F1F00E94E2
:10BEB0008D5EDC01CB0188199909AA09BB09883E6E
:10BEC0009340A105B10570F321E0C21AD108E10841
:10BED000F10888EE880E83E0981EA11CB11CC114E5
:10BEE000D104E104F10419F7DDCFFF90EF90DF906A
:10BEF000CF90BF90AF909F908F9008952FB7F894F8
:10BF00006091AB0A7091AC0A8091AD0A9091AE0A33
:10BF10002FBF08951F920F920FB60F9211242F93E7
:10BF20003F938F939F93AF93BF938091AB0A909170
:10BF3000AC0AA091AD0AB091AE0A3091AA0A23E0F2
:10BF4000230F2D3720F40196A11DB11D05C026E851
:10BF5000230F0296A11DB11D2093AA0A8093AB0A5C
:10BF60009093AC0AA093AD0AB093AE0A8091AF0A49
:10BF70009091B00AA091B10AB091B20A0196A11DA8
:10BF8000B11D8093AF0A9093B00AA093B10AB09309
:10BF9000B20ABF91AF919F918F913F912F910F90D6
:10BFA0000FBE0F901F901895CF93DF93CDB7DEB7DC
:10BFB000CE56D1090FB6F894DEBF0FBECDBF789430
:10BFC00084B5826084BD84B5816084BD85B582609E
:10BFD00085BD85B5816085BD80916E00816080934F
:10BFE0006E001092810080918100826080938100B8
:10BFF00080918100816080938100809180008160C8
:10C00000809380008091B10084608093B100809122
:10C01000B00081608093B000809191008260809335
:10C0200091008091910081608093910080919000B7
:10C030008160809390008091A10082608093A10034
:10C040008091A10081608093A1008091A000816017
:10C050008093A000809121018260809321018091D2
:10C060002101816080932101809120018160809372
:10C07000200180917A00846080937A0080917A0018
:10C08000826080937A0080917A00816080937A0048
:10C0900080917A00806880937A001092C10010929B
:10C0A000D305109292051092910526E040E052ECE3
:10C0B00061E070E087EA97E00E942F3F68E478E053
:10C0C00087EA97E00E942E586AE179E484EC93E0D5
:10C0D0000E94E95A6EE578E489EC93E00E94E95AFF
:10C0E0006CE07CE48EEC93E00E94E95A60ED70E332
:10C0F00083ED93E00E94E95A68E57AE287ED93E0E8
:10C100000E94E95A68E079E48BED93E00E94E95AD5
:10C110006CE978E480EE93E00E94E95A6FEC77E4F2
:10C1200084EE93E00E94E95A6DE977E487EE93E0AC
:10C130000E94E95A6AEB77E48BEE93E00E94E95A99
:10C1400067E977E481EF93E00E94E95A0E94A72D06
:10C150008E010F5F1F4F7E0127E0E20EF11C62EBA4
:10C16000C62E63E0D62E280140E150E060E070E08A
:10C17000C6010E940B6BF80161938F016AE370E0C6
:10C18000C6010E945C78009759F0FC0120812223AF
:10C1900039F06C01FFEFCF1ADF0AE016F10621F744
:10C1A00052E0E52E57E0F52ED12C00E010E0C8015A
:10C1B0000E949173F70181937F0181508E3F10F4AB
:10C1C000DD24D3940F5F1F4F0630110581F7D11086
:10C1D0000EC06CE478E087EA97E00E942E5886E073
:10C1E000F201A2E0B7E001900D928A95E1F70E947A
:10C1F000A15C0E94B14B61E08DE00E94085F26E0E7
:10C2000040E855E260E070E08AE097E00E942F3F4E
:10C210008CE99DE29093080A8093070A84E59AE2EC
:10C2200090930A0A8093090A80E59AE290930C0A97
:10C2300080930B0A64E170E080E090E00E94445F2C
:10C240008CEB9BE59093E4088093E30864EF71E046
:10C2500080E090E00E94445F9E01265A3F4FA096E6
:10C260003FAF2EAFA097A89587EA97E00E94C356EC
:10C27000892BF1F187EA97E00E94A156182F8A30A6
:10C2800029F08D3019F0883009F513C0E091D305FD
:10C29000F0E0E956FA4F108268EF73E087EA97E022
:10C2A0000E94FC5887E995E00E942A5B1092D30512
:10C2B000DBCF68E087EA97E00E94E9578091D305D9
:10C2C000882391F281508093D305CECF682F87EADF
:10C2D00097E00E94E957E091D305EB3328F681E01F
:10C2E0008E0F8093D305F0E0E956FA4F1083BCCF50
:10C2F0000E943F11029714F00E943F4D0E94C229F4
:10C300008091EE059091EF05892B09F4D2C48091BC
:10C31000950590919605049709F4C1C30E947E5F2C
:10C320000091D4051091D5052091D6053091D705FF
:10C33000061717072807390708F0B1C320E02224A1
:10C340002394312C40E1642E712CE0919305F091FF
:10C350009405309709F4A3C32111A1C380858530CA
:10C3600009F086C349E652E063965FAF4EAF63972C
:10C370006596FFAFEEAF6597CE018F5A9F4F0E9433
:10C380007D280E947E5FA4966CAF7DAF8EAF9FAF7D
:10C39000A4976A968FAD6A97843061F008F44AC317
:10C3A000883009F447C3893009F4CFC0853009F0DB
:10C3B00046C340C38091EC059091ED05892B09F0AF
:10C3C000BCC0CE018F5A9F4F0E9442208111B5C040
:10C3D0006796CEACDFAC6797F6018085853009F0B3
:10C3E000D2C4C6010E944B42082F10E00230110552
:10C3F0000CF4C9C43092ED052092EC0560E070E0C9
:10C40000CE018F5A9F4F0E9417285C0161E070E0B7
:10C41000CE018F5A9F4F0E9417287C0105301105CD
:10C420000CF4AEC464E0C6010E94A93EFC01018583
:10C43000128526E240E855E260E070E08AE097E08D
:10C440000E942F3FA092F5088AE097E09093F408AD
:10C450008093F3081092000A1092020A1092010AC7
:10C460000130110509F443C40CF428C4023011054D
:10C4700009F030C4F092F708E092F6083092F9081B
:10C480002092F80883E00E94943FA5968FAFA5976D
:10C49000A596FFADA597F1113BC42091FA08309104
:10C4A000FB08A9963FAF2EAFA997C901330FAA0B7E
:10C4B000BB0B89839A83AB83BC837E826D82659636
:10C4C000EEADFFAD65970081118164ED78E087EAFC
:10C4D00097E00E942E58B80187EA97E00E94FC5826
:10C4E0006DEC78E087EA97E00E942E58B20187EA67
:10C4F00097E00E94D7280E94F858A9966EAD7FADAC
:10C50000A997CE018F5A9F4F0E947C201092ED0573
:10C510001092EC050091930510919405F801828129
:10C52000938129E632E03A8329839C838B83C2017D
:10C530000E947D28012B09F006C4CE018F5A9F4F1F
:10C540000E94402180ED97E07CC28091EC059091A3
:10C55000ED05892B91F7CE018F5A9F4F0E94422003
:10C560008111EBCF3092ED052092EC050E9434351D
:10C570006C01892B19F086E0F601808720E030E01D
:10C5800043E050E060E2C2010E946C556596EEAD5A
:10C59000FFAD6597608171814FE150E0C2010E945B
:10C5A00077786BEF73E0C2010E94517826E040E893
:10C5B00055E260E070E08AE097E00E942F3F60E083
:10C5C00070E0CE018F5A9F4F0E9417288093F50884
:10C5D0008AE097E09093F4088093F3081092000AA1
:10C5E0001092020A1092010A24E338E03093F7080F
:10C5F0002093F6084AE050E05093F9084093F80879
:10C6000083E00E94943F8111BFC06DEA78E087EA21
:10C6100097E00E942E580AEF18E09EE0E92E99E07C
:10C62000F92EF801819191918F01092E000CAA0B2E
:10C63000BB0B25968CAF9DAFAEAFBFAF25972796AE
:10C640007FAE6EAE2797BE016F5B7F4F87EA97E0A4
:10C650000E94D7286BEA78E00E942E58E016F10677
:10C6600001F787EA97E00E94F8586091FE08709100
:10C67000FF08072E000C880B990B0E94547520E0D0
:10C6800030E048EC52E40E94AA749B01AC0161E0E6
:10C6900074E0C6010E949F210091020910910309D4
:10C6A000A80163E074E0C6010E94F53E60910409B0
:10C6B00070910509072E000C880B990B0E94547588
:10C6C00020E030E048EC52E40E94AA749B01AC01E7
:10C6D00067E074E0C6010E949F2160910609709195
:10C6E0000709072E000C880B990B0E94547520E057
:10C6F00030E040E251E40E94AA749B01AC0165E085
:10C7000074E0C6010E949F214091FA085091FB08F5
:10C7100069E074E0C6010E94F53E012B09F450C0A7
:10C7200067968EAD9FAD6797FC012085253009F097
:10C7300047C061E00E94A93E009709F441C024E689
:10C7400030E06E963FAF2EAF6E97FC01618572852B
:10C75000CE018F5B9F4F0E94241ECE018F5B9F4FA7
:10C760000E94AE27882361F1E12CF12C01E09E01AB
:10C77000245A3F4F41E050E060E070E0CE018F5B13
:10C780009F4F0E94BF081CC090E0A0E0B0E025963B
:10C790008CAF9DAFAEAFBFAF259727967FAE6EAE85
:10C7A000279765E978E087EA97E00E942E58BE0156
:10C7B0006F5B7F4F87EA97E00E94D7280E94F85866
:10C7C0008091FA0883FF14C08EE398E09093F708F5
:10C7D0008093F6083092F9082092F80883E00E94CE
:10C7E000943F81110CC04091FA085091FB0802C09F
:10C7F00040E050E06CE074E0C6010E94F53E62E368
:10C8000070E080E090E00E94445F23E130E03093EC
:10C81000F7082093F60844E050E05093F90840935D
:10C82000F80883E00E94943F8111A8C06BE878E08B
:10C8300087EA97E00E942E580AEF18E082E0E82E7F
:10C8400089E0F82EF801619171918F0187EA97E0F4
:10C850000E948F3E69E878E087EA97E00E942E58B0
:10C86000E016F10679F787EA97E00E94F858009100
:10C87000FA081091FB0801151105D1F0B801012E3D
:10C88000000C880B990B0E9454752DEE3EE94CE389
:10C890005EE30E94097622E538EB42E152E40E9411
:10C8A00038749B01AC0160E174E0C6010E949F21D5
:10C8B0006091FC087091FD08072E000C880B990B05
:10C8C0000E9454752DEE3EE94CE35EE30E9409762A
:10C8D00022E538EB42E152E40E9438744B015C01DE
:10C8E0009B01AC016FEF73E0C6010E949F21609134
:10C8F00000097091010916161706A4F4072E000C02
:10C90000880B990B0E94547520E030E040E251E41E
:10C910000E94AA749B01AC0164E174E0C6010E940C
:10C920009F2107C040E050E064E174E0C6010E942E
:10C93000F53E20E030E040E252E4C501B4010E943F
:10C9400004761816ACF5012B99F16596EEADFFADA6
:10C9500065976081718188E194E00E94DC21E12C7F
:10C96000F12C01E020E030E040E050E062E070E0D7
:10C97000CE018F5A9F4F0E94BF081AC090E0A0E0DE
:10C98000B0E025968CAF9DAFAEAFBFAF2597279691
:10C990007FAE6EAE279763E778E087EA97E00E9464
:10C9A0002E58BE016F5B7F4F87EA97E00E94D72821
:10C9B00080E091E00E9448698C01892B61F1259605
:10C9C0001FAE1EAE259727961FAE1EAE27978FEF80
:10C9D0009FEF29969FAF8EAF29978DE392E0239624
:10C9E0009FAF8EAF23972B961FAE1EAE2B972D9623
:10C9F0001FAF0EAF2D9780E091E061969FAF8EAF95
:10CA000061972F961FAE1EAE2F97B601CE018F5B9A
:10CA10009F4F0E943D33B801C2010E94DC21C80132
:10CA20000E94E069C6010E94E7211092ED05109274
:10CA3000EC0583CDCE018F5A9F4F0E94402184E6A2
:10CA400090E0092E000CAA0BBB0BA4968CAC9DACFD
:10CA5000AEACBFACA497880E991EAA1EBB1E8092D6
:10CA6000D4059092D505A092D605B092D70521E0C5
:10CA7000E0919305F09194058281938190939405C0
:10CA800080939305892B09F060CCE091EE05F0913D
:10CA9000EF058681978190939405809393050E947A
:10CAA0007E5F0091D8051091D9052091DA0530916B
:10CAB000DB05601771078207930708F4FAC0E0915D
:10CAC000EE05F091EF05309709F4F3C0268037802A
:10CAD000F12C2114310441F1F1018085853001F5FB
:10CAE00060E0C1010E94A93EFC0181859285A38579
:10CAF000B4850597A105B10599F4C1010E944B4287
:10CB000090E005976CF064E0C1010E94A93E3C01F1
:10CB1000892B31F0C3010E944B42823008F059C189
:10CB2000F10122803380D5CF0E947E5FDC01CB01F2
:10CB300088579C4EAF4FBF4F8093D8059093D9052F
:10CB4000A093DA05B093DB050091B50A1091B60AFF
:10CB50000115110511F401EC1AE00E947E5F4B01F2
:10CB60005C010E94AE1F882309F460C020E030E021
:10CB700041E050E060E4C2010E946C5540E450E0A6
:10CB800064E179E0C2010E94486C60EB73E0C2018D
:10CB90000E94517840E450E06BE079E0C2010E94CD
:10CBA000486CA0964EAD5FADA097401B510B052E73
:10CBB000000C660B770BCE018F5B9F4F0E941155C7
:10CBC000BE016F5B7F4FC2010E94372020E030E042
:10CBD00041E050E060E4C2010E946C5540E450E046
:10CBE00064E179E0C2010E94486C60EB73E0C2012D
:10CBF0000E94517840E450E064E079E0C2010E9474
:10CC0000486CC501B40128EE33E040E050E00E94DA
:10CC1000B773BA01A901CE018F5B9F4F0E941155D6
:10CC2000BE016F5B7F4FC2010E9437208091B50A21
:10CC30009091B60AFF20F9F0009711F08C0102C024
:10CC400001EC1AE06FE179E087EA97E00E942E5844
:10CC5000A201401B510B052E000C660B770B2AE03E
:10CC600087EA97E00E94675861E374E087EA97E0FB
:10CC70000E94FC581EC0009711F08C0102C001EC0C
:10CC80001AE06DE179E087EA97E00E942E58A20150
:10CC9000401B510B052E000C660B770B2AE087EA30
:10CCA00097E00E9467586BE179E087EA97E00E947D
:10CCB0002E580E94B62A0E947457D5CA012B09F536
:10CCC000F092F708E092F6083092F9082092F808FE
:10CCD00081E0D9CB03301105A1F4F092F708E0927E
:10CCE000F6083092F9082092F80884E0CCCBF09254
:10CCF000F708E092F6081093F9080093F80882E02C
:10CD0000C2CB69ED78E087EA97E00E942E58C0CB4D
:10CD1000A5963FADA597832F90E0A0E0B0E0898372
:10CD20009A83AB83BC837E826D8267EB78E087EA6F
:10CD300097E00E942E58B20187EA97E00E94D72818
:10CD40000E94F858E3CBC2010E94AE27882309F461
:10CD5000F4CB8985843009F0F0CB60E070E0C2014B
:10CD60000E941728A816B90609F0E7CB61E070E029
:10CD7000C2010E941728E816F90609F0DECB0AC0A6
:10CD800002E010E056CB61EF78E087EA97E00E947E
:10CD90002E58D3CBA9966EAD7FADA997C2010E9444
:10CDA0007C20E0919305F09194058281938190938A
:10CDB000940580939305892B09F0BFCBE091EE0594
:10CDC000F091EF0586819781909394058093930568
:10CDD000B4CB61E0C1010E94A93EFC01118502852E
:10CDE00062E0C1010E94A93EFC01C184D284E384B7
:10CDF000F48463E0C1010E94A93EFC0121853285D3
:10CE000043855485AD962CAF3DAF4EAF5FAFAD9728
:10CE100060E0C3010E94A93EFC0181849284A38446
:10CE2000B48461E0C3010E94A93EFC0141855285A2
:10CE300063857485411551056105710571F4F10132
:10CE40006081718187EA97E00E94FC5865E579E08E
:10CE500087EA97E00E942E5814C041505109610999
:10CE60007109FC014187528763877487452B462BE4
:10CE7000472B39F4F1016081718185E294E00E94D1
:10CE8000DC2120E030E048E152E4C501B4010E9419
:10CE9000047618163CF4F1016081718188E194E018
:10CEA0000E94DC21A1961FAFA197A2960FAFA29777
:10CEB000C701B6010E9454756B017C01AB962EAD83
:10CEC0003FADAB97A7963FAF2EAFA797F10101906B
:10CED000F081E02DAF96FFAFEEAFAF9787EA97E016
:10CEE0000E94F858AF966EAD7FADAF9787EA97E096
:10CEF0000E94FC586FE479E087EA97E00E942E5880
:10CF000042E0C701B6010E94502269E479E087EA55
:10CF100097E00E942E5842E0C501B4010E945022C1
:10CF200063E479E087EA97E00E942E58AB966EADF5
:10CF30007FADAB9787EA97E00E948F3EA2962EAD19
:10CF40003FADA29761E0812F37FF0CC081950E9411
:10CF5000085FA7964EAD5FADA7974230510509F027
:10CF600074C022C00E94085FA7968EAD9FADA797A0
:10CF70000297F9F0A7964EAD5FADA79745305105E2
:10CF8000C1F061E0C3010E94A93EFC018185928548
:10CF9000A385B485892B8A2B8B2B91F4A2962EAD79
:10CFA0003FADA29737FF05C060E0812F81950E94B9
:10CFB000B03C60E0812F0E94B03C6EE379E021C07C
:10CFC00020E030E040E85FE3C701B6010E9438741A
:10CFD0009B01AC01C501B4010E94A57487FF18C074
:10CFE000A2962EAD3FADA29737FF05C060E0812F1E
:10CFF00081950E94B03C61E0812F0E94B03C6AE3C1
:10D0000079E087EA97E00E942E58FF24F39488CDB8
:10D01000A5019401C701B6010E94A574181694F0E9
:10D02000A2964EAD5FADA29757FF05C061E0812F7C
:10D0300081950E94B03C60E0812F0E94B03C65E386
:10D0400079E0DFCF66E279E0DCCFA7968EAD9FADC9
:10D05000A797059709F095CFA7CFEAE0F7E01382ED
:10D06000128248EE53E060E070E0448355836683AB
:10D0700077838FE892E09183808325ED30E03587D8
:10D08000248724ED30E03787268720ED30E0318B90
:10D09000208B21ED30E0338B228B22ED30E0358B7D
:10D0A000248B26ED30E0378B268B118E128E138E5B
:10D0B000148EE7EAF7E01382128244835583668375
:10D0C00077839183808385EC90E09587848784ECD7
:10D0D00090E09787868780EC90E0918B808B81EC45
:10D0E00090E0938B828B82EC90E0958B848B86EC26
:10D0F00090E0978B868B118E128E138E148EEAE140
:10D10000FAE08FE093E0918380831282138214828D
:10D110001582E0E2FAE09183808312821382148206
:10D120001582E6E2FAE091838083128213821482F0
:10D130001582E4E4F8E091838083128213821482E2
:10D140001582ECE2FAE091838083128213821482CA
:10D150001582E2E3FAE091838083128213821482C3
:10D160001582E8E3FAE091838083128213821482AD
:10D170001582EEE3FAE09183808312821382148297
:10D180001582EAE4F8E0918380831282138214828C
:10D190001582E4E4FAE09183808312821382148280
:10D1A0001582EAE4FAE0918380831282138214826A
:10D1B0001582EDE0FAE01382128244835583668380
:10D1C000778329EE32E03183208324E02487109294
:10D1D000080A1092070A10920A0A1092090A10927D
:10D1E0000C0A10920B0AA2E5B8E013961C921E924C
:10D1F000129721EA32E011963C932E939093E60821
:10D200008093E5081092E7081092E8081092E90868
:10D210001092EA082FEF3FEF3093F2082093F108C5
:10D220001596FC93EE9314971092F0081092EF0865
:10D23000E0E5FAE0918380831282138214821582E2
:10D24000E6E5FAE0918380831282138214821582CC
:10D25000ECE5FAE0918380831282138214821582B6
:10D26000E2E6FAE0918380831282138214821582AF
:10D27000E8E6FAE08FEF808312821182148613862B
:10D280008FEF9FEFDC0187839087A187B287089596
:10D290000F931F93CF93DF938230910510F482E0B8
:10D2A00090E0E091B70AF091B80A20E030E0A0E009
:10D2B000B0E0309719F14081518102811381481704
:10D2C0005907C8F08417950769F4109731F0129642
:10D2D0000C93129713961C9327C00093B70A1093D0
:10D2E000B80A22C02115310519F04217530718F466
:10D2F0009A01BD01EF01DF01F801DBCF21153105F6
:10D30000F9F0281B390B2430310580F48A819B8188
:10D310006115710521F0FB019383828304C0909312
:10D32000B80A8093B70AFE01329644C0FE01E20FAC
:10D33000F31F8193919322503109398328833AC096
:10D340002091B50A3091B60A232B41F420910A02AC
:10D3500030910B023093B60A2093B50A209108024F
:10D36000309109022115310541F42DB73EB74091A6
:10D370000C0250910D02241B350BE091B50AF0917F
:10D38000B60AE217F307A0F42E1B3F0B2817390744
:10D3900078F0AC014E5F5F4F2417350748F04E0F11
:10D3A0005F1F5093B60A4093B50A8193919302C0D0
:10D3B000E0E0F0E0CF01DF91CF911F910F91089550
:10D3C000CF93DF93009709F481C0FC013297138259
:10D3D0001282A091B70AB091B80A109781F4208107
:10D3E0003181820F931F2091B50A3091B60A281718
:10D3F000390751F5F093B60AE093B50A67C0ED011D
:10D4000020E030E0CE17DF0740F44A815B819E01C7
:10D4100041155105F1F0EA01F5CFD383C283408174
:10D420005181840F951FC817D90759F488819981B4
:10D43000840F951F0296918380838A819B819383B9
:10D4400082832115310529F4F093B80AE093B70AD5
:10D450003DC0E901FB83EA8349915991C40FD51F6F
:10D46000EC17FD0761F480819181840F951F02966E
:10D47000E90199838883828193819B838A83E0E099
:10D48000F0E012968D919C911397009719F0FD0191
:10D49000DC01F7CF8D919C9111979D012E5F3F4F3D
:10D4A000820F931F2091B50A3091B60A28173907C9
:10D4B00069F4309729F41092B80A1092B70A02C0A2
:10D4C00013821282B093B60AA093B50ADF91CF916E
:10D4D00008958F929F92AF92BF92CF92DF92EF9278
:10D4E000FF92CF93DF93EC01688179818A819B81E0
:10D4F000611571058105910521F464E279ED8BE5F3
:10D5000097E02DE133EF41E050E00E94D9734901EB
:10D510005A019B01AC01A7EAB1E40E94F8736B01C8
:10D520007C01ACEEB4EFA50194010E940674DC010D
:10D53000CB018C0D9D1DAE1DBF1DB7FF03C0019714
:10D54000A109B04888839983AA83BB83BC01CD011C
:10D550009F77DF91CF91FF90EF90DF90CF90BF90BA
:10D56000AF909F908F9008958F929F92AF92BF92AD
:10D57000CF92DF92EF92FF9260910E0270910F02B4
:10D58000809110029091110261157105810591053C
:10D5900021F464E279ED8BE597E02DE133EF41E092
:10D5A00050E00E94D97349015A019B01AC01A7EADE
:10D5B000B1E40E94F8736B017C01ACEEB4EFA501FD
:10D5C00094010E940674DC01CB018C0D9D1DAE1DE3
:10D5D000BF1DB7FF03C00197A109B04880930E0299
:10D5E00090930F02A0931002B0931102BC01CD01E1
:10D5F0009F77FF90EF90DF90CF90BF90AF909F907C
:10D600008F90089560930E0270930F028093100222
:10D610009093110208953F924F925F926F927F9282
:10D620008F929F92AF92BF92CF92DF92EF92FF9232
:10D630000F931F93CF93DF935C016B017A01611508
:10D64000710519F0FB0191838083E114F10429F045
:10D65000C7010297839708F0C9C0E5012196F5013B
:10D660001081812F90E00E94366C892B11F05E01B1
:10D67000F4CF1D3229F42196F501118101E007C094
:10D680001B3221F4E5012296F501118100E0E1143D
:10D69000F104B1F0F0E1EF16F10429F4B0C010E3A9
:10D6A000E114F10401F12AE0E216F104B1F180E1A4
:10D6B000E816F10471F0E8E0EE16F104F1F413C09D
:10D6C000103341F588818F7D883549F7198122967D
:10D6D0000260F0E1EF2EF12C88248A94982CA82C7B
:10D6E000AFE0BA2E20C078E0E72EF12C88248A948F
:10D6F000982CA82CEFE1BE2E16C06FEF7FEFCB0168
:10D7000097010F2C000C440B550B0E94B773490175
:10D710005A0109C08AE0E82EF12C69E9862E982C7E
:10D72000A82C69E1B62E40E060E070E0CB01270153
:10D730000F2C000C66087708FE0150ED352E310ED7
:10D7400029E0231570F42FEB210F2A3118F439EC5E
:10D75000332E06C02FE9210F2A3130F529EA322E67
:10D76000310E232D30E02E153F05F4F44F3FC9F064
:10D7700086169706A806B90688F0A30192010E94B2
:10D78000A773232D30E040E050E0620F731F841F29
:10D79000951F621773078407950710F44FEF01C0B8
:10D7A00041E021961081C8CFC114D10451F0442327
:10D7B00011F0219703C001FF04C02297F601D18325
:10D7C000C08300FF07C090958095709561957F4F4D
:10D7D0008F4F9F4F4F3F79F482E290E09093C00AC1
:10D7E0008093BF0A3FEF2FEF9FEF0DC040E030E086
:10D7F00020E090E008C0462F372F282F04C01033B8
:10D8000009F067CF5FCF642F732F822FDF91CF9105
:10D810001F910F91FF90EF90DF90CF90BF90AF904E
:10D820009F908F907F906F905F904F903F90089562
:10D83000FC0188279927E89421912032E9F32930C7
:10D8400010F02E30C8F32B3241F02D3239F46894A9
:10D8500004C00E949D6C820F911D219120532A309B
:10D86000C0F31EF4909581959F4F089591110C94EB
:10D87000A372803219F089508550C8F70895FB01D2
:10D88000DC018D91059080190110D9F3990B089551
:10D89000FB01DC010D900020E9F711974150504049
:10D8A00028F0059000200D92C9F708951C92089564
:10D8B000FB01DC014150504048F005900D920020E2
:10D8C000C9F701C01D9241505040E0F7089543EB65
:10D8D0005AE00C946B6CFA01A191B081009719F495
:10D8E0001097E1F0CD01DC01CD010D90002011F485
:10D8F000C00113C0FB012191222319F02015D9F793
:10D90000F3CFFB012191201519F41E92119606C048
:10D910002223C1F70D900020A1F7D001FA01A193B5
:10D92000B0830895BB274A3031F4992322F4BDE235
:10D93000909581959F4F0C94A66C7AE0979F902DBF
:10D94000879F802D910D11240895BB27FB0155273A
:10D95000AA27880F991FAA1FA41710F0A41B83954C
:10D960005051B9F7A05DAA3308F0A95DA1930097C3
:10D9700079F7B111B1931192CB010C94CE72FC01E5
:10D98000238127FF10C0E9EBFAE020813181821763
:10D99000930711F41182108232962AE0EF3BF207CE
:10D9A000A1F70E94E06980E090E008950F931F9333
:10D9B000CF93DF93009731F46115710519F480E07E
:10D9C00090E03AC08B01EC016EE070E081E090E005
:10D9D0000E948772FC01892B91F380E883830115F3
:10D9E000110571F01387028781E883838091B90A5A
:10D9F0009091BA0A892B21F4F093BA0AE093B90AFC
:10DA00002097C9F0D187C08783818260838380910A
:10DA1000BB0A9091BC0A892B71F4F093BC0AE09385
:10DA2000BB0A8091BD0A9091BE0A892B21F4F09324
:10DA3000BE0AE093BD0ACF01DF91CF911F910F91F4
:10DA40000895CF93DF93EC012B8120FF33C026FF95
:10DA50000AC02F7B2B838E819F8101969F838E83AB
:10DA60008A8190E029C022FF0FC0E881F98180817E
:10DA7000082E000C990B009719F420622B831AC012
:10DA80003196F983E8830EC0EA85FB85199597FFE7
:10DA900009C02B81019611F080E201C080E1822B48
:10DAA0008B8308C02E813F812F5F3F4F3F832E83A2
:10DAB000992702C08FEF9FEFDF91CF9108950F93C9
:10DAC0001F93CF93DF93CDB7DEB708851985F80193
:10DAD000838188608383AE01445F5F4F6A857B8565
:10DAE000C8010E94996DF8012381277F2383DF916C
:10DAF000CF911F910F9108950F931F93CF93DF93B1
:10DB0000CDB7DEB708851985F801838188608383E6
:10DB1000AE01445F5F4F6A857B85C8010E946271D8
:10DB2000F8012381277F2383DF91CF911F910F91EC
:10DB300008952F923F924F925F926F927F928F92B1
:10DB40009F92AF92BF92CF92DF92EF92FF920F938C
:10DB50001F93CF93DF93CDB7DEB72B970FB6F89413
:10DB6000DEBF0FBECDBF6C017B018A01FC011782B5
:10DB70001682838181FFCCC1CE0101963C01F60162
:10DB80009381F70193FD859193FF81917F01882314
:10DB900009F4BAC1853239F493FD859193FF8191DF
:10DBA0007F01853229F4B60190E00E94DE72E7CF52
:10DBB000912C212C312CFFE1F315D8F08B3279F028
:10DBC00038F4803279F08332A1F4232D20611DC016
:10DBD0008D3261F0803369F4232D216016C0832DCE
:10DBE0008260382EE32DE4603E2E2AC0F32DF860CB
:10DBF0001DC037FC2DC020ED280F2A3040F08E329A
:10DC0000B9F436FC81C1232D2064322E19C036FEB2
:10DC100006C08AE0989E200D1124922E11C0EAE0E1
:10DC20002E9E200D1124222EF32DF0623F2E08C0CF
:10DC30008C3621F4832D8068382E02C0883641F45A
:10DC4000F70193FD859193FF81917F018111B3CFFE
:10DC5000982F9F7D9554933028F40C5F1F4F9FE3BE
:10DC600099830DC0833631F0833771F0833509F025
:10DC700059C021C0F801808189830E5F1F4F88241D
:10DC80008394912C530113C02801F2E04F0E511CD4
:10DC9000F801A080B18036FE03C0692D70E002C09B
:10DCA0006FEF7FEFC5010E94C3724C018201F32D1B
:10DCB000FF773F2E16C0280122E0420E511CF801CA
:10DCC000A080B18036FE03C0692D70E002C06FEF06
:10DCD0007FEFC5010E94B1724C01F32DF0683F2E19
:10DCE000820133FC1BC0822D90E088169906B0F4A7
:10DCF000B60180E290E00E94DE722A94F4CFF50132
:10DD000037FC859137FE81915F01B60190E00E945A
:10DD1000DE7221102A9421E0821A91088114910464
:10DD200071F7E8C0843611F0893641F5F80137FE05
:10DD300007C060817181828193810C5F1F4F08C091
:10DD400060817181072E000C880B990B0E5F1F4FAD
:10DD5000F32DFF763F2E97FF09C090958095709523
:10DD600061957F4F8F4F9F4FF0683F2E2AE030E044
:10DD7000A3010E943373882E861845C0853731F47D
:10DD8000232D2F7EB22E2AE030E025C0932D997FDF
:10DD9000B92E8F36C1F018F4883579F0B5C08037C8
:10DDA00019F0883721F0B0C0E92FE061BE2EB4FE33
:10DDB0000DC0FB2DF460BF2E09C034FE0AC0292F10
:10DDC0002660B22E06C028E030E005C020E130E039
:10DDD00002C020E132E0F801B7FE07C06081718126
:10DDE000828193810C5F1F4F06C06081718180E04A
:10DDF00090E00E5F1F4FA3010E943373882E861898
:10DE0000FB2DFF773F2E36FE0DC0232D2E7FA22E39
:10DE1000891458F434FE0BC032FC09C0832D8E7E69
:10DE2000A82E05C0B82CA32C03C0B82C01C0B92C57
:10DE3000A4FE0FC0FE01E80DF11D8081803321F4A6
:10DE40009A2D997EA92E09C0A2FE06C0B394B39460
:10DE500004C08A2D867809F0B394A3FC11C0A0FEFB
:10DE600006C0B21488F4280C922C9B180EC0B21471
:10DE700060F4B60180E290E00E94DE72B394F7CFC6
:10DE8000B21418F42B1802C0982C212CA4FE10C038
:10DE9000B60180E390E00E94DE72A2FE17C0A1FCF2
:10DEA00003C088E790E002C088E590E0B6010CC0AE
:10DEB0008A2D867859F0A1FE02C08BE201C080E273
:10DEC000A7FC8DE2B60190E00E94DE72891438F45E
:10DED000B60180E390E00E94DE729A94F7CF8A94B4
:10DEE000F301E80DF11D8081B60190E00E94DE7221
:10DEF0008110F5CF222009F442CEB60180E290E0F5
:10DF00000E94DE722A94F6CFF6018681978102C0C4
:10DF10008FEF9FEF2B960FB6F894DEBF0FBECDBFED
:10DF2000DF91CF911F910F91FF90EF90DF90CF90F5
:10DF3000BF90AF909F908F907F906F905F904F9029
:10DF40003F902F90089520FD09C0FC0123FD05C0DE
:10DF500022FF02C07383628351834083089544FD8E
:10DF600017C046FD17C0AB01BC01DA01FB01AA0FC7
:10DF7000BB1FEE1FFF1F1094D1F74A0F5B1F6E1FD0
:10DF80007F1FCB01BA01660F771F881F991F09C039
:10DF900033E001C034E0660F771F881F991F3150AE
:10DFA000D1F7620F711D811D911D08950F931F936D
:10DFB000CF93DF938C01C8010E94216DEC0197FD86
:10DFC00008C00E94366C892BB1F7B801CE010E94BF
:10DFD0001A73CE01DF91CF911F910F9108958F9207
:10DFE0009F92AF92BF92EF92FF920F931F93CF93A6
:10DFF000DF938C01D62F7A01B22E0E94216D9C01F5
:10E0000033272B32310531F02D32310561F48B2D60
:10E010008068B82ED15011F480E068C0C8010E9419
:10E02000216D97FDF9CFCB2DCD7F2B2D207309F5D9
:10E030008033F9F4AA24AA94AD0E09F443C0C801B0
:10E040000E94216D97FD3EC09C012F7D332728350E
:10E05000310549F4C264D250A9F1C8010E94216D72
:10E0600097FF07C02FC0B6FE02C0C26001C0C261E8
:10E07000DA2D812C912C540120ED280F283080F0CE
:10E08000C4FF04C0B8010E941A7319C02A3040F0BE
:10E09000C6FFF8CF2F7D3FEE320F363098F727506E
:10E0A0004C2FC501B4010E94AF6F4B015C01C260EF
:10E0B000D15059F0C8010E94216D97FFDDCFC1FDFD
:10E0C00004C0AACF812C912C5401C7FF08C0B09482
:10E0D000A09490948094811C911CA11CB11C2C2FA5
:10E0E000B501A401C7010E94A36F81E0DF91CF9128
:10E0F0001F910F91FF90EF90BF90AF909F908F90E6
:10E1000008955F926F927F928F929F92AF92BF928B
:10E11000CF92DF92EF92FF920F931F93CF93DF93F3
:10E12000CDB7DEB7A0970FB6F894DEBF0FBECDBF58
:10E130005C01962E7A01F9018E010F5F1F4F680175
:10E1400080E2D8011D928A95E9F7D50113968C904B
:10E1500080E090E0612C712C30E061E070E083FCA5
:10E16000259183FE21918F01522E211103C080E061
:10E1700090E092C02E3511F4009751F1432F50E0FA
:10E18000481759073CF42D3559F12D3219F47720F1
:10E1900009F103C0772009F46AC0452D46954695DC
:10E1A0004695D601A40FB11D452D47708B0102C0C5
:10E1B000000F111F4A95E2F7A8015C91452B4C9383
:10E1C000651459F0561410F45394E7CF5A94E5CFE0
:10E1D00031E004C07724739401C0712C0196BFCF45
:10E1E000772019F08E8180628E83311103C08824DC
:10E1F000839417C0F6019E012F5D3F4F808180956B
:10E2000081932E173F07D1F7F2CFE114F10429F0E3
:10E21000D7018C93F70131967F019A94812C992034
:10E22000F9F0C5010E94216D97FD18C0FC01FF2780
:10E2300023E0F595E7952A95E1F7EC0DFD1D20818A
:10E2400030E0AC014770552702C0359527954A95B7
:10E25000E2F720FDDACFB5010E941A73811087CF53
:10E26000E114F10411F0D7011C92C80115C0422F2E
:10E27000469546954695D601A40FB11D422F47708D
:10E280008B0102C0000F111F4A95E2F7A8015C91B3
:10E29000452B4C93622EA2CFA0960FB6F894DEBF0A
:10E2A0000FBECDBFDF91CF911F910F91FF90EF90E7
:10E2B000DF90CF90BF90AF909F908F907F906F90A6
:10E2C0005F9008955F926F927F928F929F92AF922C
:10E2D000BF92CF92DF92EF92FF920F931F93CF9353
:10E2E000DF936C01EB015A01FC0117821682512C5D
:10E2F000F601E380FE01E3FC8591E3FE8191182F96
:10E30000EF01882309F4EEC090E00E94366C892B5F
:10E3100021F0C6010E94D66FEBCF153241F4FE0109
:10E32000E3FC1591E3FE1191EF01153281F4C60172
:10E330000E94216D97FDD4C0412F50E09C013327EE
:10E3400024173507A9F2B6010E941A73CBC01A32FE
:10E3500039F4E3FC1591E3FE1191EF0101E001C0F6
:10E3600000E0F12C20ED210F2A3080F402606F2DA7
:10E3700070E080E090E040E20E94AF6FF62EFE0178
:10E38000E3FC1591E3FE1191EF01ECCF01FF03C017
:10E39000F11003C0A7C0FF24FA94183619F01C36F8
:10E3A00051F010C0FE01E3FC1591E3FE1191EF0165
:10E3B000183641F408600460FE01E3FC1591E3FEA9
:10E3C0001191EF01112309F48DC0612F70E08EEEE1
:10E3D00094E00E94A672892B09F484C000FD07C056
:10E3E000F50180809180C50102965C0102C0812CFC
:10E3F000912C1E3651F4F6014681578160E070E0A1
:10E40000202FC4010E94A36F73CF1336A9F401FD1E
:10E4100002C0FF24F394C6010E94216D97FD60C0E5
:10E420008114910429F0F4018083C40101964C0108
:10E43000FA94F110F0CF50C01B3559F49E01A4019D
:10E440006F2DC6010E948170EC01892B09F044C038
:10E450003EC0C6010E94D66F97FD42C01F3661F1D3
:10E4600028F4143639F1193651F128C0133771F0F8
:10E47000153701F123C08114910429F0F401608261
:10E48000C40101964C01FA94FF2071F0C6010E946C
:10E49000216D3C0197FD08C00E94366C892B59F311
:10E4A000B601C3010E941A7381149104A9F0F4010A
:10E4B000108212C0006203C0006101C00064202FFE
:10E4C000A4016F2DC6010E94EF6F811105C0F601F6
:10E4D0008381807329F406C000FD0ACF539408CFCE
:10E4E000552019F0852D90E002C08FEF9FEFDF914E
:10E4F000CF911F910F91FF90EF90DF90CF90BF9041
:10E50000AF909F908F907F906F905F9008950F9342
:10E510001F93CF93DF93869F8001879F100D969F57
:10E52000100D1124C8010E944869EC01009729F0E0
:10E53000A80160E070E00E94BC72CE01DF91CF9133
:10E540001F910F910895992788270895FC01059040
:10E55000061621F00020D9F7C00108953197CF01A8
:10E560000895FC010590615070400110D8F7809526
:10E5700090958E0F9F1F0895DC0101C06D9341504F
:10E580005040E0F70895FC01615070400190011087
:10E59000D8F7809590958E0F9F1F0895DC01FC01A0
:10E5A000672F71917723E1F7329704C07C916D93C7
:10E5B00070836291AE17BF07C8F308950F931F933E
:10E5C000CF93DF93FB01238121FD03C08FEF9FEFEA
:10E5D0002CC022FF16C04681578124813581421705
:10E5E000530744F4A081B1819D012F5F3F4F3183D8
:10E5F00020838C93268137812F5F3F4F378326837B
:10E6000014C08B01EC01FB010084F185E02D19950C
:10E61000892BE1F6D80116968D919C91179701965A
:10E6200017969C938E931697CE01DF91CF911F91F1
:10E630000F910895FB01238120FF12C026FD10C019
:10E640008F3F3FEF930761F082832F7D2064238308
:10E6500026813781215031093783268399270895F0
:10E660008FEF9FEF0895FA01AA27283051F120314A
:10E6700081F1E8946F936E7F6E5F7F4F8F4F9F4F56
:10E68000AF4FB1E03ED0B4E03CD0670F781F891F98
:10E690009A1FA11D680F791F8A1F911DA11D6A0F66
:10E6A000711D811D911DA11D20D009F468943F9119
:10E6B0002AE0269F11243019305D3193DEF6CF0118
:10E6C0000895462F4770405D4193B3E00FD0C9F7DE
:10E6D000F6CF462F4F70405D4A3318F0495D31FD4B
:10E6E0004052419302D0A9F7EACFB4E0A69597959E
:10E6F000879577956795BA95C9F700976105710574
:10E7000008959B01AC010A2E0694579547953795BD
:10E710002795BA95C9F7620F731F841F951FA01D17
:10E720000895F999FECF92BD81BDF89A992780B5D9
:10E730000895262FF999FECF1FBA92BD81BD20BD45
:10E740000FB6F894FA9AF99A0FBE01960895DB0174
:10E750008F939F930E94F873BF91AF91A29F800DFA
:10E76000911DA39F900DB29F900D11240895A1E2D9
:10E770001A2EAA1BBB1BFD010DC0AA1FBB1FEE1F3B
:10E78000FF1FA217B307E407F50720F0A21BB30B86
:10E79000E40BF50B661F771F881F991F1A9469F702
:10E7A00060957095809590959B01AC01BD01CF015E
:10E7B0000895052E97FB1EF400940E94F07357FDF8
:10E7C00007D00E94B77307FC03D04EF40C94F0738B
:10E7D00050954095309521953F4F4F4F5F4F08958D
:10E7E00090958095709561957F4F8F4F9F4F0895BD
:10E7F0000E940B74A59F900DB49F900DA49F800D57
:10E80000911D11240895B7FF0C94F8730E94F873BA
:10E81000821B930B0895A29FB001B39FC001A39FD9
:10E82000700D811D1124911DB29F700D811D112449
:10E83000911D0895EE0FFF1F881F8BBF0790F69163
:10E84000E02D199469279627692778278727782745
:10E8500008950E940B74332312F48A1B9B0B0C94B3
:10E8600033740E940B74B7FF0895821B930B0895B5
:10E870005058BB27AA270E9450740C94CA750E9456
:10E88000BC7538F00E94C37520F039F49F3F19F42D
:10E8900026F40C94B9750EF4E095E7FB0C94B3756F
:10E8A000E92F0E94DB7558F3BA17620773078407D4
:10E8B000950720F079F4A6F50C94FD750EF4E0951B
:10E8C0000B2EBA2FA02D0B01B90190010C01CA012A
:10E8D000A0011124FF27591B99F0593F50F4503ED5
:10E8E00068F11A16F040A22F232F342F4427585FC7
:10E8F000F3CF469537952795A795F0405395C9F7DF
:10E900007EF41F16BA0B620B730B840BBAF0915096
:10E91000A1F0FF0FBB1F661F771F881FC2F70EC035
:10E92000BA0F621F731F841F48F487957795679508
:10E93000B795F7959E3F08F0B0CF9395880F08F0F4
:10E940009927EE0F9795879508950E948F7508F483
:10E9500081E008950E94BE740C94CA750E94C3752C
:10E9600058F00E94BC7540F029F45F3F29F00C94E8
:10E97000B37551110C94FE750C94B9750E94DB753A
:10E9800068F39923B1F3552391F3951B550BBB27DE
:10E99000AA2762177307840738F09F5F5F4F220F23
:10E9A000331F441FAA1FA9F335D00E2E3AF0E0E81A
:10E9B00032D091505040E695001CCAF72BD0FE2F64
:10E9C00029D0660F771F881FBB1F261737074807F8
:10E9D000AB07B0E809F0BB0B802DBF01FF279358B0
:10E9E0005F4F3AF09E3F510578F00C94B3750C944C
:10E9F000FE755F3FE4F3983ED4F38695779567956F
:10EA0000B795F7959F5FC9F7880F911D96958795E4
:10EA100097F90895E1E0660F771F881FBB1F621703
:10EA200073078407BA0720F0621B730B840BBA0BC1
:10EA3000EE1F88F7E09508950E9423756894B11140
:10EA40000C94FE7508950E94E37588F09F5798F026
:10EA5000B92F9927B751B0F0E1F0660F771F881FE3
:10EA6000991F1AF0BA95C9F714C0B13091F00E94FD
:10EA7000FD75B1E008950C94FD75672F782F8827F8
:10EA8000B85F39F0B93FCCF3869577956795B39524
:10EA9000D9F73EF490958095709561957F4F8F4F93
:10EAA0009F4F0895E89409C097FB3EF49095809598
:10EAB000709561957F4F8F4F9F4F9923A9F0F92F44
:10EAC00096E9BB279395F695879577956795B795C2
:10EAD000F111F8CFFAF4BB0F11F460FF1BC06F5FA8
:10EAE0007F4F8F4F9F4F16C0882311F096E911C0BA
:10EAF000772321F09EE8872F762F05C0662371F0DB
:10EB000096E8862F70E060E02AF09A95660F771FEE
:10EB1000881FDAF7880F9695879597F90895990FCA
:10EB20000008550FAA0BE0E8FEEF16161706E807D7
:10EB3000F907C0F012161306E407F50798F0621BF8
:10EB4000730B840B950B39F40A2661F0232B242BCD
:10EB5000252B21F408950A2609F4A140A6958FEFEC
:10EB6000811D811D089597F99F6780E870E060E03E
:10EB700008959FEF80EC089500240A941616170656
:10EB800018060906089500240A941216130614069E
:10EB900005060895092E0394000C11F4882352F001
:10EBA000BB0F40F4BF2B11F460FF04C06F5F7F4FB9
:10EBB0008F4F9F4F089557FD9058440F551F59F0A0
:10EBC0005F3F71F04795880F97FB991F61F09F3F5A
:10EBD00079F087950895121613061406551FF2CF83
:10EBE0004695F1DF08C0161617061806991FF1CFD3
:10EBF00086957105610508940895E894BB276627FA
:10EC00007727CB0197F908950E948F7508F48FEF4D
:10EC100008950E941C760C94CA750E94BC7538F049
:10EC20000E94C37520F0952311F00C94B3750C94D9
:10EC3000B97511240C94FE750E94DB7570F3959FD5
:10EC4000C1F3950F50E0551F629FF001729FBB27E3
:10EC5000F00DB11D639FAA27F00DB11DAA1F649F7F
:10EC60006627B00DA11D661F829F2227B00DA11D32
:10EC7000621F739FB00DA11D621F839FA00D611DB8
:10EC8000221F749F3327A00D611D231F849F600DD9
:10EC9000211D822F762F6A2F11249F5750409AF002
:10ECA000F1F088234AF0EE0FFF1FBB1F661F771F8E
:10ECB000881F91505040A9F79E3F510580F00C9459
:10ECC000B3750C94FE755F3FE4F3983ED4F38695DC
:10ECD00077956795B795F795E7959F5FC1F7FE2BF9
:10ECE000880F911D9695879597F90895FA01EE0F73
:10ECF000FF1F309621053105A1F16115710561F401
:10ED00008038BFE39B0749F168949038810561F032
:10ED10008038BFEF9B0741F099234AF5FF3FE1059B
:10ED20003105210519F1E8940894E795D901AA2342
:10ED300029F4AB2FBE2FF85FD0F310C0FF5F70F443
:10ED4000A695E0F7F73950F019F0FF3A38F49F77BD
:10ED50009F930DD00F9007FC9058089546F00C94A7
:10ED6000B97560E070E080E89FE308954FE79F7712
:10ED70005F934F933F932F930E9476772F913F910C
:10ED80004F915F910E9409760C94D3760E948F7503
:10ED9000880B990B089529F416F00C94B3750C9414
:10EDA000FD750C94B9750E94E375A8F39638A0F729
:10EDB00007F80F92E8942BE33AEA48EB5FE70E94EA
:10EDC0001F760F920F920F924DB75EB70F920E946F
:10EDD000BE77ECEFF1E00E9405774F915F91EF91E4
:10EDE000FF91E595EE1FFF1F49F0FE57E0684427AD
:10EDF000EE0F441FFA95E1F74195550B0E943877C5
:10EE00000F9007FE0C942C770895DF93CF931F93F8
:10EE10000F93FF92EF92DF927B018C01689406C002
:10EE2000DA2EEF010E941C76FE01E894A59125914F
:10EE3000359145915591A6F3EF010E945074FE0162
:10EE40009701A801DA9469F7DF90EF90FF900F9196
:10EE50001F91CF91DF9108959B01AC0160E070E0BC
:10EE600080E89FE30C94AA740C94B3750C94F27729
:10EE70000E94E375D8F39923C9F3940F511DA3F3AE
:10EE80009150504094F059F0882332F0660F771F6C
:10EE9000881F91505040C1F79E3F51052CF7880FB5
:10EEA000911D9695879597F908955F3FACF0983E30
:10EEB0009CF0BB27869577956795B79508F4B16068
:10EEC0009395C1F7BB0F58F711F460FFE8CF6F5F60
:10EED0007F4F8F4F9F4FE3CF0C94FE7516F00C942D
:10EEE000F2770C94B97568940C94B3750E94E3752D
:10EEF000A8F39923C1F3AEF3DF93CF931F930F933E
:10EF0000FF92C92FDD2788232AF02197660F771FEC
:10EF1000881FDAF720E030E040E85FEB9FE38839B4
:10EF200020F0803E38F021968F770E943974E4E219
:10EF3000F2E004C00E943974E1E5F2E00E94057736
:10EF40008B01BE01EC01FB2E6F5771097595771F80
:10EF5000880B990B0E94547528E132E741E35FE387
:10EF60000E941C76AF2D9801AE01FF900F911F916A
:10EF7000CF91DF910E9450740C94CA75FA01DC01A4
:10EF8000AA0FBB1F9B01AC01BF5728F422273327D0
:10EF90004427507820C0B75190F4AB2F00244695F9
:10EFA00037952795011CA395D2F3002071F0220F0D
:10EFB000331F441FB395DAF30ED00C9438746130CC
:10EFC0007105A0E88A07B94630F49B01AC016627B9
:10EFD000772788279078309621F0208331834283E9
:10EFE000538308959F3F31F0915020F48795779592
:10EFF0006795B795880F911D9695879597F9089510
:10F0000081E090E0F8940C943B790F931F93CF9399
:10F01000DF938C01FC0101900020E9F7CF01801BF8
:10F02000910B0E944869EC01009719F0B8010E9409
:10F030007078CE01DF91CF911F910F910895FB0160
:10F04000DC0104C08D910190801921F441505040A1
:10F05000C8F7881B990B08956817790768F4FB01B6
:10F06000DC01E40FF51FA40FB51F02C002900E9241
:10F0700041505040D8F708950C943279FB01DC01DF
:10F080008D9181341CF08B350CF4805E619161347C
:10F090001CF06B350CF4605E861B611189F3990BD3
:10F0A0000895FB01DC010D900020E9F71197019014
:10F0B0000D920020E1F70895FC018191861721F05F
:10F0C0008823D9F7992708953197CF010895FB0137
:10F0D000DC018D91019080190110D9F3990B0895ED
:10F0E000FB01DC0101900D920020E1F70895FB0186
:10F0F000DC010D900020E9F711974150504028F0B5
:10F10000019000200D92C9F708951C920895FB010B
:10F11000DC014150504030F08D910190801919F47C
:10F120000020B9F7881B990B0895FB01DC014150C1
:10F13000504048F001900D920020C9F701C01D9287
:10F1400041505040E0F708950F931F93CF93DF9302
:10F15000CDB7DEB72E970FB6F894DEBF0FBECDBF8A
:10F160000E891F89888D998D26E02C831A83098347
:10F1700097FF02C080E090E801979E838D83AE01E7
:10F18000445E5F4F6A8D7B8DCE0101960E94996D22
:10F190004D815E8157FD0AC02F8138854217530784
:10F1A0000CF49A01F801E20FF31F10822E960FB6AD
:10F1B000F894DEBF0FBECDBFDF91CF911F910F91AD
:10F1C00008950F931F93CF93DF93CDB7DEB72E979C
:10F1D0000FB6F894DEBF0FBECDBF0E891F8986E043
:10F1E0008C831A8309838FEF9FE79E838D83AE0103
:10F1F000465E5F4F688D798DCE0101960E94996DB4
:10F20000EF81F885E00FF11F10822E960FB6F8946B
:10F21000DEBF0FBECDBFDF91CF911F910F9108953B
:10F22000CF93DF93CDB7DEB72E970FB6F894DEBF3E
:10F230000FBECDBF85E08C838C899D899A8389839D
:10F24000AE01485E5F4F6E897F89CE0101960E94B4
:10F2500062712E960FB6F894DEBF0FBECDBFDF9160
:10F26000CF910895FB01DC0102C001900D92415045
:0AF270005040D8F70895F894FFCF3E
:10F27A0003100000C00120000000C10A8000010044
:10F28A00000000044D515454040000000000000026
:10F29A000000000000000000000000000000000064
:10F2AA0000000000000000000000000000E93068D3
:10F2BA0056B95BDA302831063136319B31B45B00FE
:10F2CA0000000061316856B95BDA30A2315E32362D
:10F2DA00319B31B45B00000000BF08C72300000067
:10F2EA0000000000000000000061316856B95BDAD6
:10F2FA0030A2314E3236319B31B45B00000000053A
:10F30A0057685692565257C356A156B55600000032
:10F31A0000CE57AB57B95BB85B00000000A957682D
:10F32A0056B95BB85BA957A957A95700000000A9AD
:10F33A00576856B95BB85B00000000A957A957B9CE
:10F34A005BA957A957A957A957A957A957A957A9AF
:10F35A0057A957A95700000000F851A952B95BA450
:10F36A004287526D5246523453FD5569525244EB0C
:10F37A00429C421A52185291420E5200000000F06A
:10F38A005700000000A95701005E000000000000BD
:10F39A00005A42A542B95B59427042AE45F7445001
:10F3AA0046E1464444504760437D46D7458F4588E9
:10F3BA004278427442303132333435363738394143
:10F3CA004243444546000000000020326856B95BBB
:10F3DA00DA307331313236319B31B45B4C6F616450
:10F3EA0065642066726F6D20666C6173682049508F
:10F3FA003A0020444E533A002047573A00204D41E4
:10F40A00534B3A000A4E6F204950206461746120C0
:10F41A00666F756E6420696E20666C6173680A0097
:10F42A002F0064653A61643A62653A65663A6665D0
:10F43A003A65640068656C700073617665006C6F8C
:10F44A00616400676574006D6163006B696C6C00D0
:10F45A007265710069700070776400636C6561722F
:10F46A00007265626F6F74000D0A005F73746174D5
:10F47A0000560052504D004900737700666C7400C4
:10F48A0073657400707772002F616C61726D2F6FF3
:10F49A0076726874002F616C61726D2F736E73726D
:10F4AA000020006E756C6C0066616C736500747286
:10F4BA007565006E616E00696E66006F7666002380
:10F4CA00253258253258253258006974656D007303
:10F4DA00636D640072636D6400656D6974004F4EFC
:10F4EA00004F4646003B0025783A25783A25783A77
:10F4FA0025783A25783A257825D181005400530099
:10F50A006D6170002F253032782D253032782D2507
:10F51A003032782D253032782D253032782D25302D
:10F52A0032782E636F6E6669672E6A736F6E002279
:10F53A00002D002E0025252532780057495A6E6580
:10F54A0074002F726573702F23002F7265712F63F9
:10F55A006F6E66003100646D78696E00646D7800C4
:10F56A006D6F64627573006974656D7300746F7092
:10F57A00696373006D71747400726F6F74006F75D4
:10F58A007400626373740024636F6D6D616E64004E
:06F59A002564002C0000B6
:00000001FF
